:100000000C94761B0C94A01B0C94A01B0C94A01BAE
:100010000C94A01B0C94A01B0C94A01B0C94A01B74
:100020000C94A01B0C94A01B0C94A01B0C94A01B64
:100030000C94A01B0C942F480C94A01B0C94A01B98
:100040000C94A01B0C94BDA20C94FF520C94A01B0A
:100050000C949F430C94A01B0C94A01B0C94A01B0D
:100060000C94A01B0C94A01B0C94A01B0C94A01B24
:100070000C94A01B0C94A01B0C94A01B0C94A01B14
:100080000C94A01B0C94A01B0C94A01BBA513E52C4
:10009000EE51E8510052055232526E52735278526C
:1000A0008252B052B0528C5294529C52A652795FF6
:1000B000825F8C5F955F9E5FB95FC65FCF5FA75F12
:1000C000B05F1160146007600B602B602B601860DC
:1000D0001C60226026604E414E494E495459494E9B
:1000E00046CDCCCC3D0AD7233C17B7D13877CC2BA3
:1000F000329595E6241FB14F0A000020410000C848
:100100004200401C4620BCBE4CCA1B0E5AAEC59DC8
:1001100074434F4D4D554E49434154494F4E004451
:10012000525952554E004552524F525300494E4675
:100130004F004543484F0020746F6F206C6F6E670F
:1001400020657874727573696F6E2070726576655C
:100150006E7465640A0020636F6C64206578747245
:100160007573696F6E2070726576656E7465640A6A
:1001700000536C6565702E2E2E00526573756D6987
:100180006E67207072696E74003344205072696E1D
:100190007465722072656164792E00436C69636BCB
:1001A00020746F20726573756D652E2E2E004E6F54
:1001B000206D6F76652E00456E642066696C652043
:1001C0006C6973740A00426567696E2066696C65C4
:1001D000206C6973740A004D31323500534420702D
:1001E00072696E74696E67206279746520004E6F63
:1001F00074205344207072696E74696E670A0046F9
:10020000696C652064656C657465643A0044656C6E
:100210006574696F6E206661696C65642C2046693F
:100220006C653A20006F70656E206661696C65646C
:100230002C2046696C653A20002569730025696D9C
:1002400020256973002569682025696D202569735B
:1002500000256964202569682025696D202569735A
:100260000025697920256964202569682025696D44
:1002700020256973005072696E742074696D653A47
:10028000200000010F150E12FF16170E13FF0302B8
:100290001A14FFFFFF0C04FFFFFF01000EFFFF0C0D
:1002A000190DFF18FFFFFFFFFFFF50726F746563AA
:1002B0007465642050696E0A004525692025730025
:1002C0003344205072696E7465722072656164797E
:1002D0002E0032012D0126011F0111016F666600FB
:1002E00044454255473A004B494C4C45442E20006A
:1002F0004D3131332053006F6B0048656174696E76
:100300006720646F6E652E0020573A0045256920EE
:100310002573003344205072696E746572207265D3
:100320006164792E0042656420646F6E652E002042
:10033000573A004265642048656174696E672E0013
:100340003344205072696E746572204F66662E00C9
:10035000454D455247454E43595F504152534552D2
:1003600000434153455F4C494748545F4252494717
:1003700048544E45535300544F47474C455F4C49F2
:100380004748545300534F4654574152455F504FCE
:10039000574552004255494C445F50455243454EE3
:1003A00054004C4556454C494E475F44415441002A
:1003B0005A5F50524F4245004155544F4C455645A7
:1003C0004C005052494E545F4A4F420050524F47E2
:1003D00052455353004155544F5245504F52545F6C
:1003E00054454D5000564F4C554D455452494300CD
:1003F000454550524F4D0053455249414C5F584F6F
:100400004E5F584F4646004649524D574152455F50
:100410004E414D453A4D61726C696E204531362032
:1004200056312E3520284769746875622920534F4C
:10043000555243455F434F44455F55524C3A6874AB
:100440007470733A2F2F6769746875622E636F6DCD
:100450002F4D61726C696E4669726D776172652F9E
:100460004D61726C696E2050524F544F434F4C5F38
:1004700056455253494F4E3A312E30204D41434854
:10048000494E455F545950453A3344205072696E85
:100490007465722045585452554445525F434F5538
:1004A0004E543A3120555549443A6365646532618A
:1004B00032662D343161322D343734382D39623182
:1004C000322D6335356336326633363766660A0059
:1004D0002F2F20007A5F6D696E3A2000795F6D6979
:1004E0006E3A2000785F6D696E3A20005265706F39
:1004F0007274696E6720656E6473746F70207374B4
:10050000617475730A004D31343520533C696E6453
:1005100065783E206F7574206F662072616E676526
:100520002028302D31290A0053657474696E6720C4
:1005300054726176656C20416363656C65726174A9
:10054000696F6E3A200053657474696E6720526556
:10055000747261637420416363656C657261746970
:100560006F6E3A200053657474696E67205072692B
:100570006E7420416363656C65726174696F6E3A75
:10058000200053657474696E67205072696E742020
:10059000616E642054726176656C20416363656CA2
:1005A00065726174696F6E3A200043290A006162C6
:1005B0006C656420286D696E2074656D7020004341
:1005C0006F6C642065787472756465732061726500
:1005D000200023646566696E6520204445464155C8
:1005E0004C545F4B64200023646566696E6520206F
:1005F00044454641554C545F4B6920002364656671
:10060000696E65202044454641554C545F4B70202F
:1006100000504944204175746F74756E6520666999
:100620006E69736865642120507574207468652054
:100630006C617374204B702C204B6920616E6420B8
:100640004B6420636F6E7374616E74732066726F97
:100650006D2062656C6F7720696E746F20436F6EDA
:1006600066696775726174696F6E2E680A00504919
:1006700044204175746F74756E65206661696C65A0
:1006800064212074696D656F75740A005448455281
:100690004D414C2052554E415741590054686572A6
:1006A0006D616C2052756E61776179004865617487
:1006B000696E67206661696C65640048656174698C
:1006C0006E67206661696C6564005049442041751D
:1006D000746F74756E65206661696C656421205461
:1006E000656D706572617475726520746F6F2068D6
:1006F0006967680A00204B643A2000204B693A2061
:1007000000204B703A20000A20436C6173736963C8
:1007100020504944200A002054753A2000204B758F
:100720003A2000206D61783A2000206D696E3A20F1
:100730000020643A200020626961733A20004F660D
:100740006673657473206170706C696564004572CE
:10075000723A20546F6F206661722100546F6F20CF
:100760006661722066726F6D207265666572656E75
:10077000636520706F696E740A00454550524F4D95
:100780002064697361626C65640A004E6F20636166
:100790007365206C696768740A00416374697665E3
:1007A0002045787472756465723A2000556E6B6EE0
:1007B0006F776E20636F6D6D616E643A2022004C1E
:1007C000696E65204E756D626572206973206E6F6B
:1007D00074204C617374204C696E65204E756D6297
:1007E00065722B312C204C617374204C696E653A14
:1007F00020004B494C4C45442E200053544F505040
:1008000045442E20005072696E7465722073746FB7
:10081000707065642064756520746F206572726FF6
:1008200072732E2046697820746865206572726F35
:100830007220616E6420757365204D3939392074DA
:100840006F20726573746172742E202854656D7008
:100850006572617475726520697320726573657461
:100860002E2053657420697420616674657220724D
:10087000657374617274696E67290A004E6F204354
:100880006865636B73756D2077697468206C696E39
:1008900065206E756D6265722C204C617374204CFE
:1008A000696E653A2000636865636B73756D206DD2
:1008B00069736D617463682C204C617374204C699A
:1008C0006E653A20004D313130004D3331005344D4
:1008D0002072656164206572726F720A00446F6EE7
:1008E00065207072696E74696E672066696C650A4E
:1008F0000020496E76616C69642065787472756455
:1009000065722000000000C00000B8C100000000B7
:1009100000009643000096430000C843205A3A0066
:1009200020593A0020436F756E7420583A002045D4
:100930003A00205A3A0020593A00583A003A004307
:1009400061703A00205A00205900580020204D6163
:10095000783A2000205A00205900580020204D6984
:100960006E3A20004F6E20004F666600536F66742B
:1009700020656E6473746F70733A200020643A00CF
:1009800020693A0020703A0024F4D43050C38E20FD
:10099000C2A24017828B7011127A910D816CD90A14
:1009A000A861E108C7586607615143061E4B5D0503
:1009B000C145A7041A411104093D98037139310357
:1009C0004036DB0265339102D4305402802E1D0282
:1009D000632CEE01752AC501B028A0011027810102
:1009E0008F2564012B244B01E0223401AC211F012F
:1009F0008D200D01801FFC00841EED00971DDF007F
:100A0000B81CD200E61BC600201BBC00641AB20052
:100A1000B219A8000A19A0006A189900D11791000C
:100A200040178B00B516840031167E00B31579008F
:100A30003A157300C7146F0058146A00EE1366006D
:100A40008813630025135E00C7125B006C12570009
:100A500015125400C111510070114F0021114B00AB
:100A6000D61049008D104700461044000210420085
:100A7000C00F4000800F3E00420F3C00060F3B00BD
:100A8000CB0E3800930E37005C0E3500270E340075
:100A9000F30D3200C10D3100900D3000600D2E00BD
:100AA000320D2D00050D2C00D90C2B00AE0C2900A9
:100AB000850C29005C0C2700350C27000E0C260045
:100AC000E80B2400C40B2400A00B23007D0B2300A3
:100AD0005A0B2100390B2100180B2000F80A1F00C7
:100AE000D90A1E00BB0A1E009D0A1D00800A1D00B7
:100AF000630A1C00470A1B002C0A1B00110A1A007B
:100B0000F7091A00DD091900C4091900AB09190019
:100B1000920917007B091800630917004C09160099
:100B200036091600200916000A091500F5081500F7
:100B3000E0081400CC081400B8081400A40814003D
:100B4000900813007D0812006B081300580812006B
:100B50004608120034081100230811001208110081
:100B600001081100F0071000E0071000D007100086
:100B7000C0071000B0070F00A107100091070E007A
:100B800083070F0074070F0065070E0057070E005C
:100B900049070E003B070D002E070E0020070D0031
:100BA00013070D0006070D00F9060C00ED060D00F9
:100BB000E0060C00D4060C00C8060C00BC060C00B5
:100BC000B0060C00A4060B0099060C008D060B0065
:100BD00082060B0077060B006C060B0061060A000C
:100BE00057060B004C060A0042060A0038060A00A7
:100BF0002E060A0024060A001A060A00100609003A
:100C000007060A00FD050900F4050900EB050900C7
:100C1000E2050900D9050900D0050900C70509004A
:100C2000BE050900B5050800AD050800A5050900C9
:100C30009C050800940508008C0508008405080040
:100C40007C050800740508006C05070065050800B0
:100C50005D050700560508004E050700470507001B
:100C60004005080038050700310507002A05070080
:100C7000230507001C050600160507000F050700E1
:100C80000805060002050700FB040600F50407003E
:100C9000EE040600E8040600E2040700DB04060098
:100CA000D5040600CF040600C9040600C3040600EC
:100CB000BD040600B7040600B1040500AC0406003C
:100CC000A6040600A00405009B0406009504050088
:100CD000900406008A0405008504050080040600CF
:100CE0007A04050075040500700405006B04050016
:100CF00066040500610405005C0405005704050056
:100D0000520405004D040500480405004304050095
:100D10003E0404003A0405003504050030040400D4
:100D20002C04050027040400230405001E0404000D
:100D30001A04040016040500110404000D04040044
:100D4000090405000404040000040400FC0304007A
:100D5000F8030400F4030400F0030400EC030400AF
:100D6000E8030400E4030400E0030400DC030400DF
:100D7000D8030400D4030400D0030400CC0304000F
:100D8000C8030300C503030024F404D9201BC40CCA
:100D90005C0E9804C4095F0265077101F405F9004F
:100DA000FB04B30048048700C103690058035500E1
:100DB00003034500BE023A008402310053022A00B8
:100DC0002902250004022000E4011C00C8011900CA
:100DD000AF01170098011400840113007101100085
:100DE0006101100051010E0043010D0036010B009E
:100DF0002B010B0020010B00150109000C0109005B
:100E000003010800FB000800F3000800EB000700E6
:100E1000E4000600DE000600D8000600D20006004E
:100E2000CC000500C7000500C2000500BD0004009D
:100E3000B9000400B5000400B1000400AD000400D6
:100E4000A9000400A5000300A20003009F00040005
:100E50009B0003009800030095000200930003002C
:100E6000900003008D0002008B0003008800020048
:100E70008600020084000300810002007F0002005F
:100E80007D0002007B000200790002007700010073
:100E9000760002007400020072000100710002007E
:100EA0006F0002006D0001006C0002006A0001008A
:100EB0006900020067000100660001006500010092
:100EC0006400020062000100610001006000010096
:100ED0005F0002005D0001005C0001005B0001009A
:100EE0005A0001005900010058000100570001009C
:100EF000560001005500010054000100530000009D
:100F00005300010052000100510001005000010097
:100F10004F0001004E0000004E0001004D00010096
:100F20004C0001004B0000004B0001004A00010092
:100F3000490001004800000048000100470001008E
:100F40004600000046000100450000004500010089
:100F50004400010043000000430001004200000083
:100F6000420001004100000041000100400001007A
:100F70003F0000003F0001003E0000003E00010075
:100F80003D0000003D0001003C0000003C0000006E
:100F90003C0001003B0000003B0001003A00000063
:100FA0003A0001003900000039000100380000005B
:100FB0003800000038000100370000003700010051
:100FC0003600000036000000360001003500000049
:100FD000350000003500010034000000340000003E
:100FE0003400010033000000330000003300010032
:100FF0003200000032000000320001003100000029
:10100000310000003100010030000000300000001D
:10101000300001002F0000002F0000002F00000012
:101020002F0001002E0000002E0000002E00010005
:101030002D0000002D0000002D0000002D000100FB
:101040002C0000002C0000002C0000002C000100EF
:101050002B0000002B0000002B0000002B000100E3
:101060002A0000002A0000002A0000002A000100D7
:1010700029000000290000002900000029000000CC
:1010800029000100280000002800000028000000BE
:1010900028000000280001002700000027000000B1
:1010A00027000000270000002700010026000000A4
:1010B0002600000026000000260000002600010097
:1010C000250000002500000025000000250000008C
:1010D000250000002500010024000000240000007D
:1010E0002400000024000000240001002300000070
:1010F0002300000023000000230000002300000064
:101100002300000023000100220000002200000054
:101110002200000022000000220000002200010046
:10112000210000002100000021000000210000003B
:10113000210000002100000021000100200000002B
:10114000200000002000000020000000200000001F
:101150002000000020000000200001001F0000000F
:101160001F0000001F0000001F0000001F00000003
:101170001F0000001F0001001E0000001E000000F4
:101180001E0000001E0000004D3834205820592059
:101190005A2045006265640A002C207379737465D7
:1011A0006D2073746F70706564212048656174658B
:1011B000725F49443A200048656174696E67206631
:1011C00061696C65640048656174696E6720666179
:1011D000696C656400FFD0FFE0FFCFFF64FFD1FFC3
:1011E00032380C060201FF64FFD0FFFE20204E6F54
:1011F0007A7A6C653A2000200066696C616D656ED4
:10120000742065787472756465005761697420662E
:101210006F72005052494E5420504155534544007E
:10122000746F20726573756D65005761697420660F
:101230006F72207072696E74005052494E54205083
:1012400041555345440000002100240027002A0096
:1012500000002200250028002B00000020002300B1
:10126000260029000202020202020202040404040F
:101270000404040403030303030303030101010142
:10128000010101010102040810204080010204084C
:10129000102040800102040810204080804020106F
:1012A00008040201000000010200090A0000000019
:1012B0000403080700000000000000000000000018
:1012C000000000004B494C4C45442E2000202D20AE
:1012D000496E76616C6964206578747275646572B4
:1012E000206E756D62657220210A0000000000000A
:1012F00000000000000000000000000000000000EE
:101300000000000000000000000000000000000CD1
:101310000000000000001E0000000C00001E000085
:10132000000C00003E0000000C00003306701E3F61
:1013300000003306F87F3F000063071C638C000049
:1013400061860CC18C0000E1860CFF8C0000FF86DA
:101350000CFF8C0001FFC60CC00C000180C60CE124
:101360000C000180C60C7F0F000300660C3E0700D6
:101370002020506C616E6E657242756666657242C1
:10138000797465733A20002046726565204D656D5D
:101390006F72793A2000436F6D70696C65643A2012
:1013A0004D617920333020323031390A00207C20E1
:1013B000417574686F723A20286E6F6E652C2064D8
:1013C000656661756C7420636F6E666967290A00D3
:1013D000323031372D31322D32352031323A303002
:1013E00000204C61737420557064617465643A2008
:1013F000004531362056312E350A004D61726C6938
:101400006E0020536F667477617265205265736554
:10141000740A00205761746368646F6720526573B3
:1014200065740A002042726F776E206F75742052C7
:10143000657365740A002045787465726E616C206E
:1014400052657365740A00506F77657255700A00B3
:1014500073746172740A006572726F7220777269B8
:1014600074696E6720746F2066696C650A00456E4A
:101470006473746F707320256320256320256320B7
:10148000256300205A3A0020593A0020583A006556
:101490006E6473746F7073206869743A2000446FCF
:1014A0006E6520736176696E672066696C652E0AC9
:1014B000004D3239005072656865617420504C41AE
:1014C00020456E64005072656865617420504C411F
:1014D00020426564005072656865617420504C411B
:1014E0000050726570617265005072656865617464
:1014F0002041425320456E640050726568656174F6
:1015000020414253204265640050726568656174F1
:10151000204142530050726570617265004D343253
:1015200038005072656865617420504C4100436F0B
:101530006F6C646F776E004368616E6765206669E3
:101540006C616D656E740044697361626C652073D3
:1015500074657070657273004D3834005365742083
:10156000686F6D65206F6666736574730050726591
:101570006865617420414253004175746F20686F43
:101580006D6500473238004D6F766520617869736C
:10159000004D61696E004D6F76652058004D6F7685
:1015A000652059004D6F7665205A00457874727534
:1015B000646572004D6F766520302E316D6D004D83
:1015C0006F766520316D6D004D6F76652031306D21
:1015D0006D004D6F7665206178697300457874728F
:1015E00075646572004D6F7665205A004D6F7665A3
:1015F0002059004D6F7665205800457874727564E7
:101600006572004D6F7665205A004D6F76652059E2
:10161000004D6F76652058005072657061726500EC
:10162000526573746F7265206661696C736166657B
:101630000046696C616D656E74004D6F74696F6E04
:101640000054656D7065726174757265004D6169F5
:101650006E00507265686561742041425320636F6B
:101660006E66005072656865617420504C4120635D
:101670006F6E66005049442D44005049442D44008B
:101680005049442D49005049442D49005049442DAA
:1016900050005049442D50002008204661637400DA
:1016A00020082046616374002008204D61780020E6
:1016B00008204D6178002008204D61780020082026
:1016C0004D696E002008204D696E002008204D698C
:1016D0006E004F6666004F6E20004175746F746532
:1016E0006D700046616E2073706565640046616EC2
:1016F0002073706565640042656400426564004E55
:101700006F7A7A6C65004E6F7A7A6C6500436F6E03
:1017100074726F6C0042656400426564004E6F7ABB
:101720007A6C65004E6F7A7A6C650046616E207344
:10173000706565640046616E207370656564005471
:10174000656D70657261747572650056547261766C
:10175000206D696E005654726176206D696E005678
:1017600054726176206D696E00566D696E00566D1B
:10177000696E00566D696E00566D617820450056A1
:101780006D6178204500566D6178204500566D6189
:1017900078205A00566D6178205A00566D61782085
:1017A0005A00566D6178205900566D6178205900B5
:1017B000566D6178205900566D6178205800566D3D
:1017C0006178205800566D61782058004D6F74691B
:1017D0006F6E0043616E6E6F7420656E746572206B
:1017E0007375626469723A2000022E2E0001526500
:1017F0006672657368004D61696E0020204E6F7AD5
:101800007A6C653A200020004261636B004D696E7E
:10181000696D756D2054656D7020697320313730A6
:101820002E0048656174696E67206661696C656445
:101830000045787472756465206D6F72650052653D
:1018400073756D65207072696E7400524553554D05
:1018500045204F5054494F4E533A0020204E6F7A46
:101860007A6C653A20006368616E6765006F662078
:101870007468652066696C616D656E740057616996
:101880007420666F72207374617274005052494EF6
:1018900054205041555345440020204E6F7A7A6CB5
:1018A000653A2000200066696C616D656E74207574
:1018B0006E6C6F6164005761697420666F720050CE
:1018C00052494E54205041555345440020204E6FFC
:1018D0007A7A6C653A20002000506C65617365204F
:1018E000776169742E2E2E0048656174696E6720D9
:1018F0006E6F7A7A6C65005052494E5420504155B3
:101900005345440020204E6F7A7A6C653A200020BF
:101910000068656174206E6F7A7A6C652E00507273
:1019200065737320627574746F6E20746F0050520B
:10193000494E54205041555345440020204E6F7A63
:101940007A6C653A2000746F20636F6E74696E75EF
:10195000652E2E2E00616E64207072657373206296
:101960007574746F6E00496E736572742066696C6D
:10197000616D656E74005052494E5420504155536C
:1019800045440020204E6F7A7A6C653A2000200092
:1019900066696C616D656E74206C6F61640057617F
:1019A000697420666F72005052494E542050415560
:1019B00053454400526573656E643A20006F6B00B6
:1019C000627573793A2070617573656420666F7211
:1019D00020696E7075740A00627573793A207061BF
:1019E0007573656420666F7220757365720A006294
:1019F0007573793A2070726F63657373696E670AE5
:101A0000004B494C4C45442E20004B494C4C206324
:101A1000617573656420627920746F6F206D7563E2
:101A20006820696E6163746976652074696D6520EC
:101A30002D2063757272656E7420636F6D6D616EBB
:101A4000643A2000506C656173652072657365743B
:101A5000005052494E5445522048414C5445440090
:101A60005072696E7465722068616C7465642E20B2
:101A70006B696C6C28292063616C6C6564210A00B9
:101A8000656E7175657565696E67202200000000DE
:101A9000C00000B8C100000000000048420000483B
:101AA0004200008040000000005761726E696E675E
:101AB0003A20486F6D696E672042756D70204469E9
:101AC0007669736F72203C20310A00020204000024
:101AD000A0400000A0400000A0400000974300800C
:101AE000A1430000C843FFFFFF4D36303020486F50
:101AF00074656E6420746F6F20636F6C6420746F04
:101B0000206368616E67652066696C616D656E74DF
:101B10000A006175746F25692E67004D3234004DDF
:101B200032332025730057726974696E6720746FB1
:101B30002066696C653A20006F70656E2066616989
:101B40006C65642C2046696C653A20006F70656E88
:101B5000206661696C65642C2046696C653A2000DA
:101B600046696C652073656C65637465640A002062
:101B700053697A653A200046696C65206F70656E1E
:101B800065643A20006F70656E206661696C6564FB
:101B90002C2046696C653A20002066696C653A2005
:101BA00000646F696E67006672657368004E6F77D8
:101BB0002000454E4420535542524F5554494E45FE
:101BC0000A002220706F73002220706172656E74AB
:101BD0003A2200535542524F5554494E45204341F5
:101BE0004C4C207461726765743A22004B494C4C2E
:101BF00045442E2000747279696E6720746F2063EB
:101C0000616C6C207375622D67636F646520666913
:101C10006C6573207769746820746F6F206D616ED6
:101C200079206C6576656C732E204D4158206C656B
:101C300076656C2069733A004572726F723A0043A0
:101C4000616E6E6F74206F70656E2073756264696B
:101C50007220006563686F3A00416D61782045002D
:101C6000416D6178204500416D6178205A00416DD9
:101C70006178205A00416D6178205900416D61788A
:101C8000205900416D6178205800416D61782058DD
:101C900000412D74726176656C00412D747261761D
:101CA000656C00412D7265747261637400412D7220
:101CB00065747261637400416363656C00416363C2
:101CC000656C004D6F74696F6E0056652D6A6572A4
:101CD0006B0056652D6A65726B0056652D6A6572DC
:101CE0006B00567A2D6A65726B00567A2D6A6572A2
:101CF0006B0056792D6A65726B0056792D6A657294
:101D00006B0056792D6A65726B0056782D6A657284
:101D10006B0056782D6A65726B0056782D6A657275
:101D20006B004D6F74696F6E004573746570732F2F
:101D30006D6D004573746570732F6D6D005A73740B
:101D40006570732F6D6D005A73746570732F6D6DB0
:101D5000005973746570732F6D6D005973746570DD
:101D6000732F6D6D005873746570732F6D6D00580F
:101D700073746570732F6D6D004D6F74696F6E00B5
:101D800053746570732F6D6D004A65726B0041630B
:101D900063656C65726174696F6E0056656C6F6324
:101DA00069747900436F6E74726F6C0046696C2EB3
:101DB000204469612E0046696C2E204469612E0022
:101DC0004F6666004F6E20004520696E206D6D33B2
:101DD00000436F6E74726F6C002044002049002035
:101DE000204D3330312050005049442073657474C5
:101DF000696E67733A0A00204600204200204800BE
:101E000020204D3134352053004D61746572696175
:101E10006C2068656174757020706172616D6574A5
:101E20006572733A0A00205A0020590020204D3272
:101E30003036205800486F6D65206F666673657494
:101E40003A0A00204500205A00205900205800205E
:101E5000420020540020204D323035205300416490
:101E600076616E6365643A20533C6D696E5F6665AA
:101E70006564726174653E20543C6D696E5F747276
:101E80006176656C5F66656564726174653E20426B
:101E90003C6D696E5F7365676D656E745F74696DC7
:101EA000655F75733E20583C6D61785F78795F6A35
:101EB00065726B3E205A3C6D61785F7A5F6A65722D
:101EC0006B3E20453C6D61785F655F6A65726B3E75
:101ED0000A0020540020520020204D32303420507F
:101EE00000416363656C65726174696F6E2028756B
:101EF0006E6974732F7332293A20503C7072696E88
:101F0000745F616363656C3E20523C7265747261FC
:101F100063745F616363656C3E20543C74726176E8
:101F2000656C5F616363656C3E0A00204500205A62
:101F30000020590020204D3230312058004D61786A
:101F4000696D756D20416363656C65726174696F5D
:101F50006E2028756E6974732F7332293A0A002037
:101F60004500205A0020590020204D32303320589F
:101F7000004D6178696D756D206665656472617488
:101F800065732028756E6974732F73293A0A0020CF
:101F90004500205A0020590020204D393220580099
:101FA00053746570732070657220756E69743A0A97
:101FB0000020204D3230302044300A0020204D32A5
:101FC00030302044002044697361626C65640A000B
:101FD00046696C616D656E742073657474696E67B3
:101FE000733A0020204D3134392043203B20556E78
:101FF00069747320696E2043656C736975730A0098
:102000002020473231202020203B20556E697473F8
:1020100020696E206D6D0A0025753A2530327500F5
:10202000253032753A25303275002575642025300B
:1020300032753A25303275005A005900580009208F
:10204000000000000000000000000000007FFFE032
:102050000000000000000000000000007000E00030
:10206000000000000000000000000061F8600000B7
:102070000000000000000000000041F82000000007
:1020800000000000000000000040F0200000000000
:102090000000000000000000406020000000000080
:1020A000000000000000005801A07F800000000038
:1020B0000000004104005C63A0FFC00000000000BD
:1020C00000002082005EF7A0FFC0000000000000BA
:1020D000002082005EF7A0FFC000000000000000AA
:1020E0004104005C63A07F800000000000000082CB
:1020F00008005801A07F80000000000000010410CB
:1021000000406020FFC0000000000000010410003B
:1021100040F020FFC00000000000000082080041E5
:10212000F820FFC00000000000000041040061F83A
:10213000603F00000000000000000000007000E0B0
:102140001E0000000000000001FFFF807FFFE00C88
:102150000000000000000001FFFF80000000000000
:10216000000000000000000000007FFFE000000011
:102170000000000000000000007000E0000000000F
:102180000000000000000000630C60000000000080
:1021900000000000000000470E20000000000000CA
:1021A0000000000000004F0F2000000000000000B1
:1021B00000000000005F0FA0000000000000000011
:1021C000000000005E07A07F80000000000000000B
:1021D000410400406020FFC000000000000000201B
:1021E000820040F020FFC0000000000000002082BC
:1021F0000040F020FFC0000000000000004104008B
:102200004060207F80000000000000008208005E27
:1022100007A07F80000000000000010410005F0F95
:10222000A0FFC0000000000000010410004F0F20BC
:10223000FFC000000000000000820800470E20FFE1
:10224000C000000000000000410400630C603F007B
:10225000000000000000000000007000E01E000010
:10226000000000000001FFFF807FFFE00C00000085
:102270000000000001FFFF8000000000091200FCC8
:102280000A01E803D720FFFD0EFD0BFD0000000949
:10229000000E010B0B09040080808080808080008C
:1022A00000808004040409030790909090080A0AB3
:1022B000090000242424FF2424FF242424070B0BDA
:1022C0000901FF107C929050381412927C10070A7A
:1022D0000A09010042A4A4481010244A4A84070AAB
:1022E0000A090100609090906062948894620104F1
:1022F0000409040780808080030C0C0903FF204040
:1023000040808080808080404020030C0C0903FFC7
:1023100080404020202020202040408007070709DF
:102320000103109254385492100707070901011055
:102330001010FE1010100204040904FEC0C04080FA
:10234000070101090104FE020202090400C0C007DE
:102350000A0A090100020404081010204040800706
:102360000A0A090100384482828282828244380744
:102370000A0A090100103050901010101010FE07CA
:102380000A0A090100384482020408102040FE07AE
:102390000A0A090100FE02040818040202847807F0
:1023A0000A0A090100040C14244484FE04040407EE
:1023B0000A0A090100FE808080F80402028478077E
:1023C0000A0A0901003C408080B8C4828244380770
:1023D0000A0A090100FE0204040808101010100780
:1023E0000A0A09010038448244384482824438078A
:1023F0000A0A09010038448282463A02020478023D
:102400000707090400C0C0000000C0C00209090994
:1024100004FEC0C0000000C0C040800509090902D8
:102420000008102040804020100807040409010221
:10243000FE0000FE05090909020080402010081076
:10244000204080070A0A090100384482020408106B
:10245000100010070A0A09010038449AAAAAAAAA79
:102460009C403C070A0A09010010282828447C44A3
:10247000828282070A0A090100F8848284F8848231
:102480008284F8070A0A0901003C4280808080802B
:1024900080423C070A0A090100F884828282828213
:1024A0008284F8070A0A090100FE808080F8808093
:1024B0008080FE070A0A090100FE808080F8808083
:1024C000808080070A0A09010038448280808E8259
:1024D000824438070A0A09010082828282FE8282CF
:1024E000828282050A0A090200F82020202020208A
:1024F0002020F8070A0A0901003E08080808080811
:10250000888870070A0A09010082848890A0D08810
:10251000848282070A0A090100808080808080808E
:102520008080FE070A0A0901008282C6AA9282827E
:10253000828282070A0A0901008282C2A2928A86E6
:10254000828282070A0A0901007C82828282828258
:1025500082827C070A0A090100F884828284F8805A
:10256000808080080B0B0901FF38448282828282BE
:102570008A443A01070A0A090100F884828284F831
:1025800090888482070A0A0901007C8280807C028C
:102590000202827C070A0A090100FE1010101010C6
:1025A00010101010070A0A090100828282828282BA
:1025B00082824438070A0A09010082828244444424
:1025C00028282810070A0A09010082828282929232
:1025D0009292AA44070A0A09010082824428101034
:1025E00028448282070A0A090100828244281010C6
:1025F00010101010070A0A090100FE02040810203A
:10260000408080FE040C0C0903FFF08080808080F5
:102610008080808080F0070A0A0901008040402005
:10262000101008040402040C0C0902FFF010101032
:1026300010101010101010F00704040901061028E3
:1026400044820801010900FFFF03030309030A8014
:1026500040200707070901007C02027E82867A0774
:102660000A0A090100808080BCC2828282C2BC0743
:1026700007070901007C82808080827C070A0A09A2
:1026800001000202027A86828282867A070707099F
:1026900001007C8282FE80827C070A0A0901001CFC
:1026A00022222020F820202020070A0A0901FD7A92
:1026B00084848478807C82827C070A0A09010080F5
:1026C0008080BCC28282828282050A0A090200607E
:1026D0000000E02020202020F8050D0D0902FD1843
:1026E000000038080808080808888870070A0A09DE
:1026F0000100808080848890B0C88482050A0A091D
:102700000200E02020202020202020F807070709D1
:102710000100EC929292929282070707090100BC95
:10272000C282828282820707070901007C8282823C
:1027300082827C070A0A0901FDB8C4828282C4B879
:10274000808080070A0A0901FD3A46828282463A61
:102750000202020707070901009C62424040404014
:102760000707070901007C82807C02827C07090937
:102770000901002020FC20202020221C0707070937
:1027800001008282828282867A070707090100821D
:102790008244442828100707070901008282929288
:1027A00092AA44070707090100824428102844829E
:1027B000070A0A0901FD42422424241818109060D7
:1027C000070707090100FE0408102040FE060B0B56
:1027D0000902001C20202020C0202020201C010CE9
:1027E0000C0904FF808080808080808080808080D1
:1027F000060B0B090100E0101010100C1010101047
:10280000E007030309010762928CFFFFFFFFFFFF50
:10281000FFFFFFFFFFFFFFFFFFFFFFFFFFFFFFFFC8
:10282000FFFFFFFFFFFFFFFFFFFFFF0000000900AA
:102830000E010B0B090400808000008080808080E6
:10284000808006080809010008789490A0A47840C8
:10285000070A0A0901001C222020F8202060A25C3F
:10286000070606090103827C44447C82070A0A09A0
:102870000100828244287C107C101010010B0B098F
:1028800004FF8080808080008080808080040B0B2B
:102890000902FF6090806090909060109060030249
:1028A0000209030BA0A00809090900013C4299A5EF
:1028B000A1A599423C050707090103609070907833
:1028C00000F80708080901011224489090482412D2
:1028D000060404090102FC040404050101090204C0
:1028E000F80809090900013C42B9A5BDA9A5423C67
:1028F000060101090109FC04040409030660909023
:1029000060070909090101101010FE10101000FEE7
:102910000406060901046090106080F004060609B0
:10292000010460902010906003030309030A204013
:10293000800709090901FE8282828282C6BA8080EC
:10294000070A0A0901007E8A8A8A7A0A0A0A0A0A9A
:10295000020202090404C0C00403030902FD20901E
:102960006003060609010440C0404040E005060639
:102970000901047088887000F807080809010190AF
:1029800048241212244890070A0A09010040C04056
:102990004042E60A121A06070A0A09010040C0402E
:1029A000404CF2020C101E070A0A09010060902038
:1029B0001092660A121A06070A0A0901001000108E
:1029C0001020408082827C070E0E09010020100832
:1029D0000010282828447C44828282070E0E0901B8
:1029E000000810200010282828447C448282820796
:1029F0000E0E0901001028440010282828447C44A9
:102A0000828282070D0D0901003458001028282801
:102A1000447C44828282070D0D09010028280010A1
:102A2000282828447C44828282070E0E0901001067
:102A300028281010282828447C44828282070A0A09
:102A40000901001E2828284E784888888E070D0D19
:102A50000901FD3C42808080808080423C0824182F
:102A6000070E0E09010020100800FE808080F8800B
:102A7000808080FE070E0E09010008102000FE80F5
:102A80008080F880808080FE070E0E0901001028EB
:102A90004400FE808080F880808080FE070D0D0954
:102AA0000100282800FE808080F880808080FE055C
:102AB0000E0E09020040201000F8202020202020C7
:102AC0002020F8050E0E09020010204000F82020FA
:102AD000202020202020F8050E0E0902002050881A
:102AE00000F82020202020202020F8050D0D0902CC
:102AF00000505000F82020202020202020F8070A35
:102B00000A09010078444242F24242424478070DE9
:102B10000D0901003458008282C2A2928A86828204
:102B200082070E0E090100201008007C828282823A
:102B3000828282827C070E0E090100081020007C30
:102B400082828282828282827C070E0E09010010BC
:102B50002844007C82828282828282827C070D0DE0
:102B60000901003458007C82828282828282827CC7
:102B7000070D0D0901002828007C82828282828252
:102B800082827C07070709010182442810284482B9
:102B9000070C0C0901FF027C868A8A9292A2A2C2CB
:102BA0007C80070E0E0901002010080082828282BC
:102BB000828282824438070E0E090100081020002C
:102BC00082828282828282824438070E0E0901004C
:102BD0001028440082828282828282824438070DD9
:102BE0000D0901002828008282828282828282442A
:102BF00038070E0E090100081020008282442810B8
:102C00001010101010070A0A0901008080FC82824F
:102C100082FC808080060A0A09010038444448D0BA
:102C20004844444458070B0B090100201008007C5D
:102C300002027E82867A070B0B0901000810200031
:102C40007C02027E82867A070B0B09010010284461
:102C5000007C02027E82867A070A0A090100345843
:102C6000007C02027E82867A070A0A09010028286F
:102C7000007C02027E82867A070C0C090100102873
:102C80002810007C02027E82867A0707070901006D
:102C90006C12127E90926C070A0A0901FD7C8280F8
:102CA0008080827C104830070B0B0901002010083F
:102CB000007C8282FE80827C070B0B0901000810D9
:102CC00020007C8282FE80827C070B0B09010010B1
:102CD0002844007C8282FE80827C070A0A09010067
:102CE0002828007C8282FE80827C050C0C09020070
:102CF0008040200000E02020202020F8050C0C0956
:102D000002001020400000E02020202020F8050CC8
:102D10000C0902002050880000E02020202020F82C
:102D2000050B0B09020050500000E020202020205D
:102D3000F8070B0B090100483050083C448282829E
:102D40004438070A0A090100345800BCC282828252
:102D50008282070B0B090100201008007C8282820E
:102D600082827C070B0B090100081020007C828204
:102D70008282827C070B0B090100102844007C82B0
:102D8000828282827C070A0A0901003458007C8210
:102D9000828282827C070A0A0901002828007C823C
:102DA000828282827C07090909010010381000FE26
:102DB000001038100709090901FF027C8A8A92A2D3
:102DC000A27C80070B0B0901004020100082828248
:102DD0008282867A070B0B0901000810200082828C
:102DE000828282867A070B0B090100102844008238
:102DF00082828282867A070A0A09010028280082D4
:102E000082828282867A070E0E0901FD0408100074
:102E100042422424241818109060070B0B0901FE6D
:102E20008080B8C4828282C4B88080070D0D0901F9
:102E3000FD24240042422424241818109060000627
:102E40000900FE000000000001090008FE00000566
:102E5000080806000040F0C888889878100508081F
:102E6000060000C0F88888888888F80505050600EF
:102E7000012030F830200508080600002070F820F6
:102E8000202020E00509090600FF2070A8A8B888C6
:102E90008870200509090600FFE080C0B0A828302E
:102EA00028280509090600FFF8A88888888888A8C6
:102EB000F8050A0A0600FE205050505088A8A8883D
:102EC0007003030306000340A040486F6D65202592
:102ED00073257325732066697273740020666972A6
:102EE00073740A005A0059005800486F6D6520003D
:102EF00053442063617264206F6B0A006F70656ECB
:102F0000526F6F74206661696C65640A00766F6C3D
:102F1000756D652E696E6974206661696C65640AF9
:102F200000534420696E6974206661696C0A007000
:102F3000012C0190012701B0012201C0011D01F007
:102F40000118011002130130020E01600209019004
:102F5000020401C002FF000003FA004003F50080F4
:102F600003F000D003EB002004E6007004E100E071
:102F700004DC004005D700C005D2004006CD00D0DB
:102F800006C8008007C3003008BE00F008B900C0C2
:102F900009B400B00AAF00B00BAA00D00CA5000025
:102FA0000EA000500F9B00C0109600501291000020
:102FB000148C00C0158700B0178200B0197D00D0B6
:102FC0001B7800001E730040206E0090226900F004
:102FD00024640040275F0090295A00E02B55001020
:102FE0002E500020304B0010324600E0334100905C
:102FF000353C001037370070383200A0392D00B052
:103000003A2800A03B2300603C1E00103D190090B0
:103010003D1400103E0F00703E0A00C03E05000047
:103020003F0000403FFBFF803FF6FFC03FF1FF4500
:1030300072723A204D494E54454D5020424544004D
:103040004572723A204D494E54454D50004D494EFF
:1030500054454D5020747269676765726564004518
:1030600072723A204D415854454D5020424544001B
:103070004572723A204D415854454D50004D4158CB
:1030800054454D502074726967676572656400200D
:103090002F002042403A0020403A007C3C3E5E2B0C
:1030A0003D3F2F5B5D3B2C2A225C0020746F6F201C
:1030B0006C6F6E6720657874727573696F6E2070BF
:1030C000726576656E7465640A0020636F6C6420B7
:1030D000657874727573696F6E2070726576656E4F
:1030E0007465640A005072696E742070617573654E
:1030F00064004D31323500004D3234005072696E3B
:10310000742061626F72746564004D3231004E6FDD
:103110002053442063617264004368616E676520D8
:1031200053442063617264004D3231005072696E05
:10313000742066726F6D2053440053746F7020705A
:1031400072696E7400526573756D65207072696E78
:1031500074005061757365207072696E7400496EF9
:1031600069742E205344206361726400436F6E744F
:10317000726F6C00507265706172650054756E6597
:1031800000496E666F2073637265656E004D363060
:1031900030204230004368616E67652066696C616B
:1031A0006D656E7400466C6F7700466C6F770046F5
:1031B000616E2073706565640046616E2073706592
:1031C00065640042656400426564004E6F7A7A6C03
:1031D00065004E6F7A7A6C650053706565640053C4
:1031E00070656564004D61696E00544845524D41FB
:1031F0004C2052554E4157415900546865726D61DB
:103200006C2052756E617761790048617264636FFA
:103210006465642044656661756C742053657474DC
:10322000696E6773204C6F616465640A00900100E9
:10323000009001000032000000102700000000167E
:103240004300001643000080400000C8410000A079
:10325000420000A0420000C8430000BE4200060930
:1032600000FE0701920321207FFF07FF07FF0000F8
:1032700000060000010707060200808080808000B1
:1032800080030202060105A0A00507070600005002
:1032900050F850F850500507070600002078A0703D
:1032A00028F020050707060000C0C8102040981825
:1032B0000507070600006090A040A890680203037D
:1032C000060104C0408003070706010020408080FB
:1032D0008040200307070601008040202020408016
:1032E00005050506000120A870A8200505050600B3
:1032F000012020F820200203030602FFC0408005C1
:103300000101060003F8020202060200C0C0050522
:103310000506000108102040800507070600007020
:1033200088888888887003070706010040C04040ED
:103330004040E0050707060000708808708080F8AC
:10334000050707060000F81020100808F005070719
:1033500006000010305090F8101005070706000016
:10336000F880F00808887005070706000070808064
:10337000F0888870050707060000F8081020202054
:103380002005070706000070888870888870050788
:103390000706000070888878080870020505060294
:1033A00000C0C000C0C00206060602FFC0C000C0C8
:1033B00040800407070600001020408040201005D0
:1033C0000303060002F800F8040707060100804026
:1033D0002010204080050707060000708808102094
:1033E000002005070706000070880868A8A8700577
:1033F0000707060000708888F88888880507070690
:103400000000F08888F08888F00507070600007043
:10341000888080808870050707060000F08888880B
:103420008888F0050707060000F88080F08080F8A3
:10343000050707060000F88080F0808080050707F8
:10344000060000708880B8888870050707060000AD
:10345000888888F8888888010707060200808080AD
:10346000808080800507070600003810101010903B
:10347000600507070600008890A0C0A09088050797
:1034800007060000808080808080F805070706001E
:103490000088D8A8888888880507070600008888DB
:1034A000C8A898888805070706000070888888885B
:1034B0008870050707060000F08888F08080800586
:1034C000070706000070888888A890680507070627
:1034D0000000F08888F0A0908805070706000078B3
:1034E0008080700808F0050707060000F8202020FB
:1034F00020202005070706000088888888888870B3
:103500000507070600008888888888502005070777
:103510000600008888888888A850050707060000EC
:10352000888850205088880507070600008888880A
:1035300050202020050707060000F80810204080D2
:10354000F8030707060100E08080808080E0050521
:10355000050600018040201008030707060100E06F
:103560002020202020E005030306000420508805C9
:103570000101060000F8020202060205804005056E
:1035800005060000700878887805070706000080A7
:1035900080B0C88888F00505050600007080808826
:1035A00070050707060000080868988888780505F0
:1035B000050600007088F8807005070706000030D7
:1035C00048E0404040400506060600FF70888878C5
:1035D00008700507070600008080B0C88888880149
:1035E00007070602008000808080808003080806AC
:1035F00001FF200020202020A04004070706000033
:10360000808090A0C0A090030707060100C0404042
:10361000404040E0050505060000D0A8A8A8A80580
:103620000505060000B0C888888805050506000065
:1036300070888888700506060600FFF08888F0808C
:10364000800506060600FF788888780808050505C5
:10365000060000B0C8808080050505060000708067
:103660007008F00407070600004040E0404040308A
:103670000505050600008888889868050505060088
:103680000088888850200505050600008888A8A8BD
:1036900050050505060000885020508805060606DE
:1036A00000FF888888780870050505060000F81076
:1036B0002040F803070706010020404080404020DA
:1036C0000107070602008080808080808003070752
:1036D00006010080404020404080050202060002B2
:1036E000689000000006000047D63CD311241FBE9E
:1036F000CFEFD0E4DEBFCDBF12E0A0E0B1E0E6E95D
:10370000F6EC01E00BBF02C007900D92AC37B10799
:10371000D9F723E1ACE7B2E001C01D92AD3CB2079E
:10372000E1F71BE1C5E7DBE104C02197FE010E9440
:10373000A9E2C437D107C9F70E9418CF0C943EE321
:103740000C9400002F923F924F925F926F927F9263
:103750008F929F92AF92BF92CF92DF92EF92FF92A1
:103760000F931F93CF93DF93CDB7DEB7C258D10924
:103770000FB6F894DEBF0FBECDBF81E090E090930E
:10378000280B8093270B8091C6138D3409F427C32F
:10379000843511F40C945331873411F00C94953125
:1037A0008091C4139091C5138B31910509F46DC2BA
:1037B00064F497FF02C00C94AF318230910574F12C
:1037C000049709F41BC20C94AF318A35910509F4B2
:1037D0008CC24CF44C9711F00C94AF3180E00E94F5
:1037E000D0420C94AF318B35910509F482C28C35EF
:1037F000910511F00C94AF310E942048F3E92F2E6F
:10380000F1E03F2EABE0CA2EABE0DA2EE12CF12C3A
:1038100000E010E028961FAE2897ACC28091090105
:10382000882311F40C94AF31B3E98B2EB1E09B2EB9
:1038300017E1C12E1BE0D12E03E0E02E0EE0F02EAA
:103840008FE8A82E8DE0B82E00E010E0D4018D9115
:103850004D010E94033B882371F10E94D03AF80188
:10386000E458FD4F2081211104C0209180022223C1
:1038700031F0F701208131814281538103C020E082
:1038800030E0A9010E945AE00330110559F0D5013A
:103890002D913D914D915C912B013C01C301B201F1
:1038A0000E9459E0462F572FBC01F60140835183F7
:1038B000628373830AC0F70180819181A281B38101
:1038C000F60180839183A283B3830F5F1F4FF4E0DF
:1038D000CF0ED11C24E0E20EF11C34E0A30EB11C8B
:1038E0000430110509F0B2CF86E40E94323B8823F0
:1038F000C9F00E94D03A20E030E0A9010E94DDE149
:10390000181684F40E94D03A20E030E040E752E4F8
:103910000E94DDE060930001709301018093020139
:103920009093030180911E01882309F4B4C0C090D4
:103930001C0AD0901D0AE0901E0AF0901F0AA701F1
:1039400096016091170B7091180B8091190B909153
:103950001A0B0E943FDC87FF08C0C092170BD09261
:10396000180BE092190BF0921A0BC090200AD0901D
:10397000210AE090220AF090230AA70196016091A3
:103980001B0B70911C0B80911D0B90911E0B0E94C4
:103990003FDC87FF08C0C0921B0BD0921C0BE0924B
:1039A0001D0BF0921E0BC0901201D0901301E090FD
:1039B0001401F0901501A70196016091170B709109
:1039C000180B8091190B90911A0B0E94DDE11816CB
:1039D00044F4C092170BD092180BE092190BF0929E
:1039E0001A0BC0901601D0901701E0901801F090CA
:1039F0001901A701960160911B0B70911C0B80911E
:103A00001D0B90911E0B0E94DDE1181644F4C0922C
:103A10001B0BD0921C0BE0921D0BF0921E0BC09062
:103A2000240AD090250AE090260AF090270AA701E0
:103A3000960160911F0B7091200B8091210B90914A
:103A4000220B0E943FDC87FF08C0C0921F0BD09260
:103A5000200BE092210BF092220BC0901A01D09023
:103A60001B01E0901C01F0901D01A70196016091DF
:103A70001F0B7091200B8091210B9091220B0E94C3
:103A8000DDE1181644F4C0921F0BD092200BE09297
:103A9000210BF092220B0E944A3C8091510E83FD33
:103AA00086C0C090230BD090240BE090250BF090A3
:103AB000260B20910F0E3091100E4091110E509157
:103AC000120EC701B6010E943FDC882309F46FC0C3
:103AD0000E948F7A882301F1C0920F0ED092100EAF
:103AE000E092110EF092120EE3E5FCE184918F0159
:103AF0000F5F1F4F882321F00E94553CF801F6CF3D
:103B0000E6E5F1E084918F010F5F1F4F882321F0DC
:103B10000E94553CF801F6CFC090230BD090240BA7
:103B2000E090250BF090260B20910F0E3091100E97
:103B30004091110E5091120EC701B6010E9459E03A
:103B40009F77E091360E44E0E49FF0011124E85C99
:103B5000FE4F20813181428153810E94A5DC20E00B
:103B600030E042E853E40E94DDE1181604F5C0920B
:103B70000F0ED092100EE092110EF092120EE3E5AD
:103B8000FCE184918F010F5F1F4F882321F00E9479
:103B9000553CF801F6CFE7E3F1E084918F010F5F28
:103BA0001F4F882321F00E94553CF801F6CF609109
:103BB000400170914101072E000C880B990B0E9467
:103BC00046DC2091000130910101409102015091A9
:103BD00003010E94A5DC2AE037ED43E25CE30E948A
:103BE000A5DC0E942A3980E1E7E1FBE0A3E0BEE02A
:103BF00001900D928A95E1F70C94AF3180E50E9417
:103C0000323B882329F00E948C3A6B017C0103C06F
:103C1000C12CD12C760183E50E94323B882361F0D0
:103C20000E94D03A20E030E04AE754E40E94A5DC4C
:103C30000E9456E16B017C010E94204880914A015C
:103C4000811105C060E081E791E00E94DEC80E941A
:103C50004A3C8091030B9091040BA091050BB0910D
:103C6000060BC80ED91EEA1EFB1E0E94F352DC0191
:103C7000CB018C199D09AE09BF09B7FD02C00C9498
:103C8000AF3180E00E942A7BF0CF0E94389D8111E5
:103C90000C94AF3180E090E0A0E0B1E489839A8396
:103CA000AB83BC8380E090E0A1E9B3E48D839E8385
:103CB000AF83B88780E090E0A0EAB1E489879A8773
:103CC000AB87BC8780E50E94323B882319F00E94B5
:103CD0009C3A01C060E068A3BE016F5F7F4FCE01D8
:103CE00080960E9425910C94AF31109280020C9422
:103CF000AF3181E0809380020C94AF310E94D03AC2
:103D00004B015C010330110559F0F701E157F24F07
:103D100020813181428153810E9459E04B015C0135
:103D2000F701ED5FF14F2081318142815381C5015F
:103D3000B4010E9459E02B013C012DEB37E346E82A
:103D400055EB0E94DDE187FD1DC02DEB37E346E812
:103D500055E3C301B2010E943FDC18169CF00F5FCF
:103D60001F4FB4E0CB0ED11CE4E0EE0EF11C04308A
:103D7000110559F1D1018D911D010E94323B88231B
:103D800071F3BCCF0330110569F480920F0E90924D
:103D9000100EA092110EB092120EB1E02896BFAF95
:103DA0002897DDCFA3019201F601608171818281A4
:103DB00093810E945AE0D6016D937D938D939C93DD
:103DC0001397C8010E945039CACF2896FFAD289793
:103DD000F1110E94D69D0E94F3410C94AF31809165
:103DE000C4139091C5138237910511F40C94AA273E
:103DF0000CF0DBC08B34910509F46EC50CF067C084
:103E00008831910509F4ABC2B4F58231910511F402
:103E10000C94D826BCF497FF02C00C94AF318230CA
:103E200091050CF4B2C1419711F00C94AF3160E0F0
:103E30008EEA91E00E94DEC85E985E9815985E98C2
:103E40000C94AF318531910509F46EC23CF444976E
:103E500011F00C94AF31E6ECF1E023C2863191050C
:103E600009F466C2479711F00C94AF31E091C21388
:103E7000F091C31367C28C31910509F4D9C2A4F43F
:103E80008A31910509F48AC20CF096C21092F50E9F
:103E90000E94149E87ED91E090934F0D80934E0DFC
:103EA0000E94AE390C94AF318F31910509F42EC4C4
:103EB0002CF44E9709F4C6C20C94AF3180329105B0
:103EC00009F4D8C38A9709F4C7C40C94AF31883673
:103ED000910509F40DC50CF040C08235910509F437
:103EE0005EC714F58D34910509F4FEC40CF4F8C4D2
:103EF0008135910511F00C94AF310E946F450E94FD
:103F000020480E94B77A1092E60D1092E50D68EEF7
:103F100073E080E090E00E9401C860E080E493E0FC
:103F20000E94DEC80C94AF318435910509F440C776
:103F30000CF439C78535910509F471C78C359105A5
:103F400011F00C94AF3193E9C92E91E0D92E23E101
:103F5000E22E2EE0F22E10E07DC78D36910509F499
:103F600032C69CF48A36910509F467C60CF4E7C59D
:103F70008B36910509F486C68C36910511F00C94A8
:103F8000AF31109237010C94AF318F36910509F49F
:103F900019C50CF404C58037910509F484C581372F
:103FA000910509F484C50C94AF31833D910511F45A
:103FB0000C94A62A0CF06FC08139910511F40C9471
:103FC000BB2844F58737910511F40C944A2884F4F2
:103FD0008537910511F40C94022814F00C940B28E9
:103FE0008337910511F00C94AF31E7E0F4E0B8C7E6
:103FF0008937910511F40C94B52814F40C94AE286B
:104000008D37910509F450C68C38910509F47BC5AC
:104010000C94AF31893C910511F40C947D297CF40A
:104020008E3B910509F4EDC5883C910511F40C9483
:1040300035298B39910511F00C94AF319DC58C3C1D
:10404000910511F40C94B52984F48B3C910511F081
:104050000C94AF3164E5E62E6AE0F62E03E911E038
:1040600074E0D72ED00E0C94A6298D3C910511F446
:104070000C941F2A8E3C910511F00C94AF3143E94A
:10408000C42E41E0D42E5DE6E52E58E0F52E00E08A
:1040900010E00C94942A803921E0920711F40C94DA
:1040A000E42E84F58C3241E0940711F40C94002B3B
:1040B0008CF48D3D910511F40C94B62A823E910545
:1040C00011F40C94FD2A8C3D910511F00C94AF3144
:1040D0000C94A92A8E32A1E09A0711F40C942C2B8F
:1040E00014F40C94292B8F32E1E09E0711F40C9408
:1040F000802B8336914011F00C94AF31E8E3FCE162
:104100000C942731863F21E0920711F40C94E82F9C
:1041100014F58C3A41E0940711F40C94E72E4CF41A
:104120008A39914011F00C94AF310E94AA3B0C9453
:10413000AF31843FB1E09B0711F40C94CF2F853F42
:10414000914011F00C94AF310E94D4BD80E00E94E8
:1041500067920C94AF318835F2E09F0711F40C940C
:10416000F72F3CF4873F914011F40C94EB2F0C9403
:10417000AF31803A43E0940709F4BBC2873E9340D5
:1041800011F40C943E310C94AF31A090C213B09056
:10419000C31380E50E94323B882359F00E948C3A79
:1041A0006B017C0111E0672B682B692B31F410E067
:1041B00004C010E0C12CD12C760183E50E94323B73
:1041C0008823F1F00E94D03A20E030E04AE754E43E
:1041D0000E94A5DC0E9456E16B017C01111112C006
:1041E000672B682B692B71F4A114B10459F0D50128
:1041F0008C91882339F061E0C5010E94FDC807C099
:10420000112391F360E08BE991E00E94DEC883E026
:1042100090E09093280B8093270B81E080935108C6
:104220000E9420480E944A3CC114D104E104F104D8
:10423000F1F08091030B9091040BA091050BB091CC
:10424000060BC80ED91EEA1EFB1E0E94F352DC01AB
:10425000CB018C199D09AE09BF09B7FF1EC0809123
:1042600051088823D1F080E00E942A7BEECF809114
:104270005108882321F080E00E942A7BF8CF8091AA
:10428000E50E9091E60E60E0029719F489E891E05E
:1042900002C08AE791E00E94DEC8109251080C9497
:1042A000AF3184918F010F5F1F4F882321F00E944F
:1042B000553CF801F6CF10927B1110927A1140E034
:1042C00050E0BA0186E29FE00E941DC28BE1E6E267
:1042D000FFE0DE01159601900D928A95E1F780913D
:1042E000240F9091250F9C838B8381EC91E09A831E
:1042F000898340E050E0BE016F5F7F4F8AE592E026
:104300000E94E77FCE0101960E94AF7AE7EBF1E0D1
:1043100084918F010F5F1F4F882311F40C94AF31EC
:104320000E94553CF801F4CF0E94CB9B0C94AF3116
:104330001092F50E1092F60E0C94AF31803209F403
:104340001082319680818111F9CF40E061E0809147
:10435000C2139091C3130E9428820C94AF3119822A
:104360001A821B821C8218A219A21AA21BA2809177
:10437000290B882341F040E0BE016F5F7F4FCE01E3
:1043800080960E948B7E8091F60E882319F081E042
:104390008093F50E0E94F89C0C94AF318091F60E3C
:1043A000882311F40C94AF3183E50E94323B8111D4
:1043B0000C94B6310C94AF318091F60E882351F1F4
:1043C000ECEDF1E084918F010F5F1F4F882321F006
:1043D0000E94553CF801F6CF6091711170917211F5
:1043E00080917311909174114AE00E9474408FE2A1
:1043F0000E94553C60916D1170916E1180916F110A
:10440000909170114AE00E9474408AE00E94553CED
:104410000C94AF31EEEEF1E084918F010F5F1F4FEE
:10442000882311F40C94AF310E94553CF801F4CF6D
:1044300040E060E08091C2139091C3130E942882F3
:104440000C94AF318091F60E882311F40C94AF31A7
:1044500080EC90E10E94DAC180EC90E10E94F0A52E
:104460001092F40E1092F30EE090C213F090C3136A
:104470008091F60E882311F40C94AF310E949CBBFE
:104480001D8218861C821B8281EC91E09A838983AD
:1044900082E29FE09093420F8093410FF701808169
:1044A0008F3209F068C06FE270E0C7010E94FBE242
:1044B0008C010F5F1F4F9E012F5F3F4F4901011578
:1044C000110509F45EC06FE270E0C8010E94FBE2D2
:1044D0006C01009709F456C00817190708F052C07C
:1044E0005C01A01AB10AA501B801CE0180960E9414
:1044F00024E3E0E2F0E0EC0FFD1FEA0DFB1D10826B
:104500008E01005E1F4FD8018D918D01882319F017
:104510000E94553CF8CF8AE00E94553C6091410FC3
:104520007091420F6115710511F06C5F7F4F21E0B2
:10453000AE01405E5F4FCE0105960E948CA98111AD
:1045400012C0BE01605E7F4F85E292E00E94ABC95F
:104550008EE20E94553C8AE00E94553CC4010E94B4
:10456000AF7A0C94AF319092420F8092410F860146
:104570000F5F1F4FA4CF83E49FE09093420F80937F
:10458000410F87016091410F7091420F61157105D4
:1045900011F06C5F7F4F18A21BA222E0A801CE0190
:1045A00080960E948CA9811102C0F12C1EC0CE0100
:1045B00080960E940ABB8823C1F36CA57DA58EA5B9
:1045C0009FA541E00E94C5BF882379F3E8A9B0E226
:1045D000EB9FF0011124ED5BF44F309731F385EE42
:1045E00080831BA20E9485BFF82ECE0180960E9478
:1045F0009B3BFF2009F1EFEFF1E084917F012FEF6A
:10460000E21AF20A882321F00E94553CF701F5CF07
:10461000D8018D918D01882319F00E94553CF8CF67
:104620008AE00E94553C1092711110927211109202
:1046300073111092741118C0EDE0F2E084917F01C3
:10464000BFEFEB1AFB0A882321F00E94553CF701CB
:10465000F5CFF80181918F01882319F00E94553C14
:10466000F8CF8EE20E94553CCE0101960E94AF7AAF
:104670000C94AF318091F50E81110E9420488091F9
:10468000F60E882311F40C94AF3180E50E94323B82
:10469000882319F00E94C03A03C080E50E94033BC2
:1046A000182F482F61E08091C2139091C3130E948C
:1046B000288283E50E94323B882381F00E949C3A45
:1046C000AB01BC014093711150937211609373114F
:1046D0007093741180EC90E10E941DC28091F60EDF
:1046E000882319F081E08093F50E11110C94AF31FD
:1046F00051CE8091C2139091C31321E02093F40E08
:1047000040E060E00E9428820C94AF310E949EBD80
:10471000ECE3CE2ED12CE12CF12CA70196010E94C6
:104720001DE0762E672ECA01B901A70196010E94ED
:104730001DE06B017C01CA01B90128E130E040E0D5
:1047400050E00E941DE04B015C01C9016DE671E083
:104750000E9462E28E010F5F1F4F6115710599F093
:104760006F927F92DF92CF929F928F929F938F93BF
:104770007F936F9381E692E09F938F931F930F93A4
:104780000E94D6DB12C00097B1F06F927F92DF9249
:10479000CF929F928F929F938F9381E592E09F9308
:1047A0008F931F930F930E94D6DB0FB6F894DEBF52
:1047B0000FBECDBF36C081149104A104B10479F0BD
:1047C0006F927F92DF92CF929F928F9285E492E0D8
:1047D0009F938F931F930F930E94D6DBE6CFC11454
:1047E000D104E104F10469F06F927F92DF92CF92DD
:1047F0008DE392E09F938F931F930F930E94D6DBDC
:10480000D4CF6F927F9289E392E09F938F931F930F
:104810000F930E94D6DB0F900F900F900F900F9088
:104820000F9060E0C8010E94FDC8E3E5FCE18491BF
:104830007F01BFEFEB1AFB0A882321F00E94553C51
:10484000F701F5CFB80185E792E00E94ABC98AE095
:104850000E94553C0C94AF3183E50E94323B882383
:1048600011F40C94AF310E94AC3AE82E80E50E941E
:10487000323B882311F40C94AF310E949C3A162FDE
:10488000C62ED72ED7FE02C00C94AF31E2E8F2E07C
:1048900088E28E0F9491191729F031968E13FACF72
:1048A0000C94C731E8E3FCE184918F010F5F1F4F47
:1048B000882321F00E94553CF801F6CFEAEAF2E0A5
:1048C00084918F010F5F1F4F882311F40C94AF3137
:1048D0000E94553CF801F4CF0E94F89C0C94AF3133
:1048E0000E94149E0C94AF310E94A7BB0C94AF3170
:1048F00088E690E00E94DC4081110C94AF318091F9
:10490000510E83FF02C00C94AF3183E50E94323B0D
:10491000882309F440C00E94D03A0E944FE170936E
:10492000E40D6093E30D80E00E9424450E94D03A9C
:1049300020E030E04AEA52E40E943FDC18163CF0E6
:104940000E94A7BB60E080EC92E00E94DEC80E945B
:10495000D03A2091560E3091570E4091580E5091FA
:10496000590E0E94DDE11816B4F480EE91E09F9399
:104970008F938091350E90E001969F938F9389EBF2
:1049800092E09F938F931F920E94DD9C0FB6F89444
:10499000DEBF0FBECDBF0E948AD70C94AF318EE42C
:1049A0000E94323B882311F40C94AF310E949C3A50
:1049B0006093290E70932A0E80932B0E90932C0EE9
:1049C0000C94AF3183E50E94033B882359F083E5C3
:1049D0000E94323B882319F00E94AC3A01C080E06B
:1049E0008093510EE3E5FCE184918F010F5F1F4F2F
:1049F000882321F00E94553CF801F6CFE0EEF2E06A
:104A000084918F010F5F1F4F882321F00E94553C36
:104A1000F801F6CF8091510E8823A1F172EDC72ED7
:104A200072E0D72EE12CF12C20E08091510E90E025
:104A30000E2C02C0959587950A94E2F780FF17C067
:104A4000BB24B394B20E222319F08CE20E94553C91
:104A5000F60125913491F901849189010F5F1F4F6F
:104A6000882321F00E94553C9801F5CF2B2DFFEFB4
:104A7000EF1AFF0A32E0C30ED11C45E0E416F10440
:104A8000A1F60CC0ECEDF2E084918F010F5F1F4F97
:104A9000882321F00E94553CF801F6CF8AE00E945D
:104AA000553C0C94AF3187EE92E00E94C17A83E5C9
:104AB0000E94323B882369F00E94AC3A8D3320F487
:104AC00080932B010C94AF318CE380932B010C94D9
:104AD000AF31E3E5FCE184918F010F5F1F4F882325
:104AE00021F00E94553CF801F6CF40912B0150E097
:104AF00060E070E080EF92E00E943BC98AE00E9493
:104B0000553C0C94AF318091510E83FF02C00C9440
:104B1000AF3183E50E94323B882311F40C94AF310E
:104B20000E94D03A0E944FE16437710514F063E7A8
:104B300070E07093E80D6093E70D0C94AF3189E657
:104B400090E00E94DC40811111C0E7EFF2E0849117
:104B50008F010F5F1F4F882321F00E94553CF80101
:104B6000F6CF0E9431A28AE00E94553C1092280B99
:104B70001092270B0C94C43683E50E94323B8823A5
:104B800011F40C94AF310E94AC3A182F8D3308F019
:104B90001CE31093000B0E94F3526B017C01212F48
:104BA00030E0A8EEB3E00E944AE0C60ED71EE81E31
:104BB000F91EC092FC0AD092FD0AE092FE0AF09221
:104BC000FF0A0C94AF318DE690E00E94DC40811129
:104BD0000C94AF318091510E83FF02C00C94AF3121
:104BE00083E50E94323B60968FAF609781110C94F1
:104BF000DD3182E50E94323B81110C94DD310C9451
:104C0000AF318091510E83FF02C00C94AF3160E050
:104C100083E393E00E94DEC883E50E94323B609606
:104C20008FAF609781110C94783382E50E94323BFC
:104C300081110C9478330C94AF3180E50E94323BA3
:104C4000811108C083E50E94323B811109C03FEF0A
:104C500020E00AC00E94AC3A81110C94AF31F2CF2F
:104C60000E949C3A362F272F832F922F8F3F91053A
:104C700019F010F08FEF90E09093E60D8093E50D22
:104C80000C94AF3180E50E94323B811106C0109236
:104C9000E60D1092E50D0C94AF310E949C3A672B03
:104CA00011F00C94AF31F3CF8CE40E94033B8823C6
:104CB00019F00E94D03A04C060E070E080E090EC0F
:104CC0006BAF7CAF8DAF9EAF80E090E0A0E0B1E431
:104CD00089839A83AB83BC8380E090E0A1E9B3E44D
:104CE0008D839E83AF83B88780E090E0A0EAB1E433
:104CF00089879A87AB87BC8788E50E94323B8823E7
:104D000079F088E50E94323B882319F00E94D03A5E
:104D100003C060E070E0CB0169837A838B839C835E
:104D200089E50E94323B882379F089E50E94323B75
:104D3000882319F00E94D03A03C060E070E0CB01F4
:104D40006D837E838F8398878AE50E94323B882318
:104D500079F08AE50E94323B882319F00E94D03A0C
:104D600003C060E070E0CB0169877A878B879C87FE
:104D700018A219A21AA21BA28091290B81110C94CE
:104D8000AF3100E020E0AE01405E5F4FBE016F5FDB
:104D90007F4FCE01CB960E949C7D0C94AF31109238
:104DA0007F020C94AF3181E080937F020C94AF318D
:104DB00083E50E94323B8823A1F00E94D03A20E094
:104DC00030E04AE754E40E94A5DC0E9456E160937B
:104DD0002C0170932D0180932E0190932F010C9440
:104DE000AF3188E50E94033B81110C94E33489E5DF
:104DF0000E94033B81110C94E3348AE50E94033B3B
:104E000081110C94E33485E40E94033B81110C94DE
:104E1000E3340E9420480E94B77A0C94AF3183E5B6
:104E20000E94033B882311F40C94AF310E94D03AC6
:104E300020E030E04AE754E40E94A5DC0E9456E1FD
:104E40006093070B7093080B8093090B90930A0BE8
:104E50000C94AF31D6018D916D010E94033B8823E4
:104E600009F46DC0133009F063C00E94D03A4B01C1
:104E70005C0120E030E040EA51E40E943FDC87FF23
:104E80004EC0A501940160911F0E7091200E80917B
:104E9000210E9091220E0E94DDE02B013C019B012E
:104EA000AC0160917A0D70917B0D80917C0D909199
:104EB0007D0D0E94A5DC60937A0D70937B0D80932D
:104EC0007C0D90937D0DA30192016091600A709119
:104ED000610A8091620A9091630A0E94A5DC609346
:104EE000600A7093610A8093620A9093630A6091EA
:104EF000A0137091A1138091A2139091A3130E940B
:104F000044DCA30192010E94A5DC0E9456E160935B
:104F1000A0137093A1138093A2139093A313809274
:104F20001F0E9092200EA092210EB092220E07C06A
:104F30000E94D03AF70160837183828393831F5F5D
:104F4000F4E0EF0EF11C143009F084CF0E94FFCA88
:104F50000C94AF310E9420480E94F3410C94AF3171
:104F600084918F010F5F1F4F882321F00E94553CD1
:104F7000F801F6CF60E087EF93E00E943A4160E0ED
:104F800080EF93E00E943A4161E085EE93E00E9459
:104F90003A4161E085ED93E00E943A4160E08CEC9B
:104FA00093E00E943A4161E082EC93E00E943A4132
:104FB00060E088EB93E00E943A4160E080EB93E090
:104FC0000E943A4160E082EA93E00E943A4160E048
:104FD00084E993E00E943A4160E085E893E00E9412
:104FE0003A4160E087E793E00E943A4160E081E661
:104FF00093E00E943A4160E080E593E00E943A41EC
:105000000C94AF3160E08091C2139091C3130E9461
:10501000FDC80C94AF3185E40E94323B882319F01F
:105020000E94C03A03C085E40E94033B882361F0DC
:10503000E3E5FCE184918F010F5F1F4F882321F08E
:105040000E94553CF801F6CF81E40E94323B882350
:1050500019F00E94C03A03C081E40E94033B8823F8
:1050600061F0E0EDF4E084918F010F5F1F4F882322
:1050700021F00E94553CF801F6CF0091C213109127
:10508000C313D8018D918D01882309F407CD0E94A7
:10509000553CF7CFECEEF4E084918F010F5F1F4F8A
:1050A000882321F00E94553CF801F6CFE4EEF4E0AD
:1050B00084918F010F5F1F4F882321F00E94553C80
:1050C000F801F6CF329B03C00DEC11E002C002EDF7
:1050D00011E0F80181918F01882319F00E94553C5D
:1050E000F8CF8AE00E94553CECEDF4E084918F010A
:1050F0000F5F1F4F882321F00E94553CF801F6CF27
:10510000339B03C00DEC11E002C002ED11E0D801A9
:105110008D918D01882319F00E94553CF8CF8AE0CB
:105120000E94553CE4EDF4E084918F010F5F1F4F26
:10513000882321F00E94553CF801F6CF349B03C030
:105140000DEC11E002C002ED11E0F80181918F0138
:10515000882309F4A3CC0E94553CF7CF81E08093CB
:10516000C60E8093C50E0C94AF311092C60E1092ED
:10517000C50E0C94AF3183E50E94323B882319F0B1
:105180000E949C3A02C060E070E08B01112702305F
:105190001105D4F0E8E3FCE184918F010F5F1F4F0C
:1051A000882321F00E94553CF801F6CFE6E0F5E0B7
:1051B00084918F010F5F1F4F882311F40C94AF313E
:1051C0000E94553CF801F4CF88E40E94323B8823CA
:1051D000A9F00E949C3A6A3A71053CF06530F1E012
:1051E0007F072CF064E071E002C06AEA70E0F80129
:1051F000EE0FFF1FEC5BF54F7183608386E40E9426
:10520000323B8823A9F00E949C3AF801EE0FFF1F61
:10521000E85BF54F718360836F3F710519F014F0FF
:105220006FEF70E077FF02C060E070E07183608331
:1052300082E40E94323B882311F40C94AF310E9427
:105240009C3A6530710534F0653671052CF064E6E2
:1052500070E002C065E070E0000F111FF801E05C33
:10526000F54F718360830C94AF3188EC90E00E941D
:10527000DC4081110C94AF3184E40E94033B88230D
:10528000C1F10E94D03A11E020E030E0A9010E9473
:105290003FDC811101C010E01093820D112349F110
:1052A0000E94D03AE091350E24E0E29FF0011124F3
:1052B000E258F24F608371838283938320E030E071
:1052C000A90160917E0D70917F0D8091800D90916C
:1052D000810D0E943FDC81110CC080E090E0A0EEC7
:1052E000BFE380937E0D90937F0DA093800DB093CC
:1052F000810D0E947EAA0C94AF31E2E5EE2EEDE026
:10530000FE2E03E911E0F4E0DF2ED00ED8018D91DE
:105310008D010E94033B882349F00E94D03A0E94ED
:1053200056E1F7016083718382839383F4E0EF0E8B
:10533000F11CD012EBCF0E94D2C90C94AF31F4E033
:10534000EF0EF11CD01611F40C94AF31D8018D91F1
:105350008D010E94033B882391F30E94D03AF7010C
:105360006083718382839383EACF83E50E94033B4A
:105370008823D9F00E94D03AAB01BC0140936A0D5A
:1053800050936B0D60936C0D70936D0D4093620D97
:105390005093630D6093640D7093650D82E895E002
:1053A0000E9475C98AE00E94553C80E50E94033B3B
:1053B000882399F00E94D03AAB01BC0140936A0D5A
:1053C00050936B0D60936C0D70936D0D85E695E0B9
:1053D0000E9475C98AE00E94553C82E50E94033B09
:1053E000882399F00E94D03AAB01BC014093660D2E
:1053F0005093670D6093680D7093690D86E495E096
:105400000E9475C98AE00E94553C84E50E94033BD6
:10541000882309F4A4C70E94D03AAB01BC01409391
:10542000620D5093630D6093640D7093650D88E277
:1054300095E00E9475C98AE00E94553C90C783E5BB
:105440000E94033B882351F00E94D03A6093500A97
:105450007093510A8093520A9093530A84E50E94F4
:10546000033B882351F00E94D03A60934C0A70931A
:105470004D0A80934E0A90934F0A82E40E94033BA8
:10548000882351F00E948C3A6093470E7093480E27
:105490008093490E90934A0E88E50E94033B88232F
:1054A00051F00E94D03A60936E0D70936F0D80930F
:1054B000700D9093710D89E50E94033B882351F094
:1054C0000E94D03A6093720D7093730D8093740DA7
:1054D0009093750D8AE50E94033B882351F00E944A
:1054E000D03A6093760D7093770D8093780D9093FA
:1054F000790D85E40E94033B882309F430C70E949C
:10550000D03A60937A0D70937B0D80937C0D9093CD
:105510007D0D25C70F5F1F4FF4E0EF0EF11C033028
:10552000110511F40C94EB1ED6018D916D010E94B2
:10553000033B882379F30E94D03AF701608371839B
:1055400082839383C8010E945039E4CF0E94F93CC2
:1055500006C783E50E94323B882309F400C70E94F6
:105560009C3A7093410160934001F9C68DED90E043
:105570000E94DC408111F3C683E50E94323B882300
:1055800009F4EDC60091350E10E00E949C3A000F20
:10559000111FF801E25CFE4F718360838091350E2C
:1055A00090E08C01000F111F000F111F9801285C63
:1055B0003E4F7901880F991FFC01E25CFE4F60812C
:1055C0007181072E000C880B990B0E9446DC2AE0A3
:1055D00037ED43E25CE30E94A5DCF801EE5AF14F9F
:1055E00020813181428153810E94A5DCD7016D93D6
:1055F0007D938D939C931397B2C60E943F3BAFC699
:1056000083E50E94323B882319F00E949C3A02C035
:1056100064E071E079A368A380E50E94323B8823AF
:1056200039F00E949C3A6938B3E17B0730F402C03C
:1056300068EE73E07A83698304C088E893E19A8313
:105640008983BE01605E7F4FCE0101960E94A99CB6
:1056500086C60E945C3C83C683E50E94033B182FEC
:10566000882371F00E94D03A0E944FE170933D016F
:1056700060933C0121E0672B09F020E020935A0E53
:1056800080E50E94033B882359F020913C01309132
:105690003D01232B11F00E94C03A80935A0E5FC641
:1056A00011115DC6E3E5FCE184918F010F5F1F4F8F
:1056B000882321F00E94553CF801F6CF80915A0EC4
:1056C000811103C06CED71E002C06FEC71E08FEBF3
:1056D00095E00E94ABC960913C0170913D018EEA5A
:1056E00095E00E9492C9EAEAF5E084918F010F5F8C
:1056F0001F4F882309F433C60E94553CF801F5CFAB
:1057000085E40E94323B882321F00E949C3A7B0171
:1057100002C0E12CF12C83E40E94323B882331F05B
:105720000E949C3AA9966FAFA99704C025E0A9965C
:105730002FAFA99785E50E94323B882319F00E947C
:10574000C03A03C085E50E94033BE5968FAFE5971D
:10575000F7FC07C0812C912CB6E1AB2EB3E4BB2E35
:1057600006C0812C912CACE8AA2EA2E4BA2E83E5C7
:105770000E94323B882321F00E94D03A4B015C0109
:10578000E114F10411F41092350E0E94F3522B0132
:105790003C01E11003C00BEE11E00BC00EEF11E075
:1057A000D8018D918D01882309F478C90E94553C58
:1057B000F7CFF80181918F01882319F00E94553CA1
:1057C000F8CFC501B4010E944FE1072E000C880BF1
:1057D000990B0E9446DC60966FAF609761967FAF31
:1057E000619765968FAF659766969FAF6697A301A1
:1057F0009201205E314B4F4F5F4FC358DF4F2883DC
:1058000039834A835B83CD57D0408AE00E94553C60
:105810000E946F458FE78093330E81E080933701BC
:10582000E0964CAE5DAE6EAE7FAEE097E9964CAEC4
:105830005DAE6EAE7FAEE997AC961FAEAC97ED96BF
:105840001CAE1DAE1EAE1FAEED9769961FAE6997DA
:1058500030E46A963FAF6A974CE16B964FAF6B9717
:1058600056E46C965FAF6C976D961FAE6D976E9613
:105870001FAE6E976F961FAE6F97A0961FAEA09744
:10588000A8961CAE1DAE1EAE1FAEA897A4961CAE69
:105890001DAE1EAE1FAEA497C12CD12C7601FFE722
:1058A0008F2E912CA12CB12C8FE790E0A0E0B0E0DE
:1058B0002F968CAF9DAFAEAFBFAF2F97E4961CAEC7
:1058C0001DAE1EAE1FAEE49791E0AB969FAFAB97B7
:1058D00068961FAE1EAE689710E0212C312C00E0B8
:1058E000A996AFADA9970A2E000CBB0BAA96BFAF25
:1058F000AEAFAA9780913701882309F402C10E94B4
:10590000F3522B966CAF7DAF8EAF9FAF2B978091EC
:10591000310E882309F4D1C00E942F461091560EF3
:105920002090570E3090580E0091590E212F322D95
:10593000432D502F6D966FAD6D976E967FAD6E9720
:105940006F968FAD6F97A0969FADA0970E943FDC9A
:1059500087FF0CC06D961FAF6D976E962FAE6E973A
:105960006F963FAE6F97A0960FAFA097212F322D65
:10597000432D502F69966FAD69976A967FAD6A97F0
:105980006B968FAD6B976C969FAD6C970E94DDE127
:10599000181664F469961FAF69976A962FAE6A97D6
:1059A0006B963FAE6B976C960FAF6C97AB96BFAD97
:1059B000AB9760962FAD609761963FAD6197659606
:1059C0004FAD659766965FAD6697612F722D832DFB
:1059D000902FBB2309F455C00E94DDE118160CF08E
:1059E0006CC02B964CAD5DAD6EAD7FAD2B97441961
:1059F000550966097709DB01CA0188589341A10955
:105A0000B109B7FD5AC02F968CAD9DADAEADBFADFF
:105A10002F9788199909AA09BB09B595A795979554
:105A200087958093330EE4964CAF5DAF6EAF7FAF3A
:105A3000E4976096EFAD60976D96EFAF6D976196C6
:105A4000FFAD61976E96FFAF6E9765962FAD659728
:105A50006F962FAF6F9766963FAD6697A0963FAF54
:105A6000A0972B968CAD9DADAEADBFAD2B97E096BC
:105A70008CAF9DAFAEAFBFAFE097AB961FAEAB970D
:105A80001CC00E943FDC87FF18C02B968CAD9DADDB
:105A9000AEADBFAD2B97E0962CAD3DAD4EAD5FAD3D
:105AA000E097821B930BA40BB50BAC01BD014858CA
:105AB00053416109710977FFA2C720E030E040EA55
:105AC00051E460966FAD609761967FAD6197659682
:105AD0008FAD659766969FAD66970E945AE09B01D1
:105AE000AC01612F722D832D902F0E94DDE11816DD
:105AF0007CF4EAECF6E084918F010F5F1F4F811177
:105B000003C00E946F452BC40E94553CF801F3CF9F
:105B10002B968CAD9DADAEADBFAD2B97E9962CAD60
:105B20003DAD4EAD5FADE997821B930BA40BB50B5A
:105B3000B7FDABC00E9431A28AE00E94553C2B9673
:105B40008CAD9DADAEADBFAD2B978053984FAF4F91
:105B5000BF4FE9968CAF9DAFAEAFBFAFE997AC96A4
:105B60009FADAC9791116EC0ED962CAD3DAD4EAD95
:105B70005FADED97612F722D832D902F0E94DDE197
:105B800018160CF046C020E030E040E051E460968A
:105B90006FAD609761967FAD619765968FAD6597A4
:105BA00066969FAD66970E9459E09B01AC01A1E00B
:105BB000AC96AFAFAC97612F722D832D902F0E94C2
:105BC000DDE118161CF0AC961FAEAC9720E030E07B
:105BD00040E050E4612F722D832D902F0E945AE0F7
:105BE000ED966CAF7DAF8EAF9FAFED972B962CAD42
:105BF0003DAD4EAD5FAD2B97205E314B4F4F5F4FAC
:105C0000C358DF4F288339834A835B83CD57D04005
:105C10003CC02B968CAD9DADAEADBFAD2B97C358A0
:105C2000DF4F288139814A815B81CD57D040821B6B
:105C3000930BA40BB50BB7FD28C04CEA56E06BEBF9
:105C400076E020C020E030E040EA51E460966FAD9D
:105C5000609761967FAD619765968FAD6597669603
:105C60009FAD66970E9459E09B01AC01612F722D98
:105C7000832D902F0E943FDC87FF07C04CE856E041
:105C80006CE976E080E00E9453462B968CAD9DAD8A
:105C9000AEADBFAD2B97880F991FAA1FBB1FE09613
:105CA0002CAD3DAD4EAD5FADE097821B930BA40BC9
:105CB000B50B84199509A609B70981389F44A241FB
:105CC000B10568F0EEE6F6E084918F010F5F1F4F9B
:105CD000882309F416CF0E94553CF801F5CF689649
:105CE0004EAD5FAD6897AA968EAD9FADAA9784170B
:105CF00095070CF066C0E1E1F6E084918F010F5F3B
:105D00001F4F882321F00E94553CF801F6CFB701C0
:105D1000A6018CEF95E00E9475C98AE00E94553C6F
:105D2000A4964CAD5DAD6EAD7FADA49787EE95E0CA
:105D30000E9475C98AE00E94553CA8964CAD5DADA5
:105D40006EAD7FADA89782ED95E00E9475C98AE09F
:105D50000E94553CE5969FADE597992309F4FFC253
:105D6000C092330AD092340AE092350AF092360A91
:105D70002CEA35EC47E25EE3A4966CAD7DAD8EADCA
:105D80009FADA4970E94A5DC60933B0A70933C0AE8
:105D900080933D0A90933E0A2CEA35EC47E25EE39D
:105DA000A8966CAD7DAD8EAD9FADA8970E94DDE04D
:105DB0006093370A7093380A8093390A90933A0AAD
:105DC000CEC20E94585C96CD0E942048C8C20E9454
:105DD000389D8111C4C29DE8892E9AE1992EA3E0D5
:105DE000BEE02996BFAFAEAF2997FE0131965F01A5
:105DF00006EE1AE11F01F3E0F00F2C96FFAF2C978F
:105E0000F40165917591859194912996AEADBFADE0
:105E10002997CD90DD90ED90FD902996BFAFAEAF64
:105E20002997A70196010E9459E02B013C0120E02F
:105E300030E040EA51EC0E94DDE187FD10C020E037
:105E400030E040EA51E4C301B2010E943FDC181681
:105E500034F0F10140825182628273820DC0F801F8
:105E600084911816B4F7F7FAF094F7F8F094F1016A
:105E7000C082D182E282F382D101CD90DD90ED909B
:105E8000FD901D0120E030E040EA51ECC701B60171
:105E90000E94DDE187FF03C0E8E3FCE10BC020E0E6
:105EA00030E040EA51E4C701B6010E943FDC181619
:105EB00074F5F2CF84918F010F5F1F4F882321F07B
:105EC0000E94553CF801F6CFECE5F7E084918F0194
:105ED0000F5F1F4F882321F00E94553CF801F6CF39
:105EE00061E08EE497E00E94DEC80E94509B88E249
:105EF00090E099A388A388EC90E09CAF8BAFBE01A3
:105F0000605E7F4FCE01CB960E94A99C28C2B4E070
:105F10008B0E911C0F5F1F4F2C96EFAD2C97E0134B
:105F20006FCF8DE6E82E88E0F82E00E010E0F50156
:105F300081919191A191B1915F01F7018193919329
:105F4000A193B1937F01C8010E9450390F5F1F4F89
:105F50000330110561F70E94F34160E08EE397E0A2
:105F60000E94DEC883E992E09CAF8BAF04E610E0AC
:105F700019A308A3BE01655C7F4FCE0180960E94E5
:105F8000A99C8AEB92E09CAF8BAF19A308A3BE013A
:105F9000655C7F4FCE0180960E94A99CE0C1E8E33A
:105FA000FCE184918F010F5F1F4F882321F00E9435
:105FB000553CF801F6CFEAE7F7E084918F010F5FD7
:105FC0001F4F882309F4CBC10E94553CF801F5CF3F
:105FD0000E94D4BDC4C183E50E94033B882321F005
:105FE0000E94C03A91E089270E946792B8C180E080
:105FF00090E0A0E0B1E489839A83AB83BC8380E026
:1060000090E0A1E9B3E48D839E83AF83B88780E0FD
:1060100090E0A0EAB1E489879A87AB87BC870E94A9
:10602000389D882319F081E00E94D04285E40E94C7
:10603000033B882319F00E94D03A04C060E070E06E
:1060400080E090EC27966CAF7DAF8EAF9FAF279727
:106050008AE50E94323B882379F08AE50E94323B30
:10606000882319F00E94D03A03C060E070E0CB01B1
:1060700069877A878B879C8788E50E94323B8823D3
:1060800079F088E50E94323B882319F00E94D03ACB
:1060900003C060E070E0CB0169837A838B839C83CB
:1060A00089E50E94323B882379F089E50E94323BE2
:1060B000882319F00E94D03A03C060E070E0CB0161
:1060C0006D837E838F83988785E50E94033B8823B9
:1060D00019F00E94D03A04C060E070E082E094ECD5
:1060E00023966CAF7DAF8EAF9FAF23978CE40E9459
:1060F000033B882319F00E94D03A04C060E070E0AE
:106100008AEF93E46BAF7CAF8DAF9EAF82E40E94C9
:10611000323B882321F00E949C3A162F01C015E0E3
:10612000E090E50EF090E60E8091C31081110AC058
:1061300080E090E0A0EAB1E427968CAF9DAFAEAFCF
:10614000BFAF27978091290B81117AC001E0212FE1
:10615000AE01415C5F4FBE016F5F7F4FCE018D5B33
:106160009F4F0E949C7D882309F46AC083E090E0E1
:106170009093280B8093270B81E0809351088091A6
:106180005108882309F442C060E0812F0E94C5377E
:1061900080915E0E8823B1F188E090E00E94705FEC
:1061A00080915108882321F081E00E942A7BF8CF5A
:1061B0001092D6071092D7071092D8071092D907DD
:1061C00010925E0E0E9424450E946D3782E090E09E
:1061D0000E94705F0E94F352DC01CB01885390450E
:1061E000AF4FBF4F8093D6079093D707A093D807A0
:1061F000B093D90710925E0E0093510861E0812F91
:106200000E94C53781E00E942A7BB9CF81E090E0EF
:106210009093280B8093270B80E090E0A8ECB2E4E9
:1062200088A399A3AAA3BBA38091290B882341F03B
:10623000412FBE01605E7F4FCE01CB960E948B7EC8
:10624000EA94EF2809F08BC00E94F89C88C08491E2
:106250008F010F5F1F4F882321F00E94553CF801EA
:10626000F6CFEBE8F7E084918F010F5F1F4F882393
:1062700009F475C00E94553CF801F5CF81E0809388
:1062800009011092260E83E50E94323B882319F003
:106290000E94C03A03C083E50E94033B81115FC0A6
:1062A0000E94BC7F5CC0F090C413FF2029F1E3E59D
:1062B000FCE184918F010F5F1F4F882321F00E9422
:1062C000553CF801F6CF84E50E94553C6F2D70E0F7
:1062D00080E090E04AE00E94744080E20E94553CD9
:1062E00007E212E0D8018D918D01882311F40C94FE
:1062F0004E250E94553CF6CF1092360EE3E5FCE1A8
:1063000084918F010F5F1F4F882321F00E94553C1D
:10631000F801F6CF6091360E70E08AE997E00E94AE
:1063200092C98AE00E94553C1AC0E3E5FCE18491E1
:106330008F010F5F1F4F882321F00E94553CF80109
:10634000F6CF6091010B7091020B8CEA97E00E94EE
:10635000ABC982E20E94553C8AE00E94553C1092F3
:10636000280B1092270B0E949D7F0EC50E949C3A1D
:10637000AB01BC0140937111509372116093731182
:106380007093741180EC90E10E941DC2E8CF61E02F
:10639000812F0E9487606E2D812F0E945760F12C03
:1063A000B701812F0E944752B4E0CB16D104B9F651
:1063B000F092E60DE092E50DD2CF0E94D03A0E9415
:1063C0004FE17093E40D6093E30D80E00E9424455B
:1063D0000E94D03A20E030E04AEA52E40E943FDCDA
:1063E000181644F00E94A7BB60E083E193E00E948E
:1063F000DEC802C00E94F89C6091E30D7091E40D2C
:10640000072E000C880B990B0E9446DC2091560E3B
:106410003091570E4091580E5091590E0E94DDE177
:106420001816B4F480EE91E09F938F938091350E0F
:1064300090E001969F938F938CE093E09F938F93CE
:106440001F920E94DD9C0FB6F894DEBF0FBECDBF39
:106450000E948AD781E0809337012F961CAE1DAE33
:106460001EAE1FAE2F9764961CAE1DAE1EAE1FAEA5
:10647000649728961FAE289765961FAE65979CE394
:1064800066969FAF6697ACE16796AFAF6797B6E445
:106490006996BFAF6997C12CD12C50E8E52E6FEB00
:1064A000F62E812C912C54016091E30D7091E40D36
:1064B000072E000C880B990B0E9446DC162F072F25
:1064C000782E692E262F372F482F592FB601C70156
:1064D0000E943FDC882331F12091560E3091570EF7
:1064E0004091580E5091590E612F702F872D962D87
:1064F0000E943FDC881F8827881F28968FAF289727
:106500006096EFAD6097EE2389F0882379F0809153
:106510003701882309F423CF60E08AEF92E00E94DC
:10652000DEC81DCF1C2D0D2D7E2C6F2C0E94F3522A
:106530006B017C01DC01CB0164962CAD3DAD4EAD11
:106540005FAD6497821B930BA40BB50BB7FD3DC0E9
:10655000D701C60188519C4FAF4FBF4F64968CAF97
:106560009DAFAEAFBFAF64970E9431A2E8E0F3E009
:1065700084912F019FEF491A590A882321F00E9424
:10658000553CF201F5CF81149104A104B104B9F096
:10659000D501C401805F984DAF4FBF4FBC01CD0105
:1065A0006C197D098E099F0928EE33E040E050E028
:1065B0000E941DE0CA01B9010E941E4103C08FE381
:1065C0000E94553C8AE00E94553C80E00E942A7B54
:1065D0000E944A3C2090560E3090570E4090580E24
:1065E0005090590E9101A201612F702F872D962D89
:1065F0000E9459E09F7781149104A104B10449F4E9
:1066000020E030E040E85FE30E943FDC87FF0BC002
:1066100008C020E030E040EA50E40E94DDE11816B6
:1066200014F4460157012896AFAD2897AA2309F420
:1066300043C02F962CAD3DAD4EAD5FAD2F972115CC
:1066400031054105510541F0D701C601821B930B6D
:10665000A40BB50BB7FD30C09101A20165966FADDB
:10666000659766967FAD669767968FAD67976996D3
:106670009FAD69970E9459E020E030E040EC5FE375
:106680000E943FDC87FD43CFD701C601805A954168
:10669000AF4FBF4F2F968CAF9DAFAEAFBFAF2F9711
:1066A00065962FAE659766963FAE669767964FAE36
:1066B000679769965FAE699780913701882309F4DF
:1066C00026CF81149104A104B10429F4C12ED02E47
:1066D000E72CF62CE9CE90E1C91A97E2D90AE10835
:1066E000F108C818D908EA08FB08F7FE10CFEECF6A
:1066F0000E94D03A0E944FE16437710514F063E7BD
:1067000070E07093E80D6093E70D0E94D03A20E0AE
:1067100030E040EA50E40E94DDE1181614F40E94D3
:10672000F89C81E0809337018091360E8093350E7E
:106730002F961CAE1DAE1EAE1FAE2F9764961CAEDC
:106740001DAE1EAE1FAE649728961FAE28976596A5
:106750001FAE6597ACE36696AFAF6697BCE16796F0
:10676000BFAF6797E6E46996EFAF6997C12CD12C6C
:1067700030E8E32E4FEBF42E812C912C54016091E4
:10678000E70D7091E80D072E000C880B990B0E9405
:1067900046DC162F072F782E692E262F372F482FED
:1067A000592FB601C7010E943FDC882331F12091A7
:1067B0008B0D30918C0D40918D0D50918E0D612F70
:1067C000702F872D962D0E943FDC881F8827881FF9
:1067D00028968FAF28976096FFAD6097FF2389F0CA
:1067E000882379F080913701882309F4B8CD60E0DF
:1067F00085E293E00E94DEC8B2CD1C2D0D2D7E2CCB
:106800006F2C0E94F3526B017C01DC01CB0164967A
:106810002CAD3DAD4EAD5FAD6497821B930BA40BC9
:10682000B50BB7FD3DC0D701C60188519C4FAF4F96
:10683000BF4F64968CAF9DAFAEAFBFAF64970E9461
:1068400031A2EFE2F3E084912F019FEF491A590A38
:10685000882321F00E94553CF201F5CF8114910468
:10686000A104B104B9F0D501C401805F984DAF4FC8
:10687000BF4FBC01CD016C197D098E099F0928EE1F
:1068800033E040E050E00E941DE0CA01B9010E94DF
:106890001E4103C08FE30E94553C8AE00E94553C94
:1068A00080E00E942A7B0E944A3C20908B0D309011
:1068B0008C0D40908D0D50908E0D9101A201612F95
:1068C000702F872D962D0E9459E09F778114910497
:1068D000A104B10449F420E030E040E85FE30E9405
:1068E0003FDC87FF0BC008C020E030E040E450E40C
:1068F0000E94DDE1181614F4460157012896AFAD49
:106900002897AA2309F443C02F962CAD3DAD4EAD78
:106910005FAD2F97211531054105510541F0D70194
:10692000C601821B930BA40BB50BB7FD30C09101C0
:10693000A20165966FAD659766967FAD669767967F
:106940008FAD679769969FAD69970E9459E020E0E7
:1069500030E040EC5FE30E943FDC87FD43CFD7018E
:10696000C601805A9541AF4FBF4F2F968CAF9DAF58
:10697000AEAFBFAF2F9765962FAE659766963FAEC9
:10698000669767964FAE679769965FAE69978091F5
:106990003701882309F426CF81149104A104B1049E
:1069A00029F4C12ED02EE72CF62CE9CE90E1C91A9D
:1069B00097E2D90AE108F108C818D908EA08FB08E3
:1069C000F7FE10CFEECF0E94204888E50E94033BDF
:1069D000882319F05E9A10926A0889E50E94033BA9
:1069E000882319F05E9A10926B088AE50E94033B97
:1069F000882309F4B4CC159A10926C08B0CC689630
:106A00004EAD5FAD6897452B09F481C1E4964CAC5F
:106A10005DAC6EAC7FACE497480E591E6A1E7B1EBF
:106A2000E4962CAD3DAD4EAD5FADE497281B390B20
:106A30004A0B5B0BCA01B901A50194010E940DE04C
:106A4000A30192010E948AE22F968CAC9DACAEAC61
:106A5000BFAC2F97820E931EA41EB51E34E1831681
:106A60009104A104B1041CF14CEE84169104A1041C
:106A7000B1043CF450E885169104A104B10434F447
:106A800026C05BEE852E912CA12CB12C2F968CAEBE
:106A90009DAEAEAEBFAE2F978EEF90E0A0E0B0E01F
:106AA00088199909AA09BB094C015D0116C024E1A6
:106AB00030E040E050E02F962CAF3DAF4EAF5FAFDF
:106AC0002F9744E1842E912CA12CB12C06C02F9637
:106AD0008CAE9DAEAEAEBFAE2F97E6E3F7E08491ED
:106AE0009F012F5F3F4F8823C1F0CF57DF4F28838F
:106AF000C158D040CE57DF4F3883C258D0400E9493
:106B0000553CCF57DF4F2881C158D040CE57DF4F7B
:106B10003881C258D040F901E2CF2F966CAD7DADDF
:106B20008EAD9FAD2F970E941E41E1E3F7E0849167
:106B30009F012F5F3F4F8823C1F0CF57DF4F28833E
:106B4000C158D040CE57DF4F3883C258D0400E9442
:106B5000553CCF57DF4F2881C158D040CE57DF4F2B
:106B60003881C258D040F901E2CFC501B4010E947A
:106B70001E4169964FAD69976A965FAD6A976B96AD
:106B80006FAD6B976C967FAD6C978AE297E00E9431
:106B900075C96D964FAD6D976E965FAD6E976F969A
:106BA0006FAD6F97A0967FADA09783E297E00E94AC
:106BB00075C968964EAD5FAD6897433051050CF4CA
:106BC000A6C0C501B4010E9446DC20E030E040E8E8
:106BD00050E40E94A5DC6B017C0169962FAD69979A
:106BE0006A963FAD6A976B964FAD6B976C965FADAB
:106BF0006C976D966FAD6D976E967FAD6E976F9635
:106C00008FAD6F97A0969FADA0970E9459E02BED96
:106C10003FE049E450E40E94A5DC20E030E040E0A1
:106C20005FE30E94A5DC9B01AC01C701B6010E9495
:106C3000DDE06B017C01C301B2010E9446DC2FE65E
:106C400032E143E85AE30E94A5DC2B013C01B70185
:106C5000A6018DE197E00E9475C9B301A20187E109
:106C600097E00E9475C92AE939E949E15FE3C70164
:106C7000B6010E94A5DC6B017C019B01AC010E9466
:106C80005AE0A30192010E94DDE0A4966CAF7DAFB3
:106C90008EAF9FAFA497A3019201C701B6010E94D6
:106CA000A5DC20E030E040E05EE30E94A5DCA89691
:106CB0006CAF7DAF8EAF9FAFA897E7E0F7E0849110
:106CC0003F015FEF651A750A882321F00E94553C49
:106CD000F301F5CFB701A60181E097E00E9475C9E5
:106CE000A4964CAD5DAD6EAD7FADA4978BEF96E0F5
:106CF0000E9475C9A8964CAD5DAD6EAD7FADA897ED
:106D000085EF96E00E9475C98AE00E94553C2F9657
:106D10008CAD9DADAEADBFAD2F97880D991DAA1D51
:106D2000BB1DB595A795979587958093330E68966B
:106D30008EAD9FAD6897019668969FAF8EAF6897AE
:106D400060969FAD609769969FAF69976196AFAD6A
:106D500061976A96AFAF6A976596BFAD65976B9678
:106D6000BFAF6B976696EFAD66976C96EFAF6C977B
:106D70002B964CAC5DAC6EAC7FAC2B97F1E0AB9638
:106D8000FFAFAB970C945D2DCE57DF4F0FB6F89445
:106D9000DEBF0FBECDBFDF91CF911F910F91FF904E
:106DA000EF90DF90CF90BF90AF909F908F907F90AB
:106DB0006F905F904F903F902F9008959091500E5C
:106DC000E92FF0E0E758F74F80839F5F943018F485
:106DD0009093500E02C01092500E80911B0A8F5F4C
:106DE00080931B0A08958FB7F8949091FB0A209125
:106DF000FA0A291759F0E92FF0E0E658F54F2081FB
:106E000030E09F5F9F779093FB0A02C02FEF3FEF28
:106E10008FBFC90108950F931F93CF93DF93EC01A8
:106E20000E94F3520E811F812885398501151105B5
:106E30002105310559F52C852223A9F13A852150E8
:106E40002C8721E0230F2A874D85241301C01A8641
:106E5000FE0124E0329FE00DF11D11240685178507
:106E6000208931890A831B832C833D83DC01CB017C
:106E7000800F911FA11DB11D8E839F83A887B987A5
:106E80008C819D81892B79F0419A0DC0DC01CB0169
:106E9000801B910BA20BB30BB7FD05C041981E825E
:106EA0001F8218861986DF91CF911F910F91089547
:106EB000EF920F931F93E090360E00E011E02FE069
:106EC0003EE04BE05EE067E07EE083E09EE00E9413
:106ED0002BCB1F910F91EF900895CF92DF92EF92FD
:106EE000FF92CF9381E080933701C1E08091370119
:106EF000882309F444C0CC2309F441C080E00E94F7
:106F00002A7B6091E30D7091E40DC0E0611571057D
:106F100069F3072E000C880B990B0E9446DC9B013D
:106F2000AC016091560E7091570E8091580E909161
:106F3000590E0E9459E06B017C0120E030E0A9016C
:106F40000E94DDE118165CF020E030E040EA50ECF1
:106F5000C701B6010E943FDC87FFC8CF0BC020E00D
:106F600030E040EA50E4C701B6010E94DDE11816A6
:106F70000CF0BCCF89E090E00E94705FB6CFCF915B
:106F8000FF90EF90DF90CF900895CF92DF92EF9235
:106F9000FF920F931F93CF93DF9300D000D0CDB714
:106FA000DEB7182F662351F01092F4021092F0020F
:106FB0001092F1021092F2021092F3020E94F35228
:106FC000C090F002D090F102E090F202F090F30253
:106FD0009B01AC012C193D094E095F0957FD3EC0CC
:106FE00017FD16C04091F402212F012E000C330B27
:106FF0002C5F3F4FE42F042E000CFF0B2E173F0792
:107000006CF141172CF000E911E020E030E004C001
:1070100004EC19E020E030E0DC01CB01800F911F8F
:10702000A21FB31F8093F0029093F102A093F2028B
:10703000B093F30280ED97E09C838B838CE291E028
:107040009A838983BE016D5F7F4FCE0101960E94B6
:10705000A99C8091F4028F5F8093F4020F900F90AF
:107060000F900F90DF91CF911F910F91FF90EF90B4
:10707000DF90CF9008952F923F924F925F926F9240
:107080007F928F929F92AF92BF92CF92DF92EF92B8
:10709000FF920F931F93CF93DF9300D000D0CDB713
:1070A000DEB71C017A8369835C834B8389018090FE
:1070B000000190900101A0900201B0900301F9013C
:1070C000C080D180E280F38020E030E0A901C701D8
:1070D000B6010E943FDC811106C0E1EAFAE1C590E9
:1070E000D590E590F490EB81FC8120813181428143
:1070F000538160910B0E70910C0E80910D0E90914A
:107100000E0E0E943FDC87FF18C0C0920001D09293
:107110000101E0920201F0920301EB81FC81808188
:107120009181A281B38180930B0E90930C0EA0935A
:107130000D0EB0930E0E0E945837F801408051801A
:107140006280738020E030E0A901C301B2010E9497
:107150003FDC811107C085E5482E542C85E0682E60
:1071600083E4782E40920001509201016092020166
:1071700070920301F10180819181A281B38180939A
:10718000030E9093040EA093050EB093060EE981B2
:10719000FA8180819181A281B3818093070E9093BF
:1071A000080EA093090EB0930A0E0E945837EB8187
:1071B000FC81208131814281538160910B0E70915D
:1071C0000C0E80910D0E90910E0E0E94DDE11816AE
:1071D000C4F4C0920001D0920101E0920201F09249
:1071E0000301EB81FC8180819181A281B381809335
:1071F0000B0E90930C0EA0930D0EB0930E0E0E94EA
:1072000058370E9420488092000190920101A0927C
:107210000201B09203010F900F900F900F90DF9139
:10722000CF911F910F91FF90EF90DF90CF90BF9083
:10723000AF909F908F907F906F905F904F903F9016
:107240002F9008959B01AC0167E07EE083E09EE013
:107250000C943B38EF920F931F93CF93DF9300D0A2
:1072600000D0CDB7DEB769837A838B839C83E090AF
:10727000360E8E010F5F1F4F23E23BE04FE15BE0D4
:107280006BE17BE087E19BE00E942BCB0F900F909E
:107290000F900F90DF91CF911F910F91EF90089574
:1072A0000F931F93CF93DF93EC01CC0FDD1FCC0F17
:1072B000DD1F8E010157124FFE01E359F74FDE012A
:1072C000A55FB44F2D913D914D915C91608171818D
:1072D000828193810E945AE0F801608371838283E6
:1072E0009383FE01EC5FF64F85919591A591B49142
:1072F000FE01E45EF54F80839183A283B383FE0198
:10730000E05FF64F85919591A591B491CE5EDE4FE9
:1073100088839983AA83BB83DF91CF911F910F91BB
:107320000895CF93FC0180818B33A9F080911B0AD3
:10733000843088F4C62FBF018091500E20E6829FD2
:10734000C00111248656974F0E940FE38C2F0E9494
:10735000DE3681E001C080E0CF910895DF92EF92A8
:10736000FF920F931F93CF93DF93CDB7DEB76E9746
:107370000FB6F894DEBF0FBECDBF60914E0D709179
:107380004F0D6115710509F14DE150E0CE010196F7
:107390007C010E94ADDB1E8EF7018F010E191F09C3
:1073A000D190DD2019F09AE0D912F7CFF701E00F64
:1073B000F11F108260E0C7010E949139882329F0F3
:1073C000C7010E946E7A811109C081E020914E0DA3
:1073D00030914F0D232BA1F480E012C0DD2049F045
:1073E0000F5F1F4F80914E0D90914F0D080F191F89
:1073F00002C000E010E010934F0D00934E0DE5CF5A
:107400006E960FB6F894DEBF0FBECDBFDF91CF9161
:107410001F910F91FF90EF90DF9008952FE03EE0D5
:107420004BE05EE067E07EE083E09EE00C943CCAC7
:107430008F929F92BF92CF92DF92EF92FF920F9323
:107440001F93CF93DF93CDB7DEB728970FB6F8948D
:10745000DEBF0FBECDBFB02EC12ED22EF32E8C01BB
:10746000000F111F000F111FC8018D5F914F4C01BC
:10747000FC0110821182128213824D835E836F831E
:1074800078870E940E3A4D815E816F817885F40184
:107490004083518362837383E090360E20E030E0B6
:1074A000A9016B2D7C2D8D2D9F2D0E943FDC81111C
:1074B00008C0F801E756F54E85919591A591B491D4
:1074C00004C08B2D9C2DAD2DBF2D89839A83AB835A
:1074D000BC838E010F5F1F4F2FE03EE04BE05EE06C
:1074E00067E07EE083E09EE00E942BCB0E94204874
:1074F0001092990828960FB6F894DEBF0FBECDBF44
:10750000DF91CF911F910F91FF90EF90DF90CF907F
:10751000BF909F908F9008958091810290918202F8
:10752000009731F04AE050E060E070E00C9454DAEB
:1075300060E070E0CB010895809181029091820219
:10754000009731F04AE050E060E070E00C9429D9F7
:1075500060E070E0CB0108950E949C3A97FD0CC05A
:107560000E949C3A6F3F71058105910509F034F442
:107570000E949C3A862F089580E008958FEF089529
:107580008091810290918202892B39F00E94AC3A5D
:1075900091E0811103C090E001C091E0892F08952E
:1075A0000F931F93CF938091810290918202009755
:1075B000F1F0FC018F01C1912C2F2F7D89F0C53492
:1075C00011F0C536B9F7F801108260E070E00E9452
:1075D000BAD7F801C083562F472F382F292F0BC059
:1075E00060E070E0CF911F910F910C94BAD750E0FA
:1075F00040E030E020E0652F742F832F922FCF9151
:107600001F910F91089581548A3150F5482F50E011
:10761000FA0193E0F595E7959A95E1F7E254FC4E6F
:10762000208130E08770B90102C0759567958A9511
:10763000E2F760FF15C0FA01EC55FC4E20812223D1
:1076400039F08091010B9091020B820F911D02C0C5
:1076500080E090E0909382028093810281E008951F
:1076600080E008950E94033B882341F081E020914F
:10767000810230918202232B09F480E00895CF9299
:10768000DF92EF92FF921F93CF93DF9380E50E94EA
:10769000033B882309F447C00E949C3A6B017C019C
:1076A00083E50E94323B882321F00E949C3AEB0143
:1076B00002C0CFEFDFEFCE0101960397A0F5D7FC14
:1076C00032C09C2DE2E8F2E088E28E0F24919217FE
:1076D00051F131968E13FACF0E9420481C2D60E0A4
:1076E0008C2D0E948760CF3F8FEFD80759F48C2DE7
:1076F0000E942E6031E020E0892B09F030E0C32F9A
:10770000D22F04C0219761F0C0E0D0E0812F0E9409
:107710002E608C179D0739F080E00E942A7BF6CFFF
:10772000C1E0D0E0F3CFDF91CF911F91FF90EF90B8
:10773000DF90CF900895FC01238121110C94F0A5D6
:1077400008952091C30E9091C40E81E0291301C0C9
:1077500080E0089588E893E19093D5078093D4075B
:1077600080916F008D7F80936F000E94A13B8823E2
:1077700059F00E94A13B8823C1F38091C40E8F5F12
:107780008F708093C40EF1CF1092D3071092D2075E
:1077900080916F00826080936F008FB7F894109291
:1077A00045081092460810924708109248088FBF6B
:1077B0000E94204880E090E00E9402486093F50219
:1077C0007093F6028093F7029093F80281E090E0C4
:1077D0000E9402486093F9027093FA028093FB02C0
:1077E0009093FC0282E090E00E9402486093FD02C8
:1077F0007093FE028093FF02909300038CE0E5EF0C
:10780000F2E0A3E0BEE001900D928A95E1F70C94BE
:107810000E3A80E1E3E0FEE0A7E1BBE001900D92CB
:107820008A95E1F70895CF92DF92EF92FF92CF937E
:10783000DF936A017B01C3E0DEE0E091360E24E0D5
:10784000E29FF0011124E85CFE4F208131814281EA
:107850005381FC0160817181828193810E94DDE00E
:107860009B01AC016C857D858E859F850E945AE0C9
:107870006C877D878E879F870E94093CC701B60170
:107880000E942A39DF91CF91FF90EF90DF90CF9047
:107890000C9420480E94F3526093030B7093040BE6
:1078A0008093050B9093060B08959091C00095FF6F
:1078B000FCCF8093C6000895CF93DF9385E40E94A8
:1078C000323B811110C080E50E94033B882391F078
:1078D0000E94D03A6093330A7093340A8093350A39
:1078E0009093360A07C00E94AC3A882361F3E8E31C
:1078F000FCE16DC089E40E94033B882381F00E9473
:10790000D03A2CEA35EC47E25EE30E94A5DC6093B6
:107910003B0A70933C0A80933D0A90933E0A84E4AC
:107920000E94033B882381F00E94D03A2CEA35EC78
:1079300047E25EE30E94DDE06093370A7093380A05
:107940008093390A90933A0AE3E5FCE18491EF01D0
:107950002196882321F00E94553CFE01F7CF4091EB
:10796000330A5091340A6091350A7091360A84E8DE
:1079700099E00E9475C92CEA35EC47E25EE360911C
:107980003B0A70913C0A80913D0A90913E0A0E9408
:10799000DDE0AB01BC0180E899E00E9458C92CEA07
:1079A00035EC47E25EE36091370A7091380A8091C6
:1079B000390A90913A0A0E94A5DCAB01BC018CE720
:1079C00099E00E9458C910C00E94553CFE01849164
:1079D000EF0121968111F8CFC7E2D2E08991882387
:1079E00019F00E94553CFACF8AE0DF91CF910C94B8
:1079F000553CCF93DF93E3E5FCE18491EF012196C1
:107A0000882321F00E94553CFE01F7CF83E50E94B8
:107A1000033B882321F00E94C03A80931E01ECE6CC
:107A2000F9E08491EF012196882321F00E94553CD2
:107A3000FE01F7CF80911E01811103C0E8E6F9E055
:107A400002C0E4E6F9E08491EF012196882321F059
:107A50000E94553CFE01F7CFECE5F9E08491EF017F
:107A60002196882321F00E94553CFE01F7CF2091FA
:107A70008F0D3091900D4091910D5091920D60912C
:107A80001C0A70911D0A80911E0A90911F0A0E9483
:107A90005AE0AB01BC018AE599E00E9475C92091CA
:107AA000930D3091940D4091950D5091960D6091EC
:107AB000200A7091210A8091220A9091230A0E9443
:107AC0005AE0AB01BC0187E599E00E9475C920919D
:107AD000970D3091980D4091990D50919A0D6091AC
:107AE000240A7091250A8091260A9091270A0E9403
:107AF0005AE0AB01BC0184E599E00E9475C9ECE451
:107B0000F9E08491EF012196882321F00E94553CF1
:107B1000FE01F7CF20918F0D3091900D4091910D86
:107B20005091920D60911201709113018091140196
:107B3000909115010E945AE0AB01BC018AE499E0E2
:107B40000E9475C92091930D3091940D4091950D2F
:107B50005091960D60911601709117018091180156
:107B6000909119010E945AE0AB01BC0187E499E0B1
:107B70000E9475C92091970D3091980D4091990DF3
:107B800050919A0D60911A0170911B0180911C0116
:107B900090911D010E945AE0AB01BC0184E499E080
:107BA0000E9475C98AE0DF91CF910C94553C4F92A9
:107BB0005F926F927F929F92AF92BF92CF92DF922D
:107BC000EF92FF920F931F93CF93DF931F92CDB746
:107BD000DEB70E94AE39811176C280911B0A8430D3
:107BE00028F40E94F336AC0197FF4BC18091F50E4B
:107BF000882309F468C280911B0A811102C0109287
:107C0000E902EE24E3944091711150917211609158
:107C100073117091741180916D1190916E11A091FA
:107C20006F11B0917011481759076A077B0708F464
:107C3000E12C00E010E0BB24B39480E6A82E9AEC7F
:107C4000C92E98E0D92E2DE8922E80911B0A8430FF
:107C500008F039C2E11037C28091E902811133C2C4
:107C60008091C8109091C910A091CA10B091CB100A
:107C70008093711190937211A0937311B09374114A
:107C800041E050E0BE016F5F7F4F80EC90E10E94C9
:107C900029A4019719F4898190E002C08FEF9FEF2A
:107CA000F82EEE24E3944090711150907211609080
:107CB00073117090741140916D1150916E1160911B
:107CC0006F11709170114416550666067706C8F458
:107CD000E12C8F3FFFEF9F0709F480C02AE0821755
:107CE00009F4A1C08DE0F81609F49DC093E2F916DD
:107CF00019F0EAE3FE12ABC08091E8028111A7C03F
:107D000087C00E94204880EC90E10E94F0A58091FD
:107D1000DB10882359F181508093DB10989EC001BD
:107D2000112441E061E080529F4E0E942882E09140
:107D3000DB1024E0E29FF0011124E452FF4E408169
:107D400051816281738140937111509372116093DC
:107D500073117093741180EC90E10E941DC28091A8
:107D6000F60E8823D1F0B092F50E17C01092F50EE2
:107D700081E090E09093D5078093D4070E94A7BB41
:107D80000E949EBD6D3371058105910530F0D09242
:107D90004F0DC0924E0D0E94AE398091F50E8111AB
:107DA0003BC0EDEDF8E084913F019FEF691A790A3D
:107DB000882321F00E94553CF301F5CF10927911F0
:107DC0008091F60E882319F00E94C08421C00E9481
:107DD000CB9B8091F60E8111F7CF1AC0E8E3FCE14E
:107DE00084913F012FEF621A720A882321F00E94CA
:107DF000553CF301F5CFEEECF8E084913F019FEFA5
:107E0000691A790A882321F00E94553CF301F5CFC5
:107E1000E3E2FE1208C005C023E2F2124FC100E007
:107E200010E0B092E9021092E8020115110509F480
:107E30000CCF8091500EA89E000D111D1124F80149
:107E4000E656F74F108280E00E94DE3639C10F35CA
:107E5000110508F0FACEFBE3FF1202C0B092E8026F
:107E60008091E8028111F1CE8091500EF801A89E18
:107E7000E00DF11D1124E656F74FF0820F5F1F4F02
:107E8000E4CE982F2091270E3091280E8A3019F0D9
:107E90009D3009F0E1C01092E7022115310509F487
:107EA0009CCEF901E957FD4F10821092280E1092D6
:107EB000270E27E832E08901F90180812F5F3F4FCB
:107EC0008032C9F378018E3409F07BC001151105A9
:107ED00009F477C065EC78E0C8010E94BCDBDD24C2
:107EE000D394892B11F4D12C09C06EE470E0C80141
:107EF00004960E94FBE2009709F08C014AE050E0F2
:107F000060E070E0C80101960E9429D96093830265
:107F10007093840280938502909386020091290ECB
:107F200010912A0E20912B0E30912C0E0F5F1F4FB7
:107F30002F4F3F4F601771078207930729F0D11029
:107F400003C08FEB97E027C06AE270E0C7010E9490
:107F500033E39C01009711F1982F9E1910E09923AB
:107F600039F09150F701E90FF11D80811827F7CF03
:107F70004AE050E060E070E0C90101960E9429D912
:107F8000012F10E020E030E06017710782079307AF
:107F900041F086EA98E00E946A9C28CE8CE798E03F
:107FA000FACF8091830290918402A0918502B091D2
:107FB00086028093290E90932A0EA0932B0EB093E5
:107FC0002C0E80910901811122C067E470E0C70185
:107FD0000E94FBE20097D9F04AE050E060E070E0D8
:107FE00001960E9429D96430710588F4E5E0F8E033
:107FF00084918F010F5F1F4F882321F00E94553C11
:10800000F801F6CF60E08BEF97E00E94DEC868E3EE
:1080100072E0C7010E9406E3892B21F41092370118
:10802000109251086DE372E0C7010E9406E3892BAC
:1080300021F482EF97E00E94C17A62E472E0C70106
:108040000E9406E3892B11F40E94AA3B61E087E8B5
:1080500092E00E949139C1CD2F3531050CF0BDCD94
:108060009C35C1F40E94F33697FDB7CD2091E7020D
:108070002111B3CD2091270E3091280EA9014F5F19
:108080005F4F5093280E4093270EF901E957FD4F9B
:108090008083A3CD9B3319F481E08093E702809124
:1080A000E70281119ACDC90101969093280E809321
:1080B000270EF901E957FD4F40838FCD1092E8025A
:1080C00000E010E0C2CD0F90DF91CF911F910F9192
:1080D000FF90EF90DF90CF90BF90AF909F907F90F8
:1080E0006F905F904F9008958F929F92AF92BF9242
:1080F000EF92FF921F93CF93DF93CDB7DEB7A09798
:108100000FB6F894DEBF0FBECDBF611571058105B6
:10811000910581F110E0842E912CA12CB12CEE243C
:10812000E394F12CEC0EFD1EE10EF11C17FDFA9408
:10813000A50194010E941DE0F7016083B901CA0105
:108140001F5F611571058105910549F7115020F1F7
:10815000E1E0F0E0EC0FFD1FE10FF11D17FDFA95D6
:1081600080818A3010F097E301C090E3890F0E946C
:10817000553CECCF80E3A0960FB6F894DEBF0FBE5F
:10818000CDBFDF91CF911F91FF90EF90BF90AF9047
:108190009F908F900C94553CA0960FB6F894DEBF3C
:1081A0000FBECDBFDF91CF911F91FF90EF90BF9099
:1081B000AF909F908F900895EF92FF920F931F932F
:1081C000CF93DF937C0184E50E94323BD82F882334
:1081D00049F10E94AC3AC82F181604F5E3E5FCE11A
:1081E00084918F010F5F1F4F882321F00E94553C1F
:1081F000F801F6CF8DE40E94553CB70180E090E095
:108200004AE00E9474406C2FCC0F770B81EF98E00E
:108210000E9492C98AE00E94553C08C08093350EA6
:10822000D0E004C08091360E8093350E8D2FDF9103
:10823000CF911F910F91FF90EF900895CF92DF9211
:10824000EF92FF926B017C0197FF0BC08DE20E94C1
:10825000553CF094E094D094C094C11CD11CE11C16
:10826000F11C4AE0C701B601FF90EF90DF90CF907C
:108270000C947440EF92FF920F931F93CF93DF9370
:108280001F92CDB7DEB7082F162FEFE3F9E08491E8
:108290007F012FEFE21AF20A882331F099830E94BE
:1082A000553CF7019981F3CFE02FF92F84917F019D
:1082B0009FEFE91AF90A882321F00E94553CF70143
:1082C000F5CFEDE3F9E084917F012FEFE21AF20A96
:1082D000882321F00E94553CF701F5CF612F70E013
:1082E00080E090E00E941E418AE00F90DF91CF91E4
:1082F0001F910F91FF90EF900C94553C8F929F929D
:10830000AF92BF92CF92DF92EF92FF92CF936B0129
:108310007C01B42E20E030E0A9010E943FDC87FF01
:1083200007C08DE20E94553CF7FAF094F7F8F094FC
:10833000C0E060E070E080E09FE3CB1541F02DEC01
:108340003CEC4CEC5DE30E94A5DCCF5FF6CF9B01DB
:10835000AC01C701B6010E945AE06B017C010E948A
:1083600056E14B015C014AE00E947440CC2389F144
:10837000C501B4010E9444DC9B01AC01C701B601F8
:108380000E9459E06B017C018EE20E94553C20E086
:1083900030E040E251E4C701B6010E94A5DC4B0188
:1083A0005C010E944FE16B01770FEE08FF08C701E7
:1083B000B6010E941E41C701B6010E9446DC9B0126
:1083C000AC01C501B4010E9459E06B017C01C150B0
:1083D000F1F6CF91FF90EF90DF90CF90BF90AF90EC
:1083E0009F908F9008954F925F926F927F928F929D
:1083F0009F92AF92BF92CF92DF92EF92FF92CF9374
:10840000DF93EAE3F9E08491EF012196882321F0DC
:108410000E94553CFE01F7CF20918F0D3091900DB9
:108420004091910D5091920D6091030E7091040E48
:108430008091050E9091060E0E945AE042E00E9443
:108440007E41E6E3F9E08491EF012196882321F053
:108450000E94553CFE01F7CF2091930D3091940D71
:108460004091950D5091960D6091070E7091080EF8
:108470008091090E90910A0E0E945AE042E00E94FB
:108480007E41E2E3F9E08491EF012196882321F017
:108490000E94553CFE01F7CF2091970D3091980D29
:1084A0004091990D50919A0D60910B0E70910C0EA8
:1084B00080910D0E90910E0E0E945AE042E00E94B3
:1084C0007E41EEE2F9E08491EF012196882321F0CC
:1084D0000E94553CFE01F7CF60910F0E7091100E77
:1084E0008091110E9091120E42E00E947E418FB752
:1084F000F8944090F30D5090F40D6090F50D70904D
:10850000F60D8090F70D9090F80DA090F90DB090B9
:10851000FA0DC090FB0DD090FC0DE090FD0DF09099
:10852000FE0D8FBFE4E2F9E08491EF0121968823EC
:1085300021F00E94553CFE01F7CFC301B2010E9419
:108540001E41E0E2F9E08491EF012196882321F0B9
:108550000E94553CFE01F7CFC501B4010E941E41A7
:10856000ECE1F9E08491EF012196882321F00E944B
:10857000553CFE01F7CFC701B6010E941E418AE0BB
:10858000DF91CF91FF90EF90DF90CF90BF90AF90B1
:108590009F908F907F906F905F904F900C94553C80
:1085A000EF92FF920F931F93CF93DF9300D000D0F1
:1085B0001F92CDB7DEB78D830E9420484091000105
:1085C0005091010160910201709103014093EC020E
:1085D0005093ED026093EE027093EF022091400100
:1085E000309141013093EB022093EA0224E630E01F
:1085F00030934101209340010E944A3C91E09093C6
:10860000C60E8D81811119C088E50E94033BF82EAA
:1086100089E50E94033B082F8AE50E94033BE82E70
:10862000F11006C0011113C0882369F0F02E0FC0AD
:10863000002369F0F02E182F0BC0FF24F39401E003
:10864000EE24E39402C0F82E082F11E001C010E0E0
:108650000E94093C111104C0F11002C00023C1F1B5
:1086600080E090E0A0EAB0E480931F0B9093200B91
:10867000A093210BB093220B9C01AD0160910B0ED6
:1086800070910C0E80910D0E90910E0E0E943FDCA9
:1086900087FF0BC019821A821B821C82BE016F5F8A
:1086A0007F4F8FE19BE00E942239111105C0F1102C
:1086B00003C0011107C00CC080E090E00E949479D3
:1086C0001123B9F381E090E00E949479111102C066
:1086D000EE2021F082E090E00E9494790E940E3A10
:1086E0008091C50E8093C60E8091EC029091ED02B0
:1086F000A091EE02B091EF028093000190930101EE
:10870000A0930201B09303018091EA029091EB02E1
:1087100090934101809340010E944A3C83E0809302
:1087200032010E94F3410F900F900F900F900F9025
:10873000DF91CF911F910F91FF90EF9008951F92BD
:108740000F920FB60F9211240BB60F922F938F93A7
:108750009F93EF93FF93E091FA0A81E08E0F8F775A
:108760009091C6002091FB0A821731F0F0E0E658A4
:10877000F54F90838093FA0AFF91EF919F918F912B
:108780002F910F900BBE0F900FBE0F901F9018955A
:108790002F923F924F925F926F927F928F929F9211
:1087A000AF92BF92CF92DF92EF92FF92CF93DF937F
:1087B00000D000D0CDB7DEB76090E30D7090E40D2F
:1087C0008090560E9090570EA090580EB090590E73
:1087D000B301072C000C880B990B0E9446DCA50105
:1087E00094010E9459E06B017C016093160870931C
:1087F0001708809318089093190820ED3CEC4CE47E
:108800005DE36091370A7091380A8091390A90913E
:108810003A0A0E94A5DC1B012C012091120830911C
:1088200013084091140850911508C501B4010E9425
:1088300059E09B01AC01C201B1010E94A5DC1B0102
:108840002C0123E333E343E75FE360910E0870916B
:108850000F0880911008909111080E94A5DC9B01DF
:10886000AC01C201B1010E945AE069837A838B8313
:108870009C8360930E0870930F0880931008909368
:1088800011088092120890921308A0921408B092D6
:10889000150880915E0E882321F081E080930D08F9
:1088A000B9C020E030E040E251E4C701B6010E94C7
:1088B000DDE1181624F481E080930D08A4C020E0C7
:1088C00030E040E251ECC701B6010E943FDC87FD79
:1088D000E4CF672811F380910D08882351F010929E
:1088E000090810920A0810920B0810920C081092B6
:1088F0000D082091330A3091340A4091350A509185
:10890000360AC701B6010E94A5DC2B013C01609329
:108910000508709306088093070890930808209133
:10892000090830910A0840910B0850910C08C701C2
:10893000B6010E945AE04B015C01609309087093F4
:108940000A0880930B0890930C0820913B0A309101
:108950003C0A40913D0A50913E0A0E94A5DC9B01D1
:10896000AC01609301087093020880930308909310
:108970000408C301B2010E945AE029813A814B8167
:108980005C810E9459E02B013C0120E030E04FE780
:1089900053E40E94DDE120E030E0A9011816ACF4B8
:1089A000C701B6010E94DDE118166CF5A70196011A
:1089B000C501B4010E9459E06093090870930A0848
:1089C00080930B0890930C081EC0C301B2010E9453
:1089D0003FDC87FF22C020E030E0A901C701B601DB
:1089E0000E943FDC87FF16C0A7019601C501B401B4
:1089F0000E9459E06093090870930A0880930B085D
:108A000090930C0807C0412C512C8FE7682E83E40B
:108A1000782E03C0412C512C3201C301B2010F90BA
:108A20000F900F900F90DF91CF91FF90EF90DF901C
:108A3000CF90BF90AF909F908F907F906F905F90FE
:108A40004F903F902F900895CF92DF92EF92FF9238
:108A5000C090560ED090570EE090580EF090590EE0
:108A60008091E30D9091E40D0897BC01990F880B5C
:108A7000990B0E9446DC9B01AC01C701B6010E9424
:108A80003FDC87FF1FC020E030E040E050E4C7013A
:108A9000B6010E945AE00E9456E170932908609343
:108AA00028080E94F352DC01CB01805E914BAF4F4E
:108AB000BF4F8093240890932508A0932608B09375
:108AC000270808C010922408109225081092260842
:108AD00010922708FF90EF90DF90CF9008951092AA
:108AE0003F0A1092E40D1092E30D80E00E942445AD
:108AF0001092E80D1092E70D0E94A7BB1092E40DB2
:108B00001092E30D80E00E9424451092330E5D9890
:108B10001092E80D1092E70D1092340E5C980895B3
:108B20002F923F924F925F926F927F928F929F927D
:108B3000AF92BF92CF92DF92EF92FF920F931F936B
:108B4000CF93DF93EC0143E35FE281E090E0FA0131
:108B500025913491C217D3070CF05DC09C012150C0
:108B60003109220F331F220F331FD901AF5CB04DE3
:108B7000FD0165917491215D304DF901A590B4908E
:108B8000FC01EE0FFF1FEE0FFF1FEF5CF04DE590B5
:108B9000F490FD01C590D490FA0105911491F9016A
:108BA00025903490072E000C880B990B0E9446DC10
:108BB0002B013C01CA19DB09BE01DD0F880B990BA3
:108BC0000E9446DC4B015C01B7016C197D09072E40
:108BD000000C880B990B0E9446DC9B01AC01C5017F
:108BE000B4010E94A5DC6B017C01B8016219730914
:108BF000072E000C880B990B0E9446DC9B01AC01F0
:108C0000C701B6010E94DDE09B01AC01C301B201C6
:108C10000E945AE011C001964C5F5F4F803491056D
:108C200009F095CFEDE2F0E365917491072E000C09
:108C3000880B990B0E9446DCDF91CF911F910F9119
:108C4000FF90EF90DF90CF90BF90AF909F908F906C
:108C50007F906F905F904F903F902F90089560E0CD
:108C600080912F0E9091300E0E9489A16093560E34
:108C70007093570E8093580E9093590E80912D0E3D
:108C800090912E0E0E94904560938B0D70938C0DE9
:108C900080938D0D90938E0DA8958FB7F8941092B8
:108CA000310E8FBF0895CF92DF92FF920F931F93E3
:108CB000CF93DF9300D0CDB7DEB7F82E8A01809135
:108CC0000901882309F444C0E8E3FCE184916F01C1
:108CD0009FEFC91AD90A882341F069837A830E94D9
:108CE000553CF60169817A81F1CFFB0184916F01D6
:108CF0009FEFC91AD90A882321F00E94553CF6013A
:108D0000F5CFE9E9F1E184916F019FEFC91AD90A22
:108D1000882321F00E94553CF601F5CFF7FC0BC0EB
:108D20006F2DFF0C770B880B990B0E941E418AE078
:108D30000E94553C0DC0E4E9F1E184916F019FEF81
:108D4000C91AD90A882321F00E94553CF601F5CFB3
:108D500080910008811108C01092090181E0809380
:108D60000008C8010E94C17A0F900F90DF91CF9147
:108D70001F910F91FF90DF90CF900C946F458F92D1
:108D80009F92AF92BF92CF92DF92EF92FF920F939A
:108D90001F938091310E81110BC01F910F91FF9095
:108DA000EF90DF90CF90BF90AF909F908F900895FD
:108DB0000E942F460E94F3524B015C0180915E0E8F
:108DC000811117C08091D6079091D707A091D8073D
:108DD000B091D9070097A105B10559F0A5019401FB
:108DE000281B390B4A0B5B0B57FD03C081E08093B6
:108DF0005E0E6091E30D7091E40D072E000C880B60
:108E0000990B0E9446DC2091560E3091570E4091EE
:108E1000580E5091590EC12C7B018C0160E278E014
:108E20008EE198E00E9497BCC090560ED090570EED
:108E3000E090580EF090590E809168089091690862
:108E4000BC01990F880B990B0E9446DC9B01AC0179
:108E5000C701B6010E94DDE11816D4F4609110013B
:108E600070911101072E000C880B990B0E9446DCB3
:108E70009B01AC01C701B6010E943FDC87FF08C01F
:108E800080E00E94C8430E944FE17595679501C03C
:108E900060E06093330E8091240890912508A091A2
:108EA0002608B09127080097A105B10501F1A50199
:108EB0009401281B390B4A0B5B0B57FD18C00E940D
:108EC00028A26B017C018091280890912908BC019F
:108ED00080E090E00E9444DC9B01AC01C701B60138
:108EE0000E943FDC87FD5BC080E00E9424458091AA
:108EF0001A0890911B08A0911C08B0911D08A501AB
:108F00009401281B390B4A0B5B0B57FD46CF38E801
:108F1000830E33E1931EA11CB11C80921A0890921B
:108F20001B08A0921C08B0921D0880915D0E811153
:108F300032C0C0908B0DD0908C0DE0908D0DF090D4
:108F40008E0D20E030E040EA50E4C701B6010E94F7
:108F5000DDE187FD20C020E030E046EE52E4C701AD
:108F6000B6010E943FDC1816B4F06091E70D7091D5
:108F7000E80D072E000C880B990B0E9446DC9B0124
:108F8000AC01C701B6010E943FDC87FD10C080E044
:108F90008093340E02CF1092340E5C98FECE47EBD5
:108FA00051E166EC71E180E00E945346A0CF8FE76B
:108FB000EFCF880F991F880F991FFC01ED50F24FDA
:108FC0004081518162817381FC01E357F74F4083F7
:108FD000518362837383E091D207F091D307828932
:108FE0009389A489B5898093FC079093FD07A0938A
:108FF000FE07B093FF078FEF9FEF9093D507809305
:10900000D4070895CF93DF932FB7F894EC01CC0FDA
:10901000DD1FCC0FDD1FFE01ED50F24F608171812D
:10902000828193812FBF0E9446DCC358D74F28818D
:1090300039814A815B810E94A5DCDF91CF9108953F
:109040000E94A13B882321F080E00E942A7BF8CF78
:109050008091D4079091D507892BB1F708951F927D
:109060000F920FB60F9211240BB60F92BF92CF92B0
:10907000DF92EF92FF920F931F932F933F934F93A3
:109080005F936F937F938F939F93AF93BF93EF9370
:10909000FF93CF93DF9300D000D0CDB7DEB78091A0
:1090A0006E008B7F80936E0080916F008D7F809328
:1090B0006F007894C090F807D090F907E090FA0715
:1090C000F090FB07C114D104E104F104B1F18091E7
:1090D000C60E882391F10E94BD91D701C60109EB0C
:1090E000C0160BE0D006E104F10420F088EB9BE011
:1090F000A0E0B0E0C81AD90AEA0AFB0AC092F80751
:10910000D092F907E092FA07F092FB07909389005A
:10911000809388002091880030918900809184009C
:109120009091850040962817390708F036C680913F
:109130008400909185004096FFC10091D407109162
:10914000D5070115110509F444C017FF21C080910E
:10915000D2079091D307892B51F00E94A13B88231D
:1091600031F08091C40E8F5F8F708093C40E0E9487
:10917000A13B882309F450C6E091C40E1DE4E19F91
:10918000F0011124EE5FFC4F808184FD39C644C696
:109190000E94A13B882331F08091C40E8F5F8F70B5
:1091A0008093C40E015011091093D5070093D40782
:1091B000012B41F488E891E190934F0D80934E0D7F
:1091C0000E94AE391092D3071092D20788EC90E03B
:1091D000B3C1C090D207D090D307C114D10409F015
:1091E000B0C10E94A13B882349F19091C40E4DE487
:1091F000949F900111242E5F3C4F809145089091DF
:109200004608A0914708B0914808F901E75BFF4F75
:109210004081518162817381841B950BA60BB70B32
:109220008093450890934608A0934708B093480858
:10923000D9018C9188608C9369010BC08FB7F89429
:10924000109245081092460810924708109248085C
:109250008FBFD092D307C092D207C114D10409F4B2
:1092600069C1F60152A180910103418158130AC0DE
:10927000242F30E080910801082E000C990B28174C
:10928000390731F050930103409308010E940EC941
:109290001092F4071092F5071092F6071092F70754
:1092A000D601D7968D919C91D8978134BCE99B07C4
:1092B00028F48132EEE49E0748F002C080E49CE985
:1092C000969587959695879524E007C08131F7E2BA
:1092D0009F0730F09695879522E02093F30708C00A
:1092E00021E02093F3078032910510F480E290E0B2
:1092F0008C0100521109011528E01207D8F0E12F66
:10930000FF27EE0FFF1FEE0FFF1FCF018857924F71
:10931000FC01329645915491AA27059F9001049F24
:10932000210D3A1F06942A1F3A1F1124FC01859132
:1093300094911CC09801369527952C7F2857364F5D
:10934000F90185919491F901329665917491A80182
:1093500047705527649F9001659F300D749F300DB5
:10936000112443E0369527954A95E1F7821B930B2C
:109370008436910588F487E4E82E82E0F82ED70140
:109380008D917D01882319F00E94553CF8CFC801CA
:109390000E94FEBA84E690E09093F2078093F10772
:1093A0008091F3078093F007F60183AD94AD90931D
:1093B000EF078093EE078134FCE99F0728F48132A0
:1093C0000EE4900748F002C080E49CE996958795EA
:1093D0009695879524E007C0813117E2910730F018
:1093E0009695879522E02093F30708C021E020930B
:1093F000F3078032910510F480E290E08C01005276
:109400001109011528E01207D8F0E12FFF27EE0F10
:10941000FF1FEE0FFF1FCF018857924FFC013296BE
:1094200045915491AA27059F9001049F210D3A1F51
:1094300006942A1F3A1F1124FC01859194911CC0A7
:109440009801369527952C7F2857364FF90185913D
:109450009491F901329665917491A801477055274E
:10946000649F9001659F300D749F300D112473E04F
:10947000369527957A95E1F7821B930B84369105F3
:1094800088F457E4E52E52E0F52ED7018D917D0149
:10949000882319F00E94553CF8CFC8010E94FEBAFB
:1094A00084E690E0AC0160E070E04093EA075093FE
:1094B000EB076093EC077093ED079093890080931E
:1094C0008800F60182899389A489B589B695A79504
:1094D00097958795B095A095909581959F4FAF4FA3
:1094E000BF4F8093E6079093E707A093E807B093F8
:1094F000E9078093E2079093E307A093E407B09312
:10950000E5078093DE079093DF07A093E007B09311
:10951000E1078093DA079093DB07A093DC07B09311
:10952000DD071092FC071092FD071092FE071092C3
:10953000FF0707C080ED97E0909389008093880033
:109540002CC48091C60E81110E94BD912091F30719
:10955000222309F4A1C1E091D207F091D3074091F1
:10956000DA075091DB076091DC077091DD0782819B
:109570009381A481B581840F951FA61FB71F809387
:10958000DA079093DB07A093DC07B093DD0718168A
:1095900019061A061B060CF45F9AE091D207F091A7
:1095A000D3074091DE075091DF076091E00770918B
:1095B000E10786819781A085B185840F951FA61F3D
:1095C000B71F8093DE079093DF07A093E007B09367
:1095D000E107181619061A061B060CF4469AE091C4
:1095E000D207F091D3074091E2075091E3076091D1
:1095F000E4077091E50782859385A485B585840F7E
:10960000951FA61FB71F8093E2079093E307A093CF
:10961000E407B093E507181619061A061B060CF4A2
:109620002B9AE091D207F091D3074091E607509131
:10963000E7076091E8077091E90786859785A0891B
:10964000B189840F951FA61FB71F8093E6079093DB
:10965000E707A093E807B093E907181619061A065A
:109660001B060CF4299A8091DA079091DB07A091F0
:10967000DC07B091DD07181619061A061B0684F5DB
:10968000E091D207F091D3074289538964897589A3
:10969000841B950BA60BB70B8093DA079093DB071F
:1096A000A093DC07B093DD07809104014091F30D96
:1096B0005091F40D6091F50D7091F60D082E000C8F
:1096C000990BAA0BBB0B840F951FA61FB71F809386
:1096D000F30D9093F40DA093F50DB093F60D5F98F4
:1096E0008091DE079091DF07A091E007B091E1073C
:1096F000181619061A061B0684F5E091D207F09198
:10970000D3074289538964897589841B950BA60BFD
:10971000B70B8093DE079093DF07A093E007B09329
:10972000E107809105014091F70D5091F80D60918E
:10973000F90D7091FA0D082E000C990BAA0BBB0BBA
:10974000840F951FA61FB71F8093F70D9093F80DF8
:10975000A093F90DB093FA0D46988091E20790918D
:10976000E307A091E407B091E507181619061A0659
:109770001B0684F5E091D207F091D3074289538903
:1097800064897589841B950BA60BB70B8093E20740
:109790009093E307A093E407B093E5078091060157
:1097A0004091FB0D5091FC0D6091FD0D7091FE0DEF
:1097B000082E000C990BAA0BBB0B840F951FA61F3C
:1097C000B71F8093FB0D9093FC0DA093FD0DB093FC
:1097D000FE0D2B988091E6079091E707A091E8078E
:1097E000B091E907181619061A061B0684F5E091D0
:1097F000D207F091D3074289538964897589841B04
:10980000950BA60BB70B8093E6079093E707A09301
:10981000E807B093E907809107014091FF0D50914F
:10982000000E6091010E7091020E082E000C990B33
:10983000AA0BBB0B840F951FA61FB71F8093FF0DAC
:109840009093000EA093010EB093020E2998809180
:10985000FC079091FD07A091FE07B091FF070196CC
:10986000A11DB11D8093FC079093FD07A093FE07F7
:10987000B093FF072150E091D207F091D3074289BE
:1098800053896489758984179507A607B70708F473
:109890005FCEBB24B39401C0B12C4091FC07509122
:1098A000FD076091FE077091FF07E090D207F090EE
:1098B000D307F70186899789A08DB18D8417950705
:1098C000A607B70708F401C14091EA075091EB07DA
:1098D0006091EC077091ED07068D178D20A131A1E5
:1098E000AA27419FB12D529FC001629F900D619F99
:1098F000800D911D429FB00D811D9A1F519FB00D8B
:10990000811D9A1F609FB00D811D9A1F509FB10D40
:109910008A1F9A1FB6958A1F9A1F349F800D911D2A
:10992000359F900D112423AD34AD820F931F90937A
:10993000EF078093EE0747A950AD61AD72ADA0E08F
:10994000B0E0481759076A077B0720F45093EF07E8
:109950004093EE078091EE079091EF078134BCE9C8
:109960009B0728F48132EEE49E0748F002C080E4B1
:109970009CE9969587959695879524E007C0813157
:10998000F7E29F0730F09695879522E02093F30742
:1099900008C021E02093F3078032910510F480E2A3
:1099A00090E08C0100521109011528E01207E8F03F
:1099B000E12FFF27EE0FFF1FEE0FFF1FCF0188578C
:1099C000924FFC01329625913491AA27039FA00162
:1099D000029F410D5A1F06944A1F5A1F1124FC0171
:1099E00025913491241B350B1EC0A801569547952F
:1099F0004C7F4857564FFA0125913491FA0132961F
:109A000065917491A80147705527649FC001659FB7
:109A1000900D749F900D1124B3E096958795BA959B
:109A2000E1F7281B390B2436310588F4F7E4EF2ED3
:109A3000F2E0FF2ED7018D917D01882319F00E945D
:109A4000553CF8CFC8010E94FEBA24E630E0809170
:109A5000C60E882301F1C901293BBBE03B07E0F0BA
:109A600068EB7BE00E9462E2883EE3E09E0718F428
:109A70008854944F02C088EB9BE0A901481B590B06
:109A800060E070E04093F8075093F9076093FA079D
:109A90007093FB0701C0C9019093890080938800EF
:109AA0008091EA079091EB07A091EC07B091ED0748
:109AB000820F931FA11DB11D8093EA079093EB07BE
:109AC000A093EC07B093ED0743C14091FC07509180
:109AD000FD076091FE077091FF07F701828D938D5E
:109AE000A48DB58D84179507A607B70708F000C1A8
:109AF0000091F4071091F5072091F6073091F707D0
:109B000009831A832B833C83468D578D60A171A1F5
:109B1000AA27059FB12D169F6001269FD00C259F77
:109B2000C00CD11C069FB00DC11CDA1E159FB00DD4
:109B3000C11CDA1E249FB00DC11CDA1E149FB10D8A
:109B4000CA1EDA1EB695CA1EDA1E709FC00CD11C42
:109B5000719FD00C11248091EE079091EF07FF9632
:109B6000C816D90680F48C199D0940815181628103
:109B700073816C01E12CF12CC416D506E606F706BC
:109B800020F4CA0102C08081918181341CE99107CF
:109B900028F481322EE4920748F002C080E49CE968
:109BA000969587959695879524E007C0813137E291
:109BB000930730F09695879522E02093F30708C02D
:109BC00021E02093F3078032910510F480E290E0C9
:109BD0008C0100521109011548E01407E8F0E12F4B
:109BE000FF27EE0FFF1FEE0FFF1FCF018857924F89
:109BF000FC01329625913491AA27039FA001029F70
:109C0000410D5A1F06944A1F5A1F1124FC01259129
:109C10003491241B350B1EC0C801969587958C7F07
:109C20008857964FFC0125913491FC01329665913D
:109C30007491A80147705527649FC001659F900DDE
:109C4000749F900D112443E0969587954A95E1F70E
:109C5000281B390B2436310588F487E4E82E82E08E
:109C6000F82ED7018D917D01882319F00E94553C73
:109C7000F8CFC8010E94FEBA24E630E08091C60EFB
:109C8000882301F1C901293BBBE03B07E0F068EB09
:109C90007BE00E9462E2883EE3E09E0718F488546D
:109CA000944F02C088EB9BE0A901481B590B60E070
:109CB00070E04093F8075093F9076093FA077093A8
:109CC000FB0701C0C90190938900809388008981B6
:109CD0009A81AB81BC81820F931FA11DB11D80931E
:109CE000F4079093F507A093F607B093F70730C0F9
:109CF0002091F1073091F2078091C60E882301F17F
:109D0000293BFBE03F07E0F0C90168EB7BE00E94E4
:109D100062E2883E03E0900718F48854944F02C032
:109D200088EB9BE0A901481B590B60E070E0409371
:109D3000F8075093F9076093FA077093FB079C01AB
:109D400030938900209388008091F0078093F30777
:109D50002091880030918900809184009091850045
:109D600040962817390748F4809184009091850027
:109D700040969093890080938800BB2071F01092E8
:109D8000D3071092D2070E94A13B882331F0809123
:109D9000C40E8F5F8F708093C40EF8948091320E42
:109DA000882321F080916E008B7F03C080916E002C
:109DB000846080936E0080916F00826080936F005A
:109DC0000F900F900F900F90DF91CF91FF91EF9137
:109DD000BF91AF919F918F917F916F915F914F91C3
:109DE0003F912F911F910F91FF90EF90DF90CF90B7
:109DF000BF900F900BBE0F900FBE0F901F90189545
:109E00000E94A13B882309F4DDC98091C40E8F5FB5
:109E10008F708093C40ED6C91092D5071092D407C4
:109E2000D1C93FB7F8948091380890913908A09132
:109E30003A08B0913B0826B5A89B05C02F3F19F002
:109E40000196A11DB11D3FBFBA2FA92F982F8827BA
:109E5000820F911DA11DB11DBC01CD0142E0660F15
:109E6000771F881F991F4A95D1F7089508950F937A
:109E70001F93CF93DF93DC0116960D911C911797DA
:109E80001596CC911597D0E083E0D695C7958A9525
:109E9000E1F7362F3770E0E8F0E002C0F595E7957E
:109EA0003A95E2F712968C91481B4C9FD0014D9F3A
:109EB000B00D1124669566956695A60FB11DA00F8D
:109EC000B11F8C91222311F0E82B02C0E095E8230A
:109ED000EC93DF91CF911F910F910895FB01418188
:109EE000DC0112962C911297421768F013962C9170
:109EF0001397241740F0608115962C91621718F47F
:109F000024810C94374F0895FC0180819281980F31
:109F100092832181921760F494819F5F948393814F
:109F2000890F821710F08FEF820F838381E00895ED
:109F300080E00895FC011282808181508383148225
:109F4000089580E008950B96FC01849108950A9687
:109F5000FC0184910895FC01849108950E94AB4F07
:109F6000882321F0823011F083E0089586E008957F
:109F7000FC01E60FF11D849190E0982F882731961F
:109F8000E4918E0F911D089568E00C94B84F66E03F
:109F90000C94B84F2EE93FE0009729F0F901319772
:109FA000F1F70197F9CF0895909131082091300889
:109FB00050912F0860912E08A0912C08B0912D0887
:109FC000E0912A08F0912B083FB730933208F894BB
:109FD0003C91392B4C91422398E087FF02C03C937F
:109FE00001C04C93880F2081262320832081252BBC
:109FF0002083915091F7809132088FBF0895CF93BD
:10A00000C62F811102C088EF03C0813019F48AEF96
:10A010000E94D44F8C2F807F0E94D44F8C2F82952A
:10A02000807F0E94D44F88E290E0FC013197F1F7E5
:10A03000FC013197F1F7FC013197F1F70197F1F746
:10A04000CF9108959F92AF92BF92CF92DF92EF92FD
:10A05000FF920F931F93CF93DF937C018B01942E7C
:10A0600069012AE04217C9F035E14313B7C0FB018B
:10A07000A280B38040E00E9492C441E0B801C701D1
:10A080000E949BC4D5011296CC9112971696AD9062
:10A09000BC901797D0E2DC0F67C0DB011496ED91FE
:10A0A000FC91159720E030E043E061E0099580E005
:10A0B00095EDA92E91E1B92EF501C49181110BC046
:10A0C000CF3F09F44CC04C2FB801C7010E9489C48E
:10A0D000811143C083C0CF3F11F44FEFF5CFCE3F86
:10A0E00009F47CC0C03FC8F5C03E38F04C2F4F701B
:10A0F000B801C7010E9492C430C0C03D38F04C2F57
:10A100004F70B801C7010E949BC427C0C03CF8F043
:10A11000D8011496ED91FC91159720E030E040E0D5
:10A1200064E0C7010995C295C07FCE5FD0E0CE0143
:10A130000E94CA4FD8011496ED91FC91159720E02A
:10A1400030E041E064E0C7010995CE0104C0C7FDDD
:10A1500004C08C2F90E00E94CA4F80E001C081E0D3
:10A16000BFEFAB1ABB0AA8CF40E0B801C7010E94FD
:10A1700092C44EE3B801C7010E9489C4C03240F4C2
:10A180004C2F4068B801C7010E9489C440E808C04C
:10A1900040EE4C0F4068B801C7010E9489C448E8EE
:10A1A000B801C7010E9489C441E0B801C7010E94FB
:10A1B00092C4D8011496ED91FC911597950140E158
:10A1C00066E0C7010995B0E1AB0EB11CCF5FCD13BE
:10A1D000CBCF40E0B801C7010E949BC4F801C28107
:10A1E000D381F2E39F1609F46CC0F915B0F025E1B4
:10A1F000921609F473C037E1931609F483C044E161
:10A20000941296C08D81EE81FF819F0144E0849F6E
:10A21000200D311D1124C90159C086E4981609F496
:10A2200080C097E4991609F480C0ABE39A1280C00D
:10A23000F60181819381913029F0933031F4482FD8
:10A24000885004C048E0480F01C0482F21E03B81FE
:10A25000381708F420E031E05A81451708F430E05F
:10A2600051E0481708F050E0822F852B382319F46D
:10A27000252309F45DC0D6011296FC90913051F06F
:10A2800030F0923049F0933051F41FEF09C010E0E4
:10A2900001E007C011E004C010E00FEF02C010E0C1
:10A2A00000E0F7FE04C0B601CE010E946E4FF60139
:10A2B0008081800F80838181810F8183FF0C89F7EA
:10A2C00037C0B601CE010E946E4F32C01192E8171E
:10A2D000F907E1F7CE010E949A4F2AC0CE010E94F1
:10A2E000844F882331F18D81EE81FF81DF0124E0ED
:10A2F000829FA00DB11D1124CD011192E817F9071D
:10A30000E1F716C0D6011C928A8111968C931197A1
:10A310008D81815012968C9312978B8113968C931A
:10A3200007C08D81F601808303C08981D6018C939B
:10A3300081E0DF91CF911F910F91FF90EF90DF901F
:10A34000CF90BF90AF909F900895EF92FF920F93A0
:10A350001F93CF93DF93EC01142F7901862F90E0A8
:10A36000FC013197E730F10508F089C0EA5BFF4F47
:10A370000C94A9E27E0183E2E80EF11C8E01005DDF
:10A380001F4FF70180818F3F41F061E00E9487609D
:10A3900061E0F70180810E945760FFEFEF1AFF0A2A
:10A3A000E016F10671F740E062E0CE010E947FC442
:10A3B00041E064E0CE010E947FC440E065E0CE0150
:10A3C0000E947FC46FA188A50E944AC41EA257C0E4
:10A3D0008BA18F3F09F453C060E004C0411106C057
:10A3E00040E062E0CE010E947FC449C041E062E0EB
:10A3F000CE010E947FC46FA188A50E944AC43FC0BD
:10A40000642F8EA10E94FF4F3AC08EA1811102C01D
:10A4100088EF03C0813019F48AEF0E94D44FC8E25C
:10A42000D0E0112389F0F7018081807F0E94D44F12
:10A43000F70181917F018295807F0E94D44F115056
:10A44000CE010197F1F7EDCF88E290E0FC01319762
:10A45000F1F7FC013197F1F7FC013197F1F7019722
:10A46000F1F70DC0112359F0F70164918EA10E94FC
:10A47000FF4FFFEFEF1AFF0A1150F4CF4EA381E018
:10A48000DF91CF911F910F91FF90EF9008951F934F
:10A49000CF93DF93182FEB0161E00E948760209734
:10A4A00011F460E004C0CF3FD10539F461E0812FA1
:10A4B000DF91CF911F910C945760E12FF0E0EC55A4
:10A4C000FD4EE4914E2F50E0FA013197EA30F1054C
:10A4D00008F046C0E35BFF4F0C94A9E284B58068A6
:10A4E00084BDC7BD42C084B5806284BDC8BD3DC0C7
:10A4F00080918000806880938000D0938900C09311
:10A50000880033C080918000806280938000D09367
:10A510008B00C0938A0029C08091B000806880932E
:10A52000B000C093B30021C08091B00080628093DE
:10A53000B000C093B40019C08091900080688093EF
:10A540009000D0939900C09398000FC08091900024
:10A55000806280939000D0939B00C0939A0005C0C6
:10A56000C038D1050CF0A2CF9CCFDF91CF911F91C5
:10A5700008958F929F92AF92BF92CF92DF92EF9207
:10A58000FF926B017C010E94114F4B015C01C114D1
:10A59000D104E104F104F1F00E94114FDC01CB0180
:10A5A00088199909AA09BB09883E9340A105B105FC
:10A5B00070F321E0C21AD108E108F10888EE880E94
:10A5C00083E0981EA11CB11CC114D104E104F10464
:10A5D00019F7DDCFFF90EF90DF90CF90BF90AF9055
:10A5E0009F908F9008952FB7F894609134087091E0
:10A5F000350880913608909137082FBF08951F9233
:10A600000F920FB60F9211242F933F938F939F9326
:10A61000AF93BF938091340890913508A09136088C
:10A62000B09137083091330823E0230F2D3720F401
:10A630000196A11DB11D05C026E8230F0296A11D9C
:10A64000B11D209333088093340890933508A0936C
:10A650003608B09337088091380890913908A09156
:10A660003A08B0913B080196A11DB11D80933808AE
:10A6700090933908A0933A08B0933B08BF91AF91EB
:10A680009F918F913F912F910F900FBE0F901F9030
:10A690001895DB01ED91FC9109948F929F92BF92E6
:10A6A000CF92DF92EF92FF920F931F93CF93DF939E
:10A6B0001F92CDB7DEB74C01062FF42E122F522F6A
:10A6C000E62EE20EBB24BA946C018CE1C80ED11CBC
:10A6D0008E2D851B583080F0F40162817381848F48
:10A6E000F58E178EB68E96014BE3C40159830E94F6
:10A6F000495359815850ECCF812F887F080F212F63
:10A70000277021F187E02827F40162817381048F8B
:10A71000F58E178E2F5F27708FEF90E001C0880FA6
:10A720002A95EAF7868F9401245E3F4F4BE3C401DC
:10A730000F90DF91CF911F910F91FF90EF90DF90DD
:10A74000CF90BF909F908F900C9449530F90DF91C2
:10A75000CF911F910F91FF90EF90DF90CF90BF901E
:10A760009F908F900895EF92FF920F931F93CF9336
:10A77000DF937C01D62F122FC42F040F212F4C2FD3
:10A780006D2FC7010E944D53CF5F0C13F7CFDF91A0
:10A79000CF911F910F91FF90EF900895DF92EF926C
:10A7A000FF920F931F93CF93DF93EC01162FF42E9C
:10A7B000E22E0E94A4C4882331F02E2D4F2D612F4C
:10A7C000CE010E94B353DF91CF911F910F91FF9063
:10A7D000EF90DF900895EF92FF920F931F93CF9326
:10A7E000DF931F92CDB7DEB78C01DC011296ED909E
:10A7F000FC901397D196ED91FC91D29782E0099548
:10A8000020E030E04AE0B701C8010E944953F82E29
:10A81000D801D196ED91FC91D29783E00995D801AA
:10A82000D196ED91FC91D29780E00995FF20A1F19E
:10A83000F801628173819E012F5F3F4F46E4C8019A
:10A840000E9449538981D8018C9312966D917C9115
:10A8500013979E012F5F3F4F47E4C8010E94495361
:10A860008981F80181836281738120E030E048E4CE
:10A87000C8010E944953D8011B968C931B979801DD
:10A880002D5C3F4F12966D917C91139747E1C80163
:10A890000E94495381E001C080E00F90DF91CF9189
:10A8A0001F910F91FF90EF9008952F923F925F922A
:10A8B0006F927F928F929F92AF92BF92CF92DF92D0
:10A8C000EF92FF920F931F93CF93DF931F92CDB719
:10A8D000DEB71C01C62E142FD22EDC011496ED908B
:10A8E000FC901597C7010E94AB4F082FF10184819E
:10A8F00095810E94AE4F982E013019F48FE0A82E5A
:10A9000002C0AA24AA94D10114968D919C91159706
:10A910000E94A74F082FF101848195810E94A34FC7
:10A92000B82ED10114968D919C9115970E94C44F19
:10A93000B0E6BD1530F4009721F0E80EF91E01E6EF
:10A9400011C0F101848195810E94C74FF0E4FD158B
:10A9500030F4009721F0E80EF91E01E403C021E174
:10A96000E20EF11CBD1480F4D10150961C92509758
:10A9700053961C92539754961C92549751961C923E
:10A98000519752961C92C7C0B01670F3892D90E073
:10A99000F70124912F3F21F4FFEFEF1AFF0A5AC06D
:10A9A0000D114FC0D10114968D919C9115970E9465
:10A9B000AB4F97012F5F3F4FF701882311F0823093
:10A9C000E1F48491D10153968C935397F90124912A
:10A9D00054962C935497F7013396E4915096EC9348
:10A9E0005097F7013496E4915196EC935197F70103
:10A9F0003596E4915296EC9320C08491982F9F70E5
:10AA00009250D10152969C93529782958F70519695
:10AA10008C935197F9012491822F8F7054968C93C7
:10AA2000549722952F7053962C935397F701329693
:10AA3000E491E295EF705096EC93E114F10479F40F
:10AA40006AC0F7013296E491EA219C012E0F311D74
:10AA5000E20EF31E0B1509F487CF0F5F99CFF101BA
:10AA6000848195810E94AE4FB82ED10153969C905F
:10AA700053975496DC90549751968C915197C80EE9
:10AA800052969C919D0D512E591A0D2D292D452D13
:10AA90006C2DC1010E94A4C48823D1F1C7018B0D84
:10AAA000911D5C0187E0890DF82EF694F694F694DA
:10AAB000D50C41019CE1890E911C6F2C712C5D1409
:10AAC00039F15C2D8501802F8A198F15E8F4F80182
:10AAD0008491D10112966D917C9113975C965C9351
:10AAE0005C975D965C925D975F961C925F975E9611
:10AAF0008C9394014BE3C10159830E9449530F5F2A
:10AB00001F4F5981585FDFCFA60CB71C5394D7CF86
:10AB1000F101808901C080E00F90DF91CF911F91FA
:10AB20000F91FF90EF90DF90CF90BF90AF909F90EC
:10AB30008F907F906F905F903F902F900895CF926D
:10AB4000DF92EF92FF920F931F93CF93DF9300D08A
:10AB500000D0CDB7DEB78091D00D9091D10DA091EE
:10AB6000D20DB091D30DB7FF08C01092D00D109246
:10AB7000D10D1092D20D1092D30D8091D40D9091E1
:10AB8000D50DA091D60DB091D70D4091D00D50911B
:10AB9000D10D6091D20D7091D30D84179507A60742
:10ABA000B70744F48093D00D9093D10DA093D20DAC
:10ABB000B093D30D80913201882379F14091D00D6B
:10ABC0005091D10D6091D20D7091D30D8091D80D1F
:10ABD0009091D90DA091DA0DB091DB0D6A017B0146
:10ABE000C80ED91EEA1EFB1EC701B6010E9446DC34
:10ABF0002AE037ED43E25CE30E94A5DC69837A83B7
:10AC00008B839C83CE0101960E94C6C4BC018091B7
:10AC1000DE0D9091DF0D0E94DAA080915008109116
:10AC2000E00D811106C01123D1F1809132018823FA
:10AC3000B1F14091D00D5091D10D6091D20D709134
:10AC4000D30D8091D80D9091D90DA091DA0DB091CE
:10AC5000DB0D6A017B01C80ED91EEA1EFB1EC7016F
:10AC6000B6010E9446DC2AE037ED43E25CE30E9435
:10AC7000A5DCE091DC0DF091DD0D309721F06083D3
:10AC8000718382839383112329F0E091E10DF09188
:10AC9000E20D09958091500881110E94579B809187
:10ACA0005008882329F0E091E10DF091E20D09951B
:10ACB0000F900F900F900F90DF91CF911F910F91F8
:10ACC000FF90EF90DF90CF900895CF92DF92EF92B8
:10ACD000FF920F931F93CF93DF9300D000D0CDB797
:10ACE000DEB78091D00D9091D10DA091D20DB09191
:10ACF000D30DB7FF08C01092D00D1092D10D109255
:10AD0000D20D1092D30D8091D40D9091D50DA091BC
:10AD1000D60DB091D70D4091D00D5091D10D6091CD
:10AD2000D20D7091D30D84179507A607B70744F489
:10AD30008093D00D9093D10DA093D20DB093D30DED
:10AD400080913201882379F14091D00D5091D10D3D
:10AD50006091D20D7091D30D8091D80D9091D90D45
:10AD6000A091DA0DB091DB0D6A017B01C80ED91EEE
:10AD7000EA1EFB1EC701B6010E9446DC2AE037ED41
:10AD800043E25CE30E94A5DC69837A838B839C8326
:10AD9000CE0101960E947BC5BC018091DE0D909191
:10ADA000DF0D0E94DAA0809150081091E00D811112
:10ADB00006C01123D1F1809132018823B1F1409175
:10ADC000D00D5091D10D6091D20D7091D30D809125
:10ADD000D80D9091D90DA091DA0DB091DB0D6A01DB
:10ADE0007B01C80ED91EEA1EFB1EC701B6010E94D8
:10ADF00046DC2AE037ED43E25CE30E94A5DCE0910B
:10AE0000DC0DF091DD0D309721F06083718382833A
:10AE10009383112329F0E091E10DF091E20D099562
:10AE20008091500881110E94579B809150080F908B
:10AE30000F900F900F90DF91CF911F910F91FF9086
:10AE4000EF90DF90CF9008950E946556882329F0F7
:10AE5000E091E10DF091E20D099408950C9465568E
:10AE6000CF92DF92EF92FF920F931F93CF93DF93D6
:10AE700000D000D0CDB7DEB78091D00D9091D10D2C
:10AE8000A091D20DB091D30DB7FF08C01092D00D94
:10AE90001092D10D1092D20D1092D30D8091D40D3D
:10AEA0009091D50DA091D60DB091D70D4091D00DB8
:10AEB0005091D10D6091D20D7091D30D84179507EB
:10AEC000A607B70744F48093D00D9093D10DA093BB
:10AED000D20DB093D30D80913201882379F1409146
:10AEE000D00D5091D10D6091D20D7091D30D809104
:10AEF000D80D9091D90DA091DA0DB091DB0D6A01BA
:10AF00007B01C80ED91EEA1EFB1EC701B6010E94B6
:10AF100046DC20E030E048EC52E40E94A5DC698386
:10AF20007A838B839C83CE0101960E94FCC5BC0171
:10AF30008091DE0D9091DF0D0E94DAA08091500883
:10AF40001091E00D811106C01123D1F180913201E1
:10AF50008823B1F14091D00D5091D10D6091D20D67
:10AF60007091D30D8091D80D9091D90DA091DA0DEB
:10AF7000B091DB0D6A017B01C80ED91EEA1EFB1ED3
:10AF8000C701B6010E9446DC20E030E048EC52E404
:10AF90000E94A5DCE091DC0DF091DD0D309721F0F1
:10AFA0006083718382839383112329F0E091E10D03
:10AFB000F091E20D09958091500881110E94579BF4
:10AFC0000F900F900F900F90DF91CF911F910F91E5
:10AFD000FF90EF90DF90CF900895CF92DF92EF92A5
:10AFE000FF920F931F93CF93DF9300D000D0CDB784
:10AFF000DEB78091D00D9091D10DA091D20DB0917E
:10B00000D30DB7FF08C01092D00D1092D10D109241
:10B01000D20D1092D30D8091D40D9091D50DA091A9
:10B02000D60DB091D70D4091D00D5091D10D6091BA
:10B03000D20D7091D30D84179507A607B70744F476
:10B040008093D00D9093D10DA093D20DB093D30DDA
:10B0500080913201882379F14091D00D5091D10D2A
:10B060006091D20D7091D30D8091D80D9091D90D32
:10B07000A091DA0DB091DB0D6A017B01C80ED91EDB
:10B08000EA1EFB1EC701B6010E9444DC20E030E04E
:10B0900048EC52E40E94A5DC69837A838B839C830D
:10B0A000CE0101960E94FCC5BC018091DE0D9091FD
:10B0B000DF0D0E94DAA0809150081091E00D8111FF
:10B0C00006C01123E1F1809132018823C1F1409142
:10B0D000D00D5091D10D6091D20D7091D30D809112
:10B0E000D80D9091D90DA091DA0DB091DB0D6A01C8
:10B0F0007B01C80ED91EEA1EFB1EC701B6010E94C5
:10B1000044DC20E030E048EC52E40E94A5DC0E94E0
:10B1100056E1E091DC0DF091DD0D309721F0608378
:10B12000718382839383112329F0E091E10DF091E3
:10B13000E20D09958091500881110E94579B8091E2
:10B140005008882329F0E091E10DF091E20D099576
:10B150000F900F900F900F90DF91CF911F910F9153
:10B16000FF90EF90DF90CF900895CF92DF92EF9213
:10B17000FF920F931F93CF93DF9300D000D0CDB7F2
:10B18000DEB78091D00D9091D10DA091D20DB091EC
:10B19000D30DB7FF08C01092D00D1092D10D1092B0
:10B1A000D20D1092D30D8091D40D9091D50DA09118
:10B1B000D60DB091D70D4091D00D5091D10D609129
:10B1C000D20D7091D30D84179507A607B70744F4E5
:10B1D0008093D00D9093D10DA093D20DB093D30D49
:10B1E00080913201882379F14091D00D5091D10D99
:10B1F0006091D20D7091D30D8091D80D9091D90DA1
:10B20000A091DA0DB091DB0D6A017B01C80ED91E49
:10B21000EA1EFB1EC701B6010E9446DC2FE632E1A2
:10B2200043E85AE30E94A5DC69837A838B839C837D
:10B23000CE0101960E94CD9EBC018091DE0D9091C1
:10B24000DF0D0E94DAA0809150081091E00D81116D
:10B2500006C01123D1F1809132018823B1F14091D0
:10B26000D00D5091D10D6091D20D7091D30D809180
:10B27000D80D9091D90DA091DA0DB091DB0D6A0136
:10B280007B01C80ED91EEA1EFB1EC701B6010E9433
:10B2900046DC2FE632E143E85AE30E94A5DCE09168
:10B2A000DC0DF091DD0D309721F060837183828396
:10B2B0009383112329F0E091E10DF091E20D0995BE
:10B2C0008091500881110E94579B809150088823DB
:10B2D00029F0E091E10DF091E20D09950F900F90AA
:10B2E0000F900F90DF91CF911F910F91FF90EF90F2
:10B2F000DF90CF900895CF92DF92EF92FF920F935D
:10B300001F93CF93DF9300D000D0CDB7DEB78091ED
:10B31000D00D9091D10DA091D20DB091D30DB7FF6A
:10B3200008C01092D00D1092D10D1092D20D109233
:10B33000D30D8091D40D9091D50DA091D60DB091E3
:10B34000D70D4091D00D5091D10D6091D20D7091DB
:10B35000D30D84179507A607B70744F48093D00D43
:10B360009093D10DA093D20DB093D30D8091320163
:10B37000882379F14091D00D5091D10D6091D20D7B
:10B380007091D30D8091D80D9091D90DA091DA0DC7
:10B39000B091DB0D6A017B01C80ED91EEA1EFB1EAF
:10B3A000C701B6010E9446DC2AE037ED43E25CE3C8
:10B3B0000E94A5DC69837A838B839C83CE010196EE
:10B3C0000E94E6C6BC018091DE0D9091DF0D0E94C7
:10B3D000DAA0809150081091E00D811106C0112370
:10B3E000D1F1809132018823B1F14091D00D50917B
:10B3F000D10D6091D20D7091D30D8091D80D9091A7
:10B40000D90DA091DA0DB091DB0D6A017B01C80E58
:10B41000D91EEA1EFB1EC701B6010E9446DC2AE0C7
:10B4200037ED43E25CE30E94A5DCE091DC0DF09196
:10B43000DD0D309721F06083718382839383112324
:10B4400029F0E091E10DF091E20D0995809150080D
:10B4500081110E94579B0F900F900F900F90DF91DA
:10B46000CF911F910F91FF90EF90DF90CF900895B3
:10B470000F931F93CF938091D00D9091D10DA091F8
:10B48000D20DB091D30DB7FF08C01092D00D10921D
:10B49000D10D1092D20D1092D30D8091D40D9091B8
:10B4A000D50DA091D60DB091D70D4091D00D5091F2
:10B4B000D10D6091D20D7091D30D84179507A60719
:10B4C000B70744F48093D00D9093D10DA093D20D83
:10B4D000B093D30D80913201882331F14091D00D8A
:10B4E0005091D10D6091D20D7091D30D8091D80DF6
:10B4F0009091D90DA091DA0DB091DB0D8A019B01DD
:10B50000080F191F2A1F3B1FC901B8010E9446DC02
:10B510000E944FE1CB010E94CBC7BC018091DE0DA0
:10B520009091DF0D0E94DAA080915008C091E00D4B
:10B53000811106C0CC23C1F1809132018823A1F191
:10B540004091D00D5091D10D6091D20D7091D30DDD
:10B550008091D80D9091D90DA091DA0DB091DB0DAD
:10B560008A019B01080F191F2A1F3B1FC901B8013F
:10B570000E9446DCE091DC0DF091DD0D309721F06A
:10B580006083718382839383CC2329F0E091E10D62
:10B59000F091E20D099580915008882329F0CF9110
:10B5A0001F910F910C94579BCF911F910F9108956C
:10B5B0008091D00D9091D10DA091D20DB091D30D6D
:10B5C000B7FF08C01092D00D1092D10D1092D20D7D
:10B5D0001092D30D8091D40D9091D50DA091D60DE0
:10B5E000B091D70D4091D00D5091D10D6091D20DF9
:10B5F0007091D30D84179507A607B70744F480937D
:10B60000D00D9093D10DA093D20DB093D30D809116
:10B610003201882399F02091D80D3091D90D809175
:10B62000D00D9091D10D820F931F0E94CBC7BC010A
:10B630008091DE0D9091DF0D0E94DAA0809150087C
:10B640002091E00D811106C0222311F18091320179
:10B650008823F1F04091D80D5091D90D8091D00DF3
:10B660009091D10D840F951FE091DC0DF091DD0DCF
:10B67000309711F091838083222329F0E091E10D2E
:10B68000F091E20D09958091500881110E94579B1D
:10B690008091500808950C94D85A0E94D85A882353
:10B6A00029F0E091E10DF091E20D099408951F93C6
:10B6B000CF93DF9310924E088091D00D9091D10DD1
:10B6C000A091D20DB091D30D81309048A105B10564
:10B6D00040F01092D00D1092D10D1092D20D109218
:10B6E000D30DC091D00D8091520818160CF5282F5B
:10B6F000082E000C330B255031094C2F0C2E000C5A
:10B70000550B42175307A4F085301CF0CBEFC80F40
:10B7100001C0C0E08C2F0C2E000C990BAA0BBB0BA8
:10B720008093D00D9093D10DA093D20DB093D30DF3
:10B73000C0933C08D0E012E0C11109C080913201F1
:10B740008823D9F121E041E063E172E115C0C13005
:10B7500049F480913201882381F120E041E06AE0E0
:10B7600072E10AC0C23061F480913201882329F16C
:10B7700020E041E069EF71E18D2F0E945DD31DC093
:10B78000C33049F4809132018823B9F020E041E0D0
:10B7900067EF71E1F1CFC43081F4809132018823E9
:10B7A00051F021E040E06CEE71E18D2F0E945DD3FD
:10B7B0008D2F0E94F8D510933201DF5FCF5FD53017
:10B7C00009F0BACFD0935208DF91CF911F9108951D
:10B7D000CF93DF9310924E088091D00D9091D10DB0
:10B7E000A091D20DB091D30D81309048A105B10543
:10B7F00040F01092D00D1092D10D1092D20D1092F7
:10B80000D30DC091D00D8091530818160CF5282F38
:10B81000082E000C330B255031094C2F0C2E000C38
:10B82000550B42175307A4F085301CF0CBEFC80F1F
:10B8300001C0C0E08C2F0C2E000C990BAA0BBB0B87
:10B840008093D00D9093D10DA093D20DB093D30DD2
:10B85000C0933C08D0E0C11109C080913201882317
:10B86000E9F021E041E069E372E115C0C13049F43B
:10B8700080913201882391F020E041E06AE272E198
:10B880000AC0C23059F480913201882339F020E097
:10B8900041E060E272E18D2F0E945DD3DF5FCF5FF8
:10B8A000D530C9F683E080935308DF91CF91089596
:10B8B0004F925F926F927F928F929F92AF92BF92C0
:10B8C000CF92DF92EF92FF920F931F93CF93DF936C
:10B8D00000D000D000D0CDB7DEB710910A011F3FD5
:10B8E00001F10E94F352C0904108D0904208E090CC
:10B8F0004308F0904408DC01CB018C199D09AE0986
:10B90000BF09B7FD0EC02091C40E8091C30E30E078
:10B910008F5F8F70082E000C990B2817390709F0DC
:10B92000FBC10E946CC88091891382FF40C0809146
:10B93000630881113EC081E08093630890915108B3
:10B940008927809350081092510883E08093320138
:10B95000109289130E94F352DC01CB018C509E4F50
:10B96000AF4FBF4F80938A1390938B13A0938C1388
:10B97000B0938D1388EE93E09E838D8382E390E0F5
:10B980009A838983BE016B5F7F4FCE0101960E942F
:10B99000A99C16E0115069F087EC9EE00E940B37DD
:10B9A00062E070E080E090E00E94B952F3CF109224
:10B9B00063080E94F3526B017C0180915F089091B3
:10B9C0006008A0916108B0916208A7019601281B48
:10B9D000390B4A0B5B0B57FF05C080914F0888233A
:10B9E00009F4F0C1D701C6018C599F4FAF4FBF4F2B
:10B9F00080935F0890936008A0936108B0936208F9
:10BA00008091881318162CF480918813843074F474
:10BA100008C080918813992781950CF4909504971C
:10BA20002CF48091500881119FC0AFC080914E08C6
:10BA3000882309F472C080918813181664F48091E9
:10BA40008813082E000C990B97FD03969595879502
:10BA5000959587950EC080918813082E000C990B40
:10BA600097FD0396959587959595879591958195E1
:10BA7000910980904A0890904B08A0904C08B09093
:10BA80004D0881149104A104B104D1F1BC01990FB6
:10BA9000880B990B0E9446DC2B013C01C701B601C3
:10BAA000681979098A099B090E9444DC9B01AC0151
:10BAB000C301B2010E94DDE020E030E04AE754E437
:10BAC0000E94A5DC4B015C0120E030E040E253E441
:10BAD0000E94DDE187FF0FC020E030E046E952E43C
:10BAE000C501B4010E94DDE187FD0AC02AE030E013
:10BAF00040E050E009C024E630E040E050E004C0FF
:10BB000021E030E040E050E0C0924A08D0924B087B
:10BB1000E0924C08F0924D0804C021E030E040E093
:10BB200050E0A09188130A2E000CBB0B0E94B2E2D9
:10BB300024E030E040E050E00E948AE28091D00DA5
:10BB40009091D10DA091D20DB091D30D820F931F82
:10BB5000A41FB51F8093D00D9093D10DA093D20D4B
:10BB6000B093D30D10928813D701C6018856954C17
:10BB7000AF4FBF4F80935B0890935C08A0935D0824
:10BB8000B0935E0881E08093320180913001909102
:10BB900031018B5F954941F480910B01882309F4B1
:10BBA000E1C0815080930B012FB7F8948091450834
:10BBB00090914608A0914708B09148082FBF3AE0FD
:10BBC000B695A795979587953A95D1F7009741E057
:10BBD000A407B10520F08FEF9FEFA0E0B0E09695AD
:10BBE000879520913201211105C030914F08311104
:10BBF000E5C055C0009741F04091590850915A084E
:10BC00004817590708F04BC080914F08811111C0A7
:10BC1000223050F0243028F0243031F410923201D8
:10BC200003C081E0809332010E9462BC81E0809376
:10BC30004F0884E00E9477A081E08093850EE09118
:10BC40003001F091310109951092500880914F0810
:10BC5000882351F00E94C0BB91E0811101C090E0A7
:10BC600090934F0891118EC08090590890905A0877
:10BC7000A12CB12C0E94F352DC01CB018C199D093F
:10BC8000AE09BF0988169906AA06BB0640F40E94B1
:10BC9000F3526C197D0970935A086093590880918A
:10BCA0003001909131018B5F954921F080914908D5
:10BCB000882379F088E9C80E8AE3D81EE11CF11CBC
:10BCC000C0925B08D0925C08E0925D08F0925E083A
:10BCD0000FC080915B0890915C08A0915D08B091C5
:10BCE0005E08C81AD90AEA0AFB0AF7FE0E94509BAE
:10BCF00080914F08811166C080913201813049F0F6
:10BD000008F460C0843008F05DC081E080933201A7
:10BD100059C01092320156C024E01202F0011124E1
:10BD2000E956FE4F20E030E040E752E46081718147
:10BD3000828193810E94DDE069837A838B839C8377
:10BD4000E12C8E010F5F1F4F2FE03EE04BE05EE0E5
:10BD500067E07EE083E09EE00E942BCB8FEF809334
:10BD60000A01DFCD8CE080930B01809159089091FE
:10BD70005A08019790935A088093590881E080935C
:10BD8000320112CF8090590890905A08A12CB12C02
:10BD90000E94F352DC01CB018C199D09AE09BF0949
:10BDA00088169906AA06BB0668F40E94F3526C191D
:10BDB0007D0970935A086093590804C0009709F4EC
:10BDC00038CF1ACF26960FB6F894DEBF0FBECDBF80
:10BDD000DF91CF911F910F91FF90EF90DF90CF9067
:10BDE000BF90AF909F908F907F906F905F904F909B
:10BDF0000895CF92DF92EF92FF920F931F930E94CC
:10BE0000F35200915508109156082091570830912F
:10BE100058086B017C01C01AD10AE20AF30AF7FC48
:10BE200013C020915408209520935408DC01CB01C5
:10BE30008A549C4FAF4FBF4F80935508909356083C
:10BE4000A0935708B093580881E09091540891113D
:10BE500001C080E01F910F91FF90EF90DF90CF9095
:10BE60000895CF93DF931F92CDB7DEB780919E0EDA
:10BE7000811107C081E080939E0E85E69EE00E94BE
:10BE8000EB536091670E7091680E19829E012F5FCF
:10BE90003F4F4FE085E69EE00E94495353985B9ADE
:10BEA00052985A9A3898409A0E946CC810928813F7
:10BEB0000F90DF91CF910895CF93DF9300D0CDB74E
:10BEC000DEB789839A830E94309B40E050E0BA013C
:10BED00089819A810F900F90DF91CF910C9425A0CA
:10BEE0008A30910508F05DC0FC01E95AFF4F0C94BF
:10BEF000A9E281E08093490840E050E0BA0189E27C
:10BF000094E708C081E08093490840E050E0BA011E
:10BF100088E993E70C9425A081E08093490840E0EC
:10BF200050E0BA0185EE91E7F5CF81E080934908B2
:10BF300040E050E0BA0184E591E7ECCF81E08093E6
:10BF4000490840E050E0BA0187E59BE5E3CF81E096
:10BF50008093490840E050E0BA0186E792E7DACFE3
:10BF600081E08093490840E050E0BA0187E093E720
:10BF7000D1CF81E08093490810923E0810923D088D
:10BF800040E050E0BA018AEB94E7C4CF81E08093AF
:10BF9000490840E050E0BA0188EE9BE5BBCF0C9425
:10BFA000509B0895CF92DF92EF92FF920F931F93D1
:10BFB000CF93DF936C017A018B01C0E0D0E0CE1506
:10BFC000DF0589F0D8016D918D01D601ED91FC91CD
:10BFD0000190F081E02DC6010995892B11F47E01B5
:10BFE00002C02196ECCFC701DF91CF911F910F9135
:10BFF000FF90EF90DF90CF90089590E0FC01319793
:10C00000EA30F10540F5EF59FF4F0C94A9E2809119
:10C0100080008F7703C0809180008F7D80938000A7
:10C02000089584B58F7702C084B58F7D84BD08954F
:10C030008091B0008F7703C08091B0008F7D809396
:10C04000B0000895809190008F7703C08091900098
:10C050008F7D8093900008950E94BAE2CF93DF9382
:10C06000282F30E0F901EC55FD4E8491F901EC5791
:10C07000FD4ED491F901EC59FD4EC491CC2391F0C1
:10C0800081110E94FD5FEC2FF0E0EE0FFF1FE65ADA
:10C09000FD4EA591B491EC91ED2381E090E021F467
:10C0A00080E002C080E090E0DF91CF9108951F937F
:10C0B000CF93DF93282F30E0F901EC55FD4E8491AA
:10C0C000F901EC57FD4ED491F901EC59FD4EC491A4
:10C0D000CC23C9F0162F81110E94FD5FEC2FF0E0F8
:10C0E000EE0FFF1FE05BFD4EA591B4918FB7F89462
:10C0F000111105C09C91ED2FE095E92302C0EC9150
:10C10000ED2BEC938FBFDF91CF911F910895CF93CB
:10C11000DF9390E0FC01EC57FD4E2491FC01EC59BB
:10C12000FD4E8491882361F190E0880F991FFC01F6
:10C13000EA5BFD4EC591D491FC01E05BFD4EA591FB
:10C14000B491611109C09FB7F8948881209582232A
:10C150008883EC912E230BC0623061F49FB7F89472
:10C160003881822F809583238883EC912E2B2C930A
:10C170009FBF06C08FB7F894E8812E2B28838FBF0E
:10C18000DF91CF9108951F93CF93DF9310924E08C4
:10C190008091D00D9091D10DA091D20DB091D30D81
:10C1A00081309048A105B10540F01092D00D109259
:10C1B000D10D1092D20D1092D30DC091D00D80915F
:10C1C000320A1816DCF4282F082E000C330B2150ED
:10C1D00031094C2F0C2E000C550B4217530774F0ED
:10C1E000CFEFC80F8C2F90E0A0E0B0E08093D00D8F
:10C1F0009093D10DA093D20DB093D30D1092700AED
:10C2000080913C08C81714F4C0933C0880913C0806
:10C21000082E000C990B04962C2F0C2E000C330BBF
:10C220008217930724F48CEF8C0F80933C081091B5
:10C230003C08D0E011111AC080915008811106C04D
:10C2400080913201882309F48DC009C0C111F8CF53
:10C250000E94579B8091700A882391F38AC081E0E5
:10C26000C11180E024E048E156E179C01130E9F4E1
:10C2700080915008811106C080913201882309F411
:10C2800071C00BC0C130C1F785E493E60E945C5FCA
:10C290008091700A882381F36CC081E0C13009F07D
:10C2A00080E023E041E156E15AC01230E9F4809188
:10C2B0005008811106C080913201882309F452C0D0
:10C2C0000BC0C230C1F78BE493E60E945C5F8091A3
:10C2D000700A882381F34DC081E0C23009F080E00C
:10C2E00023E04AE056E13BC01330E1F4809150086E
:10C2F000811105C0809132018823A1F10BC0C330A8
:10C30000C9F781E593E60E945C5F8091700A8823FB
:10C3100089F32FC081E0C33009F080E023E043E0DF
:10C3200056E11DC01430F1F480915008811105C010
:10C33000809132018823B1F00BC0C430C9F787E582
:10C3400093E60E945C5F8091700A882389F311C094
:10C3500081E0C43009F080E023E04AEF55E16D2F21
:10C360000E9425C8DF5F1F5FD53009F063CFD093EF
:10C37000320ADF91CF911F910895EF92FF921F93A0
:10C38000CF93DF937C017093310A6093300A10924F
:10C390004E088091D00D9091D10DA091D20DB09109
:10C3A000D30D81309048A105B10540F01092D00D19
:10C3B0001092D10D1092D20D1092D30DC091D00DCC
:10C3C00080912F0A1816DCF4282F082E000C330B4E
:10C3D000215031094C2F0C2E000C550B42175307DE
:10C3E00074F0CFEFC80F8C2F90E0A0E0B0E0809306
:10C3F000D00D9093D10DA093D20DB093D30D109288
:10C40000700A80913C08C81714F4C0933C0820912E
:10C410003C08022E000C330B2C5F3F4F8C2F0C2E50
:10C42000000C990B2817390724F48CEF8C0F80939C
:10C430003C0810913C08D0E091E081E0E816F1045E
:10C4400069F122E0E216F10409F44CC0E114F104B0
:10C4500009F06CC0111191C09923B1F01C16A4F021
:10C460008091D00D9091D10DA091D20DB091D30DAE
:10C470000196A11DB11D8093D00D9093D10DA09375
:10C48000D20DB093D30DCF5F80913201882309F490
:10C49000EEC021E041E063EF75E16BC011116DC0AA
:10C4A0009923B1F01C16A4F08091D00D9091D10D7C
:10C4B000A091D20DB091D30D0196A11DB11D809315
:10C4C000D00D9093D10DA093D20DB093D30DCF5F2B
:10C4D00080913201882309F4CAC021E041E06CEE6A
:10C4E00075E147C0111149C09923B1F01C16A4F0A1
:10C4F0008091D00D9091D10DA091D20DB091D30D1E
:10C500000196A11DB11D8093D00D9093D10DA093E4
:10C51000D20DB093D30DCF5F80913201882309F4FF
:10C52000A6C021E041E065EE75E123C0111125C0F0
:10C530009923B1F01C16A4F08091D00D9091D10DEB
:10C54000A091D20DB091D30D0196A11DB11D809384
:10C55000D00D9093D10DA093D20DB093D30DCF5F9A
:10C5600080913201882309F482C021E041E06CED22
:10C5700075E18D2F0E945DD37AC01130D9F480917E
:10C580005008811106C080913201882309F46FC0E0
:10C5900009C0C130C1F70E94579B8091700A88235F
:10C5A00091F36DC081E0C13009F080E024E042EDFC
:10C5B00055E15AC01230E9F480915008811106C04B
:10C5C00080913201882309F452C00BC0C230C1F7F8
:10C5D00081E793E60E945C5F8091700A882381F373
:10C5E0004EC081E0C23009F080E023E048EC55E124
:10C5F0003BC01330E1F480915008811105C0809157
:10C6000032018823A1F10BC0C330C9F787E793E655
:10C610000E945C5F8091700A882389F330C081E0BA
:10C62000C33009F080E023E04FEB55E11DC014302A
:10C63000F1F480915008811105C080913201882366
:10C64000B1F00BC0C430C9F78DE793E60E945C5F80
:10C650008091700A882389F312C081E0C43009F008
:10C6600080E023E044EB55E16D2F0E9425C8DF5F99
:10C670001F5F90E0D53009F0E0CED0932F0ADF9114
:10C68000CF911F91FF90EF9008956FE475E680E0E1
:10C6900090E00C94BD6169E475E681E090E00C9453
:10C6A000BD6163E475E682E090E00C94BD6169EBE6
:10C6B00073E683E090E00C94BD6121E0209349088B
:10C6C00060932B0A70932C0A80932D0A90932E0A64
:10C6D00040E050E0BA018091300A9091310A0C9408
:10C6E00025A060E070E080E291E40C945D6360E07E
:10C6F00070E080E89FE30C945D636DEC7CEC8CEC67
:10C700009DE30C945D63CF92DF92EF92FF92CF9303
:10C71000C82F0E94F3526B017C0124EA30E74DE7F9
:10C720005FE360912B0A70912C0A80912D0A909101
:10C730002E0A0E943FDC87FD05C04AEF50E060E012
:10C7400070E003C040E050E0BA01C40ED51EE61E02
:10C75000F71EC0924108D0924208E0924308F0923E
:10C760004408C0930A01CF91FF90EF90DF90CF90E3
:10C7700008958091500881110C94579B6091D00DC1
:10C780007091D10D8091D20D9091D30D61157105ED
:10C790008105910579F10E9446DC20912B0A3091A8
:10C7A0002C0A40912D0A50912E0A0E94A5DC9B0173
:10C7B000AC0160910F0E7091100E8091110E90914E
:10C7C000120E0E945AE060930F0E7093100E809329
:10C7D000110E9093120E83E090E00E94836381E03B
:10C7E000809332011092D00D1092D10D1092D20D83
:10C7F0001092D30D80913201882349F08FE09EE0A2
:10C800000E949EC6BC018BEA95E10C94DAA00895C3
:10C810002F923F924F925F926F927F928F929F9250
:10C82000AF92BF92CF92DF92EF92FF920F931F933E
:10C83000CF93DF93CDB7DEB72A970FB6F894DEBF5C
:10C840000FBECDBF9A8789871B018091500888232E
:10C8500019F00E94579BFEC08091D00D9091D10D90
:10C86000A091D20DB091D30D892B8A2B8B2B09F47B
:10C87000C0C00E944A3C8101000F111F000F111F10
:10C88000F801ED5FF14F408051806280738020E0BD
:10C8900030E04AE754E4C301B2010E9459E04B0181
:10C8A0005C0120E030E04AE754E4C301B2010E9499
:10C8B0005AE06B017C0180911E018823E9F121E09F
:10C8C00022163104C1F032E02316310429F121147B
:10C8D000310491F580901C0A90901D0AA0901E0AC8
:10C8E000B0901F0AC0901201D0901301E090140183
:10C8F000F090150121C08090200A9090210AA0900C
:10C90000220AB090230AC0901601D0901701E0903F
:10C910001801F090190110C08090240A9090250A07
:10C92000A090260AB090270AC0901A01D0901B014F
:10C93000E0901C01F0901D018091D00D9091D10DDF
:10C94000A091D20DB091D30D8D839E83AF83B88714
:10C95000BC01CD010E9446DC20912B0A30912C0AAB
:10C9600040912D0A50912E0A0E94A5DC9B01AC013A
:10C97000C301B2010E945AE00D5F114FD8016D93BF
:10C980007D938D939C9313972D813E814F81588584
:10C9900057FF0DC0A50194010E943FDC87FF1BC01B
:10C9A000D8018D929D92AD92BC92139714C02D81A7
:10C9B0003E814F815885232B242B252B61F0A70125
:10C9C00096010E94DDE1181634F4D801CD92DD9273
:10C9D000ED92FC9213971092D00D1092D10D1092FF
:10C9E000D20D1092D30DC1010E94836381E0809328
:10C9F000320180913201882369F1F101EE0FFF1FAE
:10CA0000EE0FFF1FED5FF14F80819181A281B38115
:10CA100089839A83AB83BC832DEC3CEC4CEC5DE3C7
:10CA200060912B0A70912C0A80912D0A90912E0A08
:10CA30000E94DDE187FD05C0CE0101960E949EC6E1
:10CA400004C0CE0101960E94CD9EBC0189859A85C5
:10CA50000E94DAA02A960FB6F894DEBF0FBECDBFB3
:10CA6000DF91CF911F910F91FF90EF90DF90CF90CA
:10CA7000BF90AF909F908F907F906F905F904F90FE
:10CA80003F902F90089562E070E084EA95E10C9465
:10CA9000086461E070E08DE995E10C94086460E061
:10CAA00070E086E995E10C940864AF92BF92CF9252
:10CAB000DF92EF92FF920F931F93CF93DF93109229
:10CAC0004E088091D00D9091D10DA091D20DB091D2
:10CAD000D30D81309048A105B10540F01092D00DE2
:10CAE0001092D10D1092D20D1092D30DC091D00D95
:10CAF00080912A0A1816DCF4282F082E000C330B1C
:10CB0000215031094C2F0C2E000C550B42175307A6
:10CB100074F0CFEFC80F8C2F90E0A0E0B0E08093CE
:10CB2000D00D9093D10DA093D20DB093D30D109250
:10CB3000700A80913C08C81714F4C0933C08809197
:10CB40003C08082E000C990B04962C2F0C2E000C80
:10CB5000330B8217930724F48CEF8C0F80933C08DF
:10CB6000D0913C0810E088E5E82E85E1F82E9DE1A3
:10CB7000C92E95E1D92E23E8A22E25E1B22ED1119E
:10CB80001AC080915008811106C08091320188231B
:10CB900009F495C009C0C111F8CF0E94579B80913C
:10CBA000700A882391F328C181E0C11180E024E05C
:10CBB00041E955E181C0D130E9F4809150088111FB
:10CBC00006C080913201882309F479C00BC0C130BE
:10CBD000C1F783EC90E60E945C5F8091700A882325
:10CBE00081F30AC181E0C13009F080E023E047E829
:10CBF00055E162C0D230F9F480915008811106C02D
:10CC000080913201882309F45AC00DC0C230C1F7A7
:10CC1000B0924F0DA0924E0D0E94AE398091700AD5
:10CC2000882371F3E9C081E0C23009F080E020E29E
:10CC300049E755E141C0D33001F580915008811199
:10CC400005C0809132018823D1F10FC0C330C9F7EC
:10CC5000D0924F0DC0924E0D0E94AE390E94509B53
:10CC60008091700A882369F3C7C081E0C33009F05E
:10CC700080E020E24CE555E11FC0D43001F5809101
:10CC80005008811105C0809132018823C1F00DC088
:10CC9000C430C9F7F0924F0DE0924E0D0E94AE39AC
:10CCA0008091700A882379F3A7C081E0C43009F02D
:10CCB00080E020E247E455E1612F0E9425C8809181
:10CCC000C310811120C0D530E1F48091500881114A
:10CCD00005C0809132018823A1F009C0C530C9F791
:10CCE0000E9407B98091700A882399F385C081E07A
:10CCF000C53009F080E020E247E355E1612F0E9452
:10CD000025C806E001C005E08091E30D9091E40D97
:10CD10002091E70D3091E80D232B11F4892B21F19F
:10CD2000D01321C080915008811105C0809132013B
:10CD30008823C9F00FC0CD13F9CF1092E60D1092E1
:10CD4000E50D0E946F450E94509B8091700A8823D8
:10CD500069F352C081E0CD1380E020E24EE255E15C
:10CD6000612F0E9425C80F5FD0131DC0809150080D
:10CD7000811105C0809132018823A9F00BC0CD1329
:10CD8000F9CF8EEF97E60E945C5F8091700A88234E
:10CD900089F332C081E0CD1380E023E042E255E127
:10CDA000612F0E9425C881E0800FD8131DC080919B
:10CDB0005008811105C0809132018823A9F00BC071
:10CDC000CD13F9CF87E097E60E945C5F8091700AEF
:10CDD000882389F311C081E0CD1380E023E04DE684
:10CDE00055E1612F0E9425C81F5FDF5F153009F0F4
:10CDF000C6CE0E5F00932A0ADF91CF911F910F914B
:10CE0000FF90EF90DF90CF90BF90AF9008951F9369
:10CE1000CF93DF9310924E088091D00D9091D10D59
:10CE2000A091D20DB091D30D81309048A105B105EC
:10CE300040F01092D00D1092D10D1092D20D1092A0
:10CE4000D30DC091D00D8091290A1816DCF4282F3B
:10CE5000082E000C330B215031094C2F0C2E000CE6
:10CE6000550B4217530774F0CFEFC80F8C2F90E08B
:10CE7000A0E0B0E08093D00D9093D10DA093D20D9F
:10CE8000B093D30D1092700A80913C08C81714F427
:10CE9000C0933C0880913C08082E000C990B049626
:10CEA0002C2F0C2E000C330B8217930724F48CEFDD
:10CEB0008C0F80933C0810913C08D0E011111AC0EF
:10CEC00080915008811106C080913201882309F4B5
:10CED00089C009C0C111F8CF0E94579B8091700A88
:10CEE000882391F387C081E0C11180E024E045E10F
:10CEF00055E175C0113039F580915008811106C097
:10CF000080913201882309F46DC015C0C130C1F78A
:10CF100040914A0A50914B0A6091420A7091430A2B
:10CF20008091460A9091470A0E94C09F8091700AA2
:10CF3000882331F35FC081E0C13009F080E020E256
:10CF400049E055E14CC0123029F58091500881111B
:10CF500006C080913201882309F444C013C0C23056
:10CF6000C1F740914A0A50914B0A6FEF7FEF8091D1
:10CF7000460A9091470A0E94C09F8091700A8823B8
:10CF800041F338C081E0C23009F080E020E249EE90
:10CF900054E125C0133031F580915008811105C04E
:10CFA000809132018823F1F013C0C330C9F740915A
:10CFB0004A0A50914B0A6091420A7091430A80E0FC
:10CFC00090E00E94C09F8091700A882349F312C0AC
:10CFD00081E0C33009F080E020E249EF54E16D2F99
:10CFE0000E9425C8DF5F1F5FD53009F067CF84E05E
:10CFF0008093290ADF91CF911F9108951F93CF93BA
:10D00000DF9310924E088091D00D9091D10DA09198
:10D01000D20DB091D30D81309048A105B10540F0FB
:10D020001092D00D1092D10D1092D20D1092D30DFE
:10D03000C091D00D8091280A1816DCF4282F082EF4
:10D04000000C330B215031094C2F0C2E000C550BCA
:10D050004217530774F0CFEFC80F8C2F90E0A0E079
:10D06000B0E08093D00D9093D10DA093D20DB093EA
:10D07000D30D1092700A80913C08C81714F4C09325
:10D080003C0880913C08082E000C990B04962C2F2C
:10D090000C2E000C330B8217930724F48CEF8C0FAB
:10D0A00080933C0810913C08D0E011111AC0809187
:10D0B0005008811106C080913201882309F489C08B
:10D0C00009C0C111F8CF0E94579B8091700A882334
:10D0D00091F387C081E0C11180E024E041EE54E18A
:10D0E00075C0113039F580915008811106C08091CA
:10D0F0003201882309F46DC015C0C130C1F74091D9
:10D10000480A5091490A6091400A7091410A809101
:10D11000440A9091450A0E94C09F8091700A88231A
:10D1200031F35FC081E0C13009F080E020E245EDDD
:10D1300054E14CC0123029F580915008811106C08D
:10D1400080913201882309F444C013C0C230C1F772
:10D150004091480A5091490A6FEF7FEF8091440A4D
:10D160009091450A0E94C09F8091700A882341F3E4
:10D1700038C081E0C23009F080E020E245EB54E1A4
:10D1800025C0133031F580915008811105C0809180
:10D1900032018823F1F013C0C330C9F74091480A27
:10D1A0005091490A6091400A7091410A80E090E0F4
:10D1B0000E94C09F8091700A882349F312C081E0C9
:10D1C000C33009F080E020E245EC54E16D2F0E946D
:10D1D00025C8DF5F1F5FD53009F067CF84E08093FB
:10D1E000280ADF91CF911F9108952CEA35EC47E290
:10D1F0005EE36091650A7091660A8091670A90917A
:10D20000680A0E94DDE06093370A7093380A8093C1
:10D21000390A90933A0A08952CEA35EC47E25EE326
:10D220006091690A70916A0A80916B0A90916C0A08
:10D230000E94A5DC60933B0A70933C0A80933D0AF0
:10D2400090933E0A08952F924F926F927F928F9201
:10D250009F92AF92BF92CF92DF92EF92FF920F9385
:10D260001F93CF93DF9310924E088091D00D909131
:10D27000D10DA091D20DB091D30D81309048A10570
:10D28000B10540F01092D00D1092D10D1092D20D38
:10D290001092D30DD091D00D80916F0A1816DCF446
:10D2A000282F082E000C330B215031094D2F0D2E45
:10D2B000000C550B4217530774F0DFEFD80F8D2F7A
:10D2C00090E0A0E0B0E08093D00D9093D10DA093BA
:10D2D000D20DB093D30D1092700A80913C08D817EC
:10D2E00014F4D0933C0880913C08082E000C990B54
:10D2F00004962D2F0D2E000C330B8217930724F468
:10D300008CEF8D0F80933C08C0913C08412C63E06A
:10D31000262E74E9672E77E1772EE9EACE2EE7E133
:10D32000DE2EF7EBAF2EF7E1BF2EAEEB8A2EA7E194
:10D330009A2EC1111DC080915008811106C08091A4
:10D340003201882309F4AAC109C0D111F8CF0E9483
:10D35000579B8091700A882391F3A8C181E0D11175
:10D3600080E024E04CEC57E1642D0E9425C896C172
:10D37000C13009F03FC080915008811106C08091F2
:10D380003201882309F48AC116C0D130C1F7E12CDB
:10D3900010ECF12E09E714E420E030E040E85FE310
:10D3A00064E57AE085EC97E10E944BCE8091700AAB
:10D3B000882329F37BC12F9287EE8F931F9281E000
:10D3C0008F9384E59AE09F938F93BF92AF929F9241
:10D3D0008F924F9281E0D13009F080E08F930E94CC
:10D3E000DCD58DB79EB70C960FB6F8949EBF0FBED6
:10D3F0008DBF54C1C23009F041C0809150088111E5
:10D4000006C080913201882309F448C116C0D23089
:10D41000C1F7E12C10ECF12E09E714E420E030E034
:10D4200040E85FE368E57AE080EB97E10E944BCE4D
:10D430008091700A882329F339C12F9287EE8F9348
:10D440001F9281E08F9388E59AE09F938F93A2EAE1
:10D45000B7E1BF93AF93DF92CF924F9281E0D2308A
:10D4600009F080E08F930E94DCD58DB79EB70C96B3
:10D470000FB6F8949EBF0FBE8DBF10C1C33009F028
:10D4800041C080915008811106C0809132018823EB
:10D4900009F404C116C0D330C1F7E12C10ECF12E11
:10D4A00009E714E420E030E040E85FE36CE57AE06F
:10D4B0008BE997E10E944BCE8091700A882329F373
:10D4C000F5C02F9287EE8F931F9281E08F938CE5AA
:10D4D0009AE09F938F93ADE8B7E1BF93AF937F92AC
:10D4E0006F924F9281E0D33009F080E08F930E94D9
:10D4F000DCD58DB79EB70C960FB6F8949EBF0FBEC5
:10D500008DBFCCC0C43009F043C080915008811158
:10D5100006C080913201882309F4C0C016C0D430FF
:10D52000C1F7E12C10ECF12E09E714E420E030E023
:10D5300040E85FE360E67AE086E897E10E944BCE40
:10D540008091700A882329F3B1C02F9287EE8F93C0
:10D550001F9281E08F9380E69AE09F938F93A8E7D4
:10D56000B7E1BF93AF93AFE7B7E1BF93AF934F92EC
:10D5700081E0D43009F080E08F930E94DCD58DB734
:10D580009EB70C960FB6F8949EBF0FBE8DBF86C097
:10D59000C53009F041C080915008811106C08091CA
:10D5A0003201882309F47AC015C0D530C1F7E12CC7
:10D5B00010ECF12E09E714E420E030E0A90160E569
:10D5C0007AE083E797E10E944BCE8091700A88232E
:10D5D00031F36CC02F9287EE8F931F921F9280E5DC
:10D5E0009AE09F938F93A9E6B7E1BF93AF93AEE61E
:10D5F000B7E1BF93AF934F9281E0D53009F080E05F
:10D600008F930E94DCD58DB79EB70C960FB6F89419
:10D610009EBF0FBE8DBF42C0C63009F03FC0809193
:10D620005008811105C0809132018823B9F115C0DD
:10D63000D630C9F7E12C10ECF12E09E714E420E014
:10D6400030E0A9016CE47AE08FE597E10E944BCECF
:10D650008091700A882339F329C02F9287EE8F9327
:10D660001F921F928CE49AE09F938F93ABE4B7E1F3
:10D67000BF93AF93A5E5B7E1BF93AF934F9281E01E
:10D68000D63009F080E08F930E94DCD58DB79EB72D
:10D690000C960FB6F8949EBF0FBE8DBF4394CF5F1C
:10D6A00095E0491246CE87E080936F0ADF91CF91D3
:10D6B0001F910F91FF90EF90DF90CF90BF90AF90B0
:10D6C0009F908F907F906F904F902F9008950C9423
:10D6D000FFCA0C94D2C9AF92BF92CF92DF92EF9261
:10D6E000FF920F931F93CF93DF9310924E084091B8
:10D6F000D00D5091D10D6091D20D7091D30D41306C
:10D7000050486105710540F01092D00D1092D10D76
:10D710001092D20D1092D30DC091D00D90916E0A3F
:10D720001916DCF4292F092E000C330B2150310976
:10D730004C2F0C2E000C550B4217530774F0CFEFF3
:10D74000C90F4C2F50E060E070E04093D00D509333
:10D75000D10D6093D20D7093D30D1092700A9091F9
:10D760003C08C91714F4C0933C0820913C08022ED1
:10D77000000C330B2C5F3F4F4C2F0C2E000C550B25
:10D780002417350724F49CEF9C0F90933C081091CC
:10D790003C08D0E090E0880F991FFC01E05CF54F59
:10D7A0006F019C012C5B354F5901FC01E85BF54F83
:10D7B0007F0111111DC080915008811106C0809118
:10D7C0003201882309F493C009C0C111F8CF0E9427
:10D7D000579B8091700A882391F391C081E0C11119
:10D7E00080E024E04FE357E16D2F0E9425C87FC001
:10D7F000113041F580915008811106C080913201AD
:10D80000882309F474C010C0C130C1F72FEF30E095
:10D8100040E050E0B70185E397E10E94C2CE8091DD
:10D82000700A882359F36BC0F701808191810E94AF
:10D83000CBC79C0181E0C13009F080E000E04BE201
:10D8400057E152C0123041F580915008811106C055
:10D8500080913201882309F44AC010C0C230C1F758
:10D8600024E031E045E050E0B50184E297E10E9418
:10D87000C2CE8091700A882359F341C0F50180819E
:10D8800091810E94CBC79C0181E0C23009F080E009
:10D8900000E04DE157E128C0133049F58091500870
:10D8A000811105C080913201882309F110C0C33075
:10D8B000C9F724E630E045E050E0B60189E197E1A0
:10D8C0000E94C2CE8091700A882361F318C0F601CD
:10D8D000808191810E94CBC79C0181E0C33009F017
:10D8E00080E000E045E157E16D2F0E946CD5DF5FDD
:10D8F0001F5FD53009F05DCF84E080936E0ADF9121
:10D90000CF911F910F91FF90EF90DF90CF90BF903C
:10D91000AF90089581E00C946B6B80E00C946B6B7E
:10D920003F924F925F926F927F928F929F92AF92AF
:10D93000BF92CF92DF92EF92FF920F931F93CF93FC
:10D94000DF9310924E088091D00D9091D10DA0914F
:10D95000D20DB091D30D81309048A105B10540F0B2
:10D960001092D00D1092D10D1092D20D1092D30DB5
:10D97000C091D00D80916D0A1816DCF4282F082E66
:10D98000000C330B215031094C2F0C2E000C550B81
:10D990004217530774F0CFEFC80F8C2F90E0A0E030
:10D9A000B0E08093D00D9093D10DA093D20DB093A1
:10D9B000D30D1092700A80913C08C81714F4C093DC
:10D9C0003C0880913C08082E000C990B04962C2FE3
:10D9D0000C2E000C330B8217930724F48CEF8C0F62
:10D9E00080933C0830903C08D0E054E6452E512C02
:10D9F000612C712C64E2C62E67E5D62E75EFA72E3A
:10DA000078E6B72EECE08E2EE9E69E2E31101DC092
:10DA100080915008811106C080913201882309F459
:10DA2000D7C109C0C111F8CF0E94579B8091700ADD
:10DA3000882391F3EEC281E0C11180E024E04DE043
:10DA400057E16D2F0E9425C8C3C181E0381236C04E
:10DA500080915008811106C080913201882309F419
:10DA6000B7C11DC0C130C1F7C0934E0810924A081B
:10DA700010924B0810924C0810924D0804EE16EBD1
:10DA800024E031E040E050E063EE7DE086E097E1A5
:10DA90000E943DD48091700A8823F1F2BAC280912D
:10DAA000E30D9091E40D0E94CBC79C0181E0C13051
:10DAB00009F080E000E04FEF56E187C192E03912B3
:10DAC00037C080915008811106C0809132018823AF
:10DAD00009F47EC11EC0C230C1F781E080934E08B8
:10DAE00010924A0810924B0810924C0810924D0860
:10DAF00000EC16EB24E630E040E050E067EE7DE01D
:10DB00008BEF96E10E943DD48091700A8823E9F260
:10DB100080C28091E70D9091E80D0E94CBC79C01D7
:10DB200081E0C23009F080E000E047EF56E14DC1EE
:10DB3000A3E03A1235C080915008811106C080914F
:10DB40003201882309F444C11CC0C330C1F781E00D
:10DB500080934E0810924A0810924B0810924C087D
:10DB600010924D082FEF30E040E050E065EE7DE090
:10DB70008DEE96E10E94C2CE8091700A8823F9F260
:10DB800048C28091E50D9091E60D0E94CBC79C01A3
:10DB900081E0C33009F080E000E043EE56E115C1BA
:10DBA000B4E03B122AC080915008811105C08091D9
:10DBB0003201811111C00CC1C430C9F790913F0AE4
:10DBC00081E0892780933F0A83E08093320180912E
:10DBD000700A882361F31DC280913F0A811103C03E
:10DBE00022ED36E102C026ED36E181E0C43009F0D5
:10DBF00080E001E04AED56E1E8C025E0321241C084
:10DC000080915008811106C080913201882309F467
:10DC1000DFC014C0C530C1F7E12CF12C02E813E4D9
:10DC200020E030E0A90167E271E08BEC96E10E9410
:10DC30004BCE8091700A882339F3EBC181E08F933A
:10DC400084E08F931F921F9287E291E09F938F93BE
:10DC5000ADEBB6E1BF93AF93A4ECB6E1BF93AF9346
:10DC6000DF9381E0C53009F080E08F930E94DCD51E
:10DC70008DB79EB70C960FB6F8949EBF0FBE8DBFA2
:10DC8000A7C096E0391241C080915008811106C0AA
:10DC900080913201882309F49BC014C0C630C1F7BB
:10DCA000E12CF12C02E813E420E030E0A90163E26A
:10DCB00071E086EB96E10E944BCE8091700A88233A
:10DCC00039F3A7C181E08F9384E08F931F921F9255
:10DCD00083E291E09F938F93A8EAB6E1BF93AF935D
:10DCE000AFEAB6E1BF93AF93DF9381E0C63009F0AE
:10DCF00080E08F930E94DCD58DB79EB70C960FB64F
:10DD0000F8949EBF0FBE8DBF63C097E0391260C00C
:10DD100080915008811106C080913201882309F456
:10DD200057C047C0C730C1F70E94309B83E0809343
:10DD30003201A0EAB6E1B093DF0DA093DE0D8FE1D2
:10DD400091E09093DD0D8093DC0D1092D80D109230
:10DD5000D90D1092DA0D1092DB0D4092D40D509235
:10DD6000D50D6092D60D7092D70D20E030E048ECD2
:10DD700052E460911F0170912001809121019091E6
:10DD800022010E94A5DC0E9456E16093D00D7093A1
:10DD9000D10D8093D20D9093D30DABE7B9E5B0933D
:10DDA0003101A09330018091700A882309F4B4CF27
:10DDB00030C18FE191E00E94E6C69C0181E0C7304E
:10DDC00009F080E000E048E956E16D2F0E946CD533
:10DDD0002CEA35EC47E25EE360913B0A70913C0A25
:10DDE00080913D0A90913E0A0E94DDE06093690AAD
:10DDF00070936A0A80936B0A90936C0A2CEA35EC54
:10DE000047E25EE36091370A7091380A8091390ADF
:10DE100090913A0A0E94A5DC6093650A7093660AA5
:10DE20008093670A9093680AB8E03B1233C08091F0
:10DE30005008811106C080913201882309F4E1C0A5
:10DE40001CC0C830C1F7E12C18E1F12E0CE116E43A
:10DE500020E030E040E85FE363E37AE082E996E1C6
:10DE60000E94C8CD8EE297E59093310180933001F6
:10DE70008091700A8823F9F2CCC083E39AE00E9473
:10DE80007BC59C0181E0C83009F080E000E04CE8EF
:10DE900056E173C029E0321237C0809150088111D9
:10DEA00006C080913201882309F4ABC020C0C9307C
:10DEB000C1F7E12C18E1F12E0CE116E42AE037ED70
:10DEC00043E25CE369E67AE086E896E10E94C8CD29
:10DED000D0923101C09230019092E20D8092E10D1A
:10DEE0001092E00D8091700A8823D9F292C089E6E1
:10DEF0009AE00E947BC59C0181E0C93009F080E076
:10DF000000E040E856E139C08AE038123AC080911A
:10DF10005008811106C080913201882309F471C034
:10DF200020C0CA30C1F7E12C18E1F12E0CE116E453
:10DF300020E030E040E85FE365E67AE08AE796E1DA
:10DF40000E94C8CDD0923101C0923001B092E20D52
:10DF5000A092E10D1092E00D8091700A8823D9F211
:10DF600058C085E69AE00E947BC59C0181E0CA30DA
:10DF700009F080E000E044E756E16D2F0E946CD587
:10DF800040C09BE039121CC080915008811105C02F
:10DF9000809132018823A9F10BC0CB30C9F78DE8FD
:10DFA0009CE60E945C5F8091700A882389F331C0EF
:10DFB00081E0CB3009F080E023E043E656E11EC06B
:10DFC000ACE03A121EC080915008811105C08091CA
:10DFD00032018823B1F00BC0CC30C9F78AE89CE647
:10DFE0000E945C5F8091700A882389F312C081E0EF
:10DFF000CC3009F080E023E042E556E16D2F0E942D
:10E0000025C8DF5F3394D53009F000CD8DE08093D3
:10E010006D0ADF91CF911F910F91FF90EF90DF90EC
:10E02000CF90BF90AF909F908F907F906F905F90B8
:10E030004F903F9008958F929F92AF92BF92CF9250
:10E04000DF92FF920F931F93CF93DF9300D000D006
:10E0500000D0CDB7DEB710924E088091D00D9091D0
:10E06000D10DA091D20DB091D30D81309048A10572
:10E07000B10540F01092D00D1092D10D1092D20D3A
:10E080001092D30D1091D00D8091640A1816DCF413
:10E09000282F082E000C330B21503109412F012E5F
:10E0A000000C550B4217530774F01FEF180F812F08
:10E0B00090E0A0E0B0E08093D00D9093D10DA093BC
:10E0C000D20DB093D30D1092700A80913C081817AE
:10E0D00014F410933C0880913C08082E000C990B16
:10E0E0000496212F012E000C330B8217930724F482
:10E0F0008CEF810F80933C08F0903C0800E083E9AE
:10E10000A82E82E0B82E94E6C92ED12C2AEB822EBE
:10E1100022E0922EF1101AC080915008811106C0A1
:10E1200080913201882309F4A6C009C01111F8CFEB
:10E130000E94579B8091700A882391F3A3C081E0CD
:10E14000111180E024E04DE456E192C081E0F81224
:10E150001DC080915008811106C080913201882332
:10E1600009F489C00BC01130C1F780E99CE60E9418
:10E170005C5F8091700A882381F384C081E0113054
:10E1800009F080E023E041E456E172C022E0F2129F
:10E190001DC080915008811106C0809132018823F2
:10E1A00009F469C00BC01230C1F783EF98E80E94F0
:10E1B0005C5F8091700A882381F364C081E0123033
:10E1C00009F080E023E04AE356E152C083E0F81210
:10E1D0001DC080915008811106C0809132018823B2
:10E1E00009F449C00BC01330C1F78FE897E80E94CB
:10E1F0005C5F8091700A882381F344C081E0133012
:10E2000009F080E023E041E356E132C024E0F2125D
:10E2100032C080915008811105C08091320188235D
:10E2200051F11FC01430C9F70E94D4BDBE82AD8227
:10E23000DA82C982BE016B5F7F4FCE0101960E94D8
:10E24000A99C9C828B82DA82C982BE016D5F7F4F5E
:10E25000CE0101960E94A99C8091700A8823E9F260
:10E2600011C081E0143009F080E020E240E256E184
:10E27000602F0E9425C80F5FF394053009F04ACF44
:10E280000093640A26960FB6F894DEBF0FBECDBF8A
:10E29000DF91CF911F910F91FF90DF90CF90BF90B2
:10E2A000AF909F908F9008951F93CF93DF9310921C
:10E2B0004E088091D00D9091D10DA091D20DB091CA
:10E2C000D30D81309048A105B10540F01092D00DDA
:10E2D0001092D10D1092D20D1092D30DC091D00D8D
:10E2E0008091790A18160CF5282F082E000C330B94
:10E2F000255031094C2F0C2E000C550B421753079B
:10E30000A4F085301CF0CBEFC80F01C0C0E08C2F0B
:10E310000C2E000C990BAA0BBB0B8093D00D909385
:10E32000D10DA093D20DB093D30DC0933C08D0E093
:10E3300012E0C11109C0809132018823D9F121E096
:10E3400041E067EA79E115C0C13049F480913201BA
:10E35000882381F120E041E06EE979E10AC0C23012
:10E3600061F480913201882329F120E041E060E9E5
:10E3700079E18D2F0E945DD31DC0C33049F4809197
:10E3800032018823B9F020E041E06EE879E1F1CF75
:10E39000C43081F480913201882351F021E040E0C3
:10E3A00063E879E18D2F0E945DD38D2F0E94F8D50F
:10E3B00010933201DF5FCF5FD53009F0BACFD09331
:10E3C000790ADF91CF911F9108951F93CF93DF9327
:10E3D00010924E088091D00D9091D10DA091D20D48
:10E3E000B091D30D81309048A105B10540F0109255
:10E3F000D00D1092D10D1092D20D1092D30DC0916C
:10E40000D00D8091780A18160CF5282F082E000CD4
:10E41000330B255031094C2F0C2E000C550B421795
:10E420005307A4F085301CF0CBEFC80F01C0C0E04B
:10E430008C2F0C2E000C990BAA0BBB0B8093D00DCC
:10E440009093D10DA093D20DB093D30DC0933C08FF
:10E45000D0E012E0C11109C0809132018823D9F1C6
:10E4600021E041E066E779E115C0C13049F48091CF
:10E470003201882381F120E041E066E679E10AC0BB
:10E48000C23061F480913201882329F120E041E01B
:10E4900065E579E18D2F0E945DD31DC0C33049F43D
:10E4A000809132018823B9F020E041E066E479E10F
:10E4B000F1CFC43081F480913201882351F021E002
:10E4C00040E06BE379E18D2F0E945DD38D2F0E9498
:10E4D000F8D510933201DF5FCF5FD53009F0BACFA6
:10E4E000D093780ADF91CF911F9108951F93CF9316
:10E4F000DF9310924E088091D00D9091D10DA09194
:10E50000D20DB091D30D81309048A105B10540F0F6
:10E510001092D00D1092D10D1092D20D1092D30DF9
:10E52000C091D00D8091770A18160CF5282F082E6F
:10E53000000C330B255031094C2F0C2E000C550BC1
:10E5400042175307A4F085301CF0CBEFC80F01C071
:10E55000C0E08C2F0C2E000C990BAA0BBB0B8093E8
:10E56000D00D9093D10DA093D20DB093D30DC09345
:10E570003C08D0E012E0C11109C08091320188232B
:10E58000D9F121E041E06EE279E115C0C13049F4F2
:10E5900080913201882381F120E041E06EE179E150
:10E5A0000AC0C23061F480913201882329F120E051
:10E5B00041E061E179E18D2F0E945DD31DC0C33040
:10E5C00049F4809132018823B9F020E041E06FE006
:10E5D00079E1F1CFC43081F480913201882351F088
:10E5E00021E040E064E079E18D2F0E945DD38D2F22
:10E5F0000E94F8D510933201DF5FCF5FD53009F06C
:10E60000BACFD093770ADF91CF911F9108951F93CE
:10E61000CF93DF9310924E088091D00D9091D10D41
:10E62000A091D20DB091D30D81309048A105B105D4
:10E6300040F01092D00D1092D10D1092D20D109288
:10E64000D30DC091D00D8091760A18160CF5282FA5
:10E65000082E000C330B255031094C2F0C2E000CCA
:10E66000550B42175307A4F085301CF0CBEFC80FB1
:10E6700001C0C0E08C2F0C2E000C990BAA0BBB0B19
:10E680008093D00D9093D10DA093D20DB093D30D64
:10E69000C0933C08D0E012E0C11109C08091320162
:10E6A0008823D9F121E041E067EF78E115C0C1305E
:10E6B00049F480913201882381F120E041E068EE45
:10E6C00078E10AC0C23061F480913201882329F1D7
:10E6D00020E041E069ED78E18D2F0E945DD31DC0FF
:10E6E000C33049F4809132018823B9F020E041E041
:10E6F00067ED78E1F1CFC43081F480913201882355
:10E7000051F021E040E06CEC78E18D2F0E945DD368
:10E710008D2F0E94F8D510933201DF5FCF5FD53087
:10E7200009F0BACFD093760ADF91CF911F91089567
:10E730001F93CF93DF9310924E088091D00D90914C
:10E74000D10DA091D20DB091D30D81309048A1058B
:10E75000B10540F01092D00D1092D10D1092D20D53
:10E760001092D30DC091D00D8091750A18160CF53A
:10E77000282F082E000C330B255031094C2F0C2E5E
:10E78000000C550B42175307A4F085301CF0CBEF5B
:10E79000C80F01C0C0E08C2F0C2E000C990BAA0BE7
:10E7A000BB0B8093D00D9093D10DA093D20DB0935D
:10E7B000D30DC0933C08D0E012E0C11109C0809194
:10E7C00032018823D9F121E041E06FEB78E115C0F7
:10E7D000C13049F480913201882381F120E041E089
:10E7E00066EB78E10AC0C23061F48091320188237F
:10E7F00029F120E041E066EA78E18D2F0E945DD3A7
:10E800001DC0C33049F4809132018823B9F020E063
:10E8100041E064EA78E1F1CFC43081F480913201C3
:10E82000882351F021E040E069E978E18D2F0E94D2
:10E830005DD38D2F0E94F8D510933201DF5FCF5F3B
:10E84000D53009F0BACFD093750ADF91CF911F91DF
:10E8500008951F93CF93DF9310924E088091D00DAF
:10E860009091D10DA091D20DB091D30D81309048EF
:10E87000A105B10540F01092D00D1092D10D10926B
:10E88000D20D1092D30DC091D00D8091740A18163C
:10E890000CF5282F082E000C330B255031094C2F76
:10E8A0000C2E000C550B42175307A4F085301CF0BA
:10E8B000CBEFC80F01C0C0E08C2F0C2E000C990BC1
:10E8C000AA0BBB0B8093D00D9093D10DA093D20DCA
:10E8D000B093D30DC0933C08D0E012E0C11109C041
:10E8E000809132018823D9F121E041E06CE878E1A0
:10E8F00015C0C13049F480913201882381F120E0B4
:10E9000041E06DE778E10AC0C23061F480913201E4
:10E91000882329F120E041E06DE678E18D2F0E9407
:10E920005DD31DC0C33049F4809132018823B9F012
:10E9300020E041E066E678E1F1CFC43081F48091D7
:10E940003201882351F021E040E06BE578E18D2F22
:10E950000E945DD38D2F0E94F8D510933201DF5FA6
:10E96000CF5FD53009F0BACFD093740ADF91CF9141
:10E970001F910895CF92DF92EF92FF921F93CF9352
:10E98000DF9310924E088091D00D9091D10DA091FF
:10E99000D20DB091D30D81309048A105B10540F062
:10E9A0001092D00D1092D10D1092D20D1092D30D65
:10E9B000C091D00D8091730A1816DCF4282F082E10
:10E9C000000C330B215031094C2F0C2E000C550B31
:10E9D0004217530774F0CFEFC80F8C2F90E0A0E0E0
:10E9E000B0E08093D00D9093D10DA093D20DB09351
:10E9F000D30D1092700A80913C08C81714F4C0938C
:10EA00003C0880913C08082E000C990B04962C2F92
:10EA10000C2E000C330B8217930724F48CEF8C0F11
:10EA200080933C0810913C08D0E081E0EE24E39410
:10EA3000F12C22E0C22ED12C111125C08823B1F077
:10EA40001C16A4F08091D00D9091D10DA091D20D03
:10EA5000B091D30D0196A11DB11D8093D00D90935F
:10EA6000D10DA093D20DB093D30DCF5F8091320121
:10EA7000882309F446C020E041E06BE478E18D2F63
:10EA80000E945DD33EC01130E1F4809150088111A5
:10EA900005C0809132018823A1F10BC0C130C9F7B4
:10EAA000D0923E08C0923D088091700A882389F375
:10EAB00031C081E0C13009F080E020E24EE358E14E
:10EAC0001DC01230F1F480915008811105C0809171
:10EAD00032018823B1F00BC0C230C9F7F0923E0872
:10EAE000E0923D088091700A882389F313C081E089
:10EAF000C23009F080E020E241E358E16D2F0E942E
:10EB000025C8DF5F1F5F80E0D53009F095CF83E037
:10EB10008093730ADF91CF911F91FF90EF90DF9068
:10EB2000CF9008950F931F93CF93DF9310924E08C9
:10EB30008091D00D9091D10DA091D20DB091D30DB7
:10EB400081309048A105B10540F01092D00D10928F
:10EB5000D10D1092D20D1092D30DC091D00D809195
:10EB6000720A1816DCF4282F082E000C330B2150E3
:10EB700031094C2F0C2E000C550B4217530774F023
:10EB8000CFEFC80F8C2F90E0A0E0B0E08093D00DC5
:10EB90009093D10DA093D20DB093D30D1092700A23
:10EBA00080913C08C81714F4C0933C0880913C083D
:10EBB000082E000C990B04962C2F0C2E000C330BF6
:10EBC0008217930724F48CEF8C0F80933C081091EC
:10EBD0003C08D0E081E002E0111122C08823B1F0AE
:10EBE0001C16A4F08091D00D9091D10DA091D20D62
:10EBF000B091D30D0196A11DB11D8093D00D9093BE
:10EC0000D10DA093D20DB093D30DCF5F809132017F
:10EC1000882309F468C021E041E062E278E14DC058
:10EC2000113011F58823B1F0C230A4F48091D00DD9
:10EC30009091D10DA091D20DB091D30D0196A11D4F
:10EC4000B11D8093D00D9093D10DA093D20DB093B0
:10EC5000D30DCF5F80913201882309F444C020E0B6
:10EC600040E06DE078E129C01230E9F4809150086D
:10EC7000811105C0809132018823A9F109C0C230F9
:10EC8000C9F70E94579B8091700A882399F333C07B
:10EC900081E0C23009F080E024E048E058E16D2FC7
:10ECA0000E9425C820C0133061F48091320188236E
:10ECB000D1F020E041E066E078E18D2F0E945DD345
:10ECC00012C0143081F480913201882351F021E088
:10ECD00040E06BEF77E18D2F0E945DD38D2F0E9476
:10ECE000F8D500933201DF5F1F5F80E0D53009F077
:10ECF00073CFD093720ADF91CF911F910F91089536
:10ED0000AF92BF92CF92DF92EF92FF920F931F9339
:10ED1000CF93DF93CDB7DEB76F970FB6F894DEBF12
:10ED20000FBECDBF83E49FE09093420F8093410FCD
:10ED300081E090E090937B1180937A1110927D1185
:10ED400010927C1140E050E0BA0187E49FE00E94FD
:10ED50001DC28091410F9091420F2BE1FC0134962E
:10ED6000DE01159601900D922A95E1F7FC01828152
:10ED700093819C838B8381EC91E09A83898340E02B
:10ED800050E0BE016F5F7F4F8AE592E00E94E77F0F
:10ED9000CE0101960E94AF7AA0907C11B0907D11B7
:10EDA00010924E088091D00D9091D10DA091D20D6E
:10EDB000B091D30D81309048A105B10540F010927B
:10EDC000D00D1092D10D1092D20D1092D30D109142
:10EDD000D00D8091710A1816DCF4282F082E000C33
:10EDE000330B21503109412F012E000C550B4217D6
:10EDF000530774F01FEF180F812F90E0A0E0B0E0F0
:10EE00008093D00D9093D10DA093D20DB093D30DDC
:10EE10001092700A80913C08181714F410933C0863
:10EE200080913C08082E000C990B0496212F012E8E
:10EE3000000C330B8217930724F48CEF810F80931F
:10EE40003C0800913C08F12C21E0A21AB108011104
:10EE50001BC080915008811105C080913201882328
:10EE600099F009C01111F9CF0E94579B8091700A47
:10EE7000882399F35EC181E0111180E024E046EF20
:10EE800057E16F2D0E9425C868EF7EE087E49FE080
:10EE90000E94A0A58091F80E8F3231F50130F1F477
:10EEA00080915008811105C0809132018823B1F012
:10EEB0000BC01130C9F70E94CB9B10923C08809187
:10EEC000700A882389F335C181E0113009F080E0B0
:10EED00020E24DEE57E16F2D0E9425C8650192E0BA
:10EEE000EE24E394E00E87C00130C1F78091500812
:10EEF000882309F43FC01130E9F5809198108823E8
:10EF000019F1815080939810882361F090E0019767
:10EF10004FE1489F9001499F300D1124C9018E593E
:10EF2000904F02C082E29FE02BE1FC013496A7E4FF
:10EF3000BFE001900D922A95E1F7FC018281938157
:10EF40009093460F8093450F81E090E0A0E0B0E001
:10EF500020919810211103C080E090E0DC018093A3
:10EF6000D00D9093D10DA093D20DB093D30D1092EC
:10EF70003C0822C080913201882309F4AFCF81E0A0
:10EF8000113009F080E020E249EE57E1A4CF8AE099
:10EF90000E94553CCE0101960E94AF7A10923C0827
:10EFA00082E090E0A0E0B0E08093D00D9093D10D8E
:10EFB000A093D20DB093D30D81E08093700A83E0CB
:10EFC00080933201B6C00913ABC060E070E0C601A7
:10EFD0000E94D3819091F70E80915008992309F4F3
:10EFE00082C081110DC080913201811177C09E2DA8
:10EFF00021E0C21AD1084FEFC416D40621F792C0FF
:10F000001013F1CF1D8218861C821B8281EC91E0C7
:10F010009A83898380914A0F882319F063E47FE003
:10F0200002C062E27FE06C5F7F4F21E048EF5EE06C
:10F03000CE0105960E948CA9811124C0E3E5FCE174
:10F0400084918F010F5F1F4F882321F00E94553C50
:10F05000F801F6CFE3EDF7E184918F010F5F1F4FC9
:10F06000811103C008EF1EE004C00E94553CF80166
:10F07000F3CFF80181918F01882309F488CF0E9492
:10F08000553CF7CF8BE1FE013596A7E4BFE0019038
:10F090000D928A95E1F72B813C813093460F2093A6
:10F0A000450F809198108A3008F074CF91E0980F46
:10F0B00090939810FFE18F9FC0011124DC01AA59A1
:10F0C000B04F4BE1E7E4FFE001900D924A95E1F784
:10F0D000FC01EE59F04F338322835CCF81E01013A3
:10F0E00080E041E019C0811106C08091320188237F
:10F0F00009F47DCF0DC01013F8CF88EF9EE00E9479
:10F100005E840E94509B8091700A882371F311C025
:10F1100081E0101380E040E06F2D0E94429F67CF96
:10F120009F5F66CFF3940F5F85E0F81290CE9093C7
:10F13000710A6F960FB6F894DEBF0FBECDBFDF9198
:10F14000CF911F910F91FF90EF90DF90CF90BF90E4
:10F15000AF90089561E0FC0180810C9457608EBDF2
:10F160000DB407FEFDCF08958FEF8EBD0DB407FEE1
:10F17000FDCF8EB50895CF92DF92EF92FF921F934D
:10F18000CF93DF9300D000D0CDB7DEB76C01162F40
:10F19000FC019281892F806A86958CBD90FD03C009
:10F1A00081E0963009F480E08DBD60E0F601808159
:10F1B00029833A834B835C830E9457606CE271E041
:10F1C000C6010E94FEA6812F80640E94AF7888E16C
:10F1D000E82EF12C5C814B813A812981DA01C90149
:10F1E0000E2C04C0B695A795979587950A94D2F7EB
:10F1F00029833A834B835C830E94AF78F8E0EF1A4F
:10F20000F10829813A814B815C8188EFE8168FEF04
:10F21000F80621F7112321F0183021F08FEF03C0F9
:10F2200085E901C087E80E94AF781C3011F40E9484
:10F23000B47810E00E94B478F601838387FF04C09D
:10F240001F3F11F01F5FF6CF0F900F900F900F90A0
:10F25000DF91CF911F91FF90EF90DF90CF900895B5
:10F26000EF92FF920F931F93CF93DF93EC017901FD
:10F270008C81833039F089E0440F551F661F771F5A
:10F280008A95D1F79A01AB0161E1CE010E94BB786A
:10F29000882331F084E08983CE010E94AA783CC0A3
:10F2A0000E94F3528B010E94B4788B838F3F49F404
:10F2B0000E94F352601B710B6D327140A0F381E12B
:10F2C00003C08E3F49F08FE08983CE010E94AA7867
:10F2D0008FEF0E94AF7820C08FEF8EBDF701D7016E
:10F2E000A150BE4F0DB407FEFDCF9EB591938EBDCC
:10F2F000EA17FB07B9F70DB407FEFDCF8EB58C9367
:10F300000E94B4780E94B478CE010E94AA788FEF50
:10F310000E94AF7881E001C080E0DF91CF911F9122
:10F320000F91FF90EF9008954F925F926F927F92AE
:10F330008F929F92AF92BF92EF92FF920F931F9383
:10F34000CF93DF937C01FC01EA51F54E6491EC010F
:10F35000CC0FDD1FCC0FDD1FFE01E652F54E4590B0
:10F36000559065907490062E000C770B880B990BC6
:10F370000E9446DC4B015C0120E030E040EC5FE3A2
:10F38000C301B2010E94A5DCA50194010E94A5DC85
:10F39000AB01BC0100E010E09801C7010E94183ADF
:10F3A000FE01E253F54E2591359145915491C501E9
:10F3B000B4010E94A5DC4B015C0120E030E0A90112
:10F3C0000E943FDC882309F44BC000E010E0980164
:10F3D000B501A4017058C7010E94183AF701E5531E
:10F3E000F54E649161111BC0E3E5FCE184913F019E
:10F3F0009FEF691A790A882321F00E94553CF30196
:10F40000F5CFE9EAFAE184913F019FEF691A790AA1
:10F41000882321F00E94553CF301F5CF6AE0FE01FC
:10F42000E756F54E459055906590749070E080E0F9
:10F4300090E00E9446DC9B01AC01C301B2010E9436
:10F44000DDE02B013C01A5019401C501B4010E943E
:10F450005AE0AB01BC0193018201C7010E94183A36
:10F46000F701ED5DF14F81E08083F701E659F74F39
:10F470008083FE01E55FF44F1082118212821382B5
:10F48000C7010E945039FE01E357F54E85919591D1
:10F49000A591B4918E010D5F114FF8018083918386
:10F4A000A283B3830E940E3AC95ED44FF8018081D3
:10F4B0009181A281B38188839983AA83BB83DF91E1
:10F4C000CF911F910F91FF90EF90BF90AF909F90C1
:10F4D0008F907F906F905F904F9008950F931F9340
:10F4E000CF93DF938C01E3E5FCE18491EF0121965A
:10F4F000882321F00E94553CFE01F7CFB80180E837
:10F500009AE10E94ABC982E20E94553C8AE00E94C7
:10F51000553C81E0DF91CF911F910F91089580912B
:10F520005A0E81111AC060913C0170913D01072E65
:10F53000000C880B990B0E9446DC9B01AC0160918A
:10F54000560E7091570E8091580E9091590E0E9450
:10F550003FDC881F8827881F089580E0089521ECEC
:10F5600031E0FC013183208304960C949B3B5E9A2E
:10F57000EAE6F8E010825E9A1182159A12825E9A8B
:10F5800008958C01E8E3FCE18491EF012196882342
:10F5900021F00E94553CFE01F7CFE0E6FAE18491AC
:10F5A000EF012196882321F00E94553CFE01F7CF00
:10F5B0000E946F450E94B77A0E94315F61E0C801E6
:10F5C0000E94DEC80E94509B0E9462BC84E00E94A0
:10F5D00077A08091660E8695869510929C0E8093FA
:10F5E0009D0E0E9452BC8091660E86958695880F6E
:10F5F00010929C0E80939D0E81E59AE10E94C0A01E
:10F600008091660E86958695982F990F890F109296
:10F610009C0E80939D0E84E49AE10E94C0A00E94FB
:10F62000C0BB8111D3CF2FEF8BE49DE121508040EF
:10F630009040E1F700C00000F8942FEF84E39CE0D5
:10F64000215080409040E1F700C000000E946F45CB
:10F65000A895FECF4F925F926F927F928F929F926A
:10F66000AF92BF92CF92DF92EF92FF920F931F93D0
:10F67000CF93DF93082F0E94585C0E94F3526B01D6
:10F680007C0110912B01112309F465C08091270B97
:10F690009091280B009709F45EC040912A0B50917D
:10F6A0002B0B60912C0B70912D0B46015701841A86
:10F6B000950AA60AB70AB7FC60C08330910509F124
:10F6C00034F401970CF447C0E3E5FCE106C004976D
:10F6D00009F041C0E3E5FCE12AC08491EF012196E5
:10F6E000882321F00E94553CFE01F7CFEFEEF9E1AF
:10F6F0008491EF012196882371F10E94553CFE010F
:10F70000F7CFE3E5FCE18491EF012196882321F016
:10F710000E94553CFE01F7CFE8EDF9E18491EF013D
:10F7200021968823C1F00E94553CFE01F7CF8491B9
:10F73000EF012196882321F00E94553CFE01F7CF6E
:10F74000E0ECF9E18491EF012196882321F00E94F9
:10F75000553CFE01F7CF212F30E0A8EEB3E00E9428
:10F760004AE0C60ED71EE81EF91EC0922A0BD092A0
:10F770002B0BE0922C0BF0922D0BC091000BCC23A5
:10F7800091F00E94F352C090FC0AD090FD0AE090E4
:10F79000FE0AF090FF0ADC01CB018C199D09AE092D
:10F7A000BF09B7FFA0C180911B0A843010F40E94EA
:10F7B000D73D0E94F3528090070B9090080BA090C9
:10F7C000090BB0900A0B81149104A104B10471F1EA
:10F7D000C090030BD090040BE090050BF090060B4B
:10F7E000C80CD91CEA1CFB1C9B01AC012C193D095F
:10F7F0004E095F0957FD1AC0E8E3FCE18491EF016F
:10F800002196882321F00E94553CFE01F7CF60919C
:10F81000010B7091020B8AE09AE10E94ABC98AE069
:10F820000E94553C81E09AE10E94C17A2091290B07
:10F83000211128C080902C0190902D01A0902E01C4
:10F84000B0902F0181149104A104B104D9F0C090AB
:10F85000030BD090040BE090050BF090060BC80C46
:10F86000D91CEA1CFB1CDC01CB018C199D09AE09DB
:10F87000BF09B7FD07C0011105C00E94A13B882345
:10F8800009F44FC10E94A13B882391F0E091C40E7E
:10F890003DE4E39FF0011124E75BFC4F6081809120
:10F8A000C40E9091C30E891729F08F5F8F70F9CF26
:10F8B0006091E50D70E084E00E94475280913F0A1C
:10F8C000882309F4FAC00091270110912801D091F2
:10F8D0002901C0912A016091E30D7091E40D6E5FE2
:10F8E0007F4F072E000C880B990B0E9446DC980175
:10F8F0004D2F5C2F0E943FDC87FDDFC0F090C40ECF
:10F90000912CA12CB12CE12C8DE4882E8091C30E7A
:10F91000F81609F45CC08F2D90E0889EF001899E56
:10F92000F00D1124EE5FFC4F42815381648175819B
:10F93000452B462B472B81F4468157816085718585
:10F94000452B462B472B41F44285538564857585AD
:10F95000452B462B472BB1F1889E9001899E300D97
:10F960001124A9014E5F5C4F6A01FA016685778513
:10F97000808991890E9446DC2B013C01F601628955
:10F980007389848995890E9444DC9B01AC01C30181
:10F99000B2010E94DDE0F60123A134A145A156A1E8
:10F9A0000E94A5DC3B016C019B01AC01692D7A2D05
:10F9B0008B2D9E2D0E943FDC87FF04C0962CA72C28
:10F9C000BC2CED2C81E08F0D8F70F82E9FCF2091F5
:10F9D0001F01309120014091210150912201692D98
:10F9E0007A2D8B2D9E2D0E94A5DC9B01AC01B801C8
:10F9F0008D2F9C2F0E945AE06B017C0198014D2FA6
:10FA00005C2F0E943FDC87FD14C000912301109100
:10FA10002401D0912501C091260198014D2F5C2F22
:10FA2000B601C7010E94DDE118161CF08601DE2D2B
:10FA3000CF2DC0902E0BD0902F0BE090300BF0907C
:10FA4000310BA7019601B8018D2F9C2F0E943FDC3E
:10FA500087FF1CC020E037ED43EA5CE3B8018D2F3F
:10FA60009C2F0E94A5DC4B015C0128E431EE4AE7A3
:10FA70005FE3C701B6010E94A5DC9B01AC01C50193
:10FA8000B4010E945AE08B01D82FC92FC801AD2FB5
:10FA9000BC2F80932E0B90932F0BA093300BB09321
:10FAA000310BB8018D2F9C2F0E944FE17093E40D14
:10FAB0006093E30D80E00E9424450E94BF4687ECDE
:10FAC0009EE0DF91CF911F910F91FF90EF90DF901B
:10FAD000CF90BF90AF909F908F907F906F905F90EE
:10FAE0004F900C940B370E94F3526B017C012C2F2A
:10FAF00030E0A8EEB3E00E944AE0DC01CB018C0DBF
:10FB00009D1DAE1DBF1D8093FC0A9093FD0AA0931E
:10FB1000FE0AB093FF0A0E9431A28AE00E94553C7F
:10FB200042CE5E9A10926A085E9A10926B08159AFD
:10FB300010926C085E9AA6CE8F929F92AF92BF925F
:10FB4000CF92DF92FF920F931F93CF93DF931F9279
:10FB5000CDB7DEB74C016B015A01122F8091510EC7
:10FB600083FD36C020E030E0A901F501608171819C
:10FB7000828193810E943FDC882351F1F0905A0EDC
:10FB8000F11024C02091E30D3091E40D80913C01EF
:10FB900090913D0128173907CCF4E8E3FCE184910A
:10FBA0008F010F5F1F4F882321F00E94553CF80101
:10FBB000F6CFE9EEFAE184918F010F5F1F4F8823A2
:10FBC00009F49BC00E94553CF801F5CF0E946D37A7
:10FBD00091E09093290B8091F50E882321F01092EB
:10FBE000F50E9093420B0E94149E002321F080E0BA
:10FBF00090E00E94705F0E94204890E1E3E0FEE008
:10FC0000A2E3BBE001900D929A95E1F720E030E08D
:10FC1000A901F40160817181828193810E943FDC9E
:10FC2000882329F00E948F7A882309F45EC080918E
:10FC3000030E9091040EA091050EB091060EF601F0
:10FC400080839183A283B3838091070E9091080EE5
:10FC5000A091090EB0910A0E84839583A683B78381
:10FC600082E08983B601CE0101960E94259120E0B1
:10FC700030E0A901F50160817181828193810E9448
:10FC80003FDC882381F0002339F081E090E00E947E
:10FC9000705F80E00E942A7B40E050E060EA71E4FF
:10FCA000C5010E94133C002321F082E090E00E94F5
:10FCB000705F61E0812F0E94C53780E00E942A7B3F
:10FCC0000E94F352DC01CB0188539045AF4FBF4FE8
:10FCD0008093D6079093D707A093D807B093D907FE
:10FCE00010925E0EFF24F39408C040E050E060E202
:10FCF00071E4C4010E94133C9ACF8F2D0F90DF91C5
:10FD0000CF911F910F91FF90DF90CF90BF90AF9058
:10FD10009F908F900895AF92BF92CF92DF92EF9213
:10FD2000FF920F931F93CF93DF9300D000D0CDB7F6
:10FD3000DEB77C016B01042F10915E0E1092D60786
:10FD40001092D7071092D8071092D90710925E0E22
:10FD500080E00E94244511110E946D3761E0802FE0
:10FD60000E94C5370E94093C20E030E0A901F7015C
:10FD700060817181828193810E943FDC882371F1CF
:10FD8000112321F082E090E00E94705F83E090E018
:10FD90009093280B8093270B81E0809351088091EA
:10FDA0005108882351F0112341F060E0802F0E9418
:10FDB000C53781E00E942A7BF2CF81E090E09093EA
:10FDC000280B8093270B83E090E00E94705F40E057
:10FDD00050E068EC71E4C7010E94133C0E948F7AE6
:10FDE000811149C0F60180819181A281B38189830B
:10FDF0009A83AB83BC8383E0A82EB12C01E010E092
:10FE0000C12CD12C98ECE92E92E4F92E20E030E0C0
:10FE1000A90169817A818B819C810E94DDE118169C
:10FE200064F484E090E00E94705F40E050E060EA9B
:10FE300070E4CE0101960E94133CB092280BA09270
:10FE4000270B1092510885E090E00E94705F80912E
:10FE50003D0890913E08009721F481E00E942A7BA2
:10FE6000F6CF1093280B0093270BC982DA82EB821E
:10FE7000FC82019759F286E090E00E94705F8091C9
:10FE80003E0B90913F0BA091400BB091410B8093A2
:10FE90000F0E9093100EA093110EB093120E80933C
:10FEA000230B9093240BA093250BB093260B0E9459
:10FEB000D69D80E090E0A8ECB2E489839A83AB837E
:10FEC000BC839E012F5F3F4F4BE05EE066E37BE02B
:10FED00082E39BE00E943B3880E090E0A0EAB0E43F
:10FEE00089839A83AB83BC83BE016F5F7F4F8AE3B4
:10FEF0009BE00E94223987E090E00E94705F809131
:10FF0000420B882349F08091F60E882319F081E096
:10FF10008093F50E1092420B1092290B0F900F90C8
:10FF20000F900F90DF91CF911F910F91FF90EF9065
:10FF3000DF90CF90BF90AF900895CF93DF930E9452
:10FF40004A3CE0911A0AF0E0E758F74F8081882395
:10FF500081F0EDEBF9E18491EF012196882321F006
:10FF60000E94553CFE01F7CF8AE0DF91CF910C94BF
:10FF7000553CDF91CF910895CF93DF938FB7F894DD
:10FF80009091FB0A9093FA0A8FBFE4EBF9E1849118
:10FF9000EF012196882321F00E94553CFE01F7CF06
:10FFA0008091290E90912A0EA0912B0EB0912C0ECB
:10FFB000BC01CD016F5F7F4F8F4F9F4F0E941E414D
:10FFC0008AE00E94553CDF91CF910C949D7F2F9247
:10FFD0003F924F925F926F927F928F929F92AF92D9
:10FFE000BF92CF92DF92EF92FF920F931F93CF9326
:10FFF000DF93CDB7DEB7C257D1090FB6F894DEBF95
:020000021000EC
:100000000FBECDBF7C015B014A012DB73EB7AF9655
:100010003FAF2EAFAF97AD961FAEAD972B0134E03B
:10002000430E511C8E01015A1F4F91EC692E91E035
:10003000792E80E490E08C0F9D1F0496E1969FAF8F
:100040008EAFE197F5018781823008F489C18485FC
:100050009585A685B7858F719927AA27BB27892BF8
:100060008A2B8B2B09F07CC125E03FE0232B11F07C
:100070001092050F45E05FE0BE016F5F7F4FC20148
:100080000E9478C118160CF06BC18C85482F4871FE
:10009000403109F0DBC020917A1130917B11215061
:1000A00031092230310508F4D1C02DB63EB6BE016B
:1000B0006F5F7F4FC8010E946FBF81E0F7019081A1
:1000C0009111BCC0E1E0F0E0D8010D900020E9F70B
:1000D000E01BF10BEA0FFB1F31962DB73EB72E1B2D
:1000E0003F0B0FB6F8943EBF0FBE2DBFEDB7FEB766
:1000F00031966F01811102C0B70102C063E772E05F
:10010000C6010E940FE3B801C6010E94F0E263E756
:1001100072E0C6010E94F0E225961FAE2597289650
:100120001FAE289724961FAE1EAE249722967FAE50
:100130006EAE229721E0A801B201E1968EAD9FAD8F
:10014000E1970E948CA9811150C080917A11909101
:100150007B11892B09F049C0E3E5FCE184919F0103
:100160002F5F3F4F882381F0E2962FAFE297E3960F
:100170003FAFE3970E94553CE2962FADE297E3969E
:100180003FADE397F901EACFEFE3FCE184919F01F2
:100190002F5F3F4F811102C0980110C0E2962FAF30
:1001A000E297E3963FAFE3970E94553CE2962FAD6E
:1001B000E297E3963FADE397F901E8CFF90181912A
:1001C0009F01882379F0E2962FAFE297E3963FAF45
:1001D000E3970E94553CE3963FADE397E2962FAD3F
:1001E000E297ECCF8AE00E94553C8BE1FE01EC5B8C
:1001F000FF4FDE01959601900D928A95E1F72496C6
:100200008EAD9FAD24979CA38BA37AA269A240E0F8
:1002100050E0BE016F5D7F4FC6010E94E77FCE01B7
:1002200081960E94AF7ACE01805C9F4F0E94AF7A88
:100230000FB6F8943EBE0FBE2DBE04CF80E00190F5
:100240000020E9F73197EE19FF093ECF99819923F4
:1002500009F486C0953E09F4F5CE9E3209F4F2CE3B
:100260009091050F9E3209F4EDCE8A7009F0EACE26
:1002700081E0403109F080E08093F70E811108C0E1
:100280008985873409F0DECE8A858E3709F4DACE87
:1002900080917A1190917B118130910579F08230B3
:1002A0009105C1F1892B09F0CDCEBE016F5F7F4F63
:1002B00088EF9EE00E946FBF67010AC080917C11A9
:1002C00090917D11019690937D1180937C11BACE0F
:1002D000F60181916F01882319F00E94553CF8CFF7
:1002E00088EFC82E8EE0D82EF60181916F01882309
:1002F00019F00E94553CF8CF80E20E94553C6D8D6C
:100300007E8D8F8D98A14AE00E9474408AE00E9401
:10031000553C98CEBE016F5F7F4F88EF9EE00E94F4
:100320006FBF8114910441F068EF7EE0C4010E9428
:10033000DDE2892B69F414C0AD963FADAD97832FF4
:1003400090E02091500D3091510D8217930741F0AC
:10035000AD963FADAD973F5FAD963FAFAD9772CED7
:10036000AF968EAD9FADAF970FB6F8949EBF0FBE00
:100370008DBFCE58DF4F0FB6F894DEBF0FBECDBF96
:10038000DF91CF911F910F91FF90EF90DF90CF9071
:10039000BF90AF909F908F907F906F905F904F90A5
:1003A0003F902F900895EF92FF920F931F93CF935A
:1003B000DF93CDB7DEB76F970FB6F894DEBF0FBEF1
:1003C000CDBF7B0101E41FE023E43FE0F80131836E
:1003D000208322E030E030937B1120937A119093B8
:1003E000510D8093500D40E050E0BA0187E49FE04A
:1003F0000E941DC2F801808191812BE1FC0134969D
:10040000DE01159601900D922A95E1F7FC0182819B
:1004100093819C838B8381EC91E09A838983A701EC
:10042000BE016F5F7F4F8AE592E00E94E77FCE01B9
:1004300001960E94AF7A6F960FB6F894DEBF0FBE9A
:10044000CDBFDF91CF911F910F91FF90EF90089555
:100450006F927F928F929F92AF92BF92DF92EF92B4
:10046000FF920F931F93CF93DF93CDB7DEB7AE9775
:100470000FB6F894DEBF0FBECDBF2091F60E22233B
:1004800009F408C2D62E7C018091C310882309F498
:10049000A5C0442309F4D1C18091DB10882329F140
:1004A000E8E3FCE184918F010F5F1F4F882321F067
:1004B0000E94553CF801F6CFE5EFFBE184918F01F6
:1004C0000F5F1F4F882321F00E94553CF801F6CFA3
:1004D00061E070E080E090E00E941E418AE00E94AE
:1004E000553C8CEE9BE10E94C17A81EE90E19EA783
:1004F0008DA78FE28093E01081E0898310E00FE107
:1005000080919810181778F4019FC0011124AE0152
:100510004F5F5F4FBE01635D7F4F8E59904F0E94CA
:100520003FBF1F5FEDCF898187FD0FC0AE014F5FD9
:100530005F4FBE01635D7F4F8CEB90E10E943FBF38
:100540008DA59EA501979EA78DA7EDA5FEA510825E
:10055000E091DB1084E0E89FF0011124E452FF4EAB
:100560008091711190917211A0917311B0917411D9
:1005700080839183A283B383E3E5FCE184918F01BF
:100580000F5F1F4F882321F00E94553CF801F6CFE2
:10059000B70183ED9BE10E94ABC96091DB109DE840
:1005A000699FB001112460527F4E88EC9BE10E944C
:1005B000ABC940917111509172116091731170919A
:1005C000741182EC9BE10E943BC98AE00E94553C79
:1005D0008091DB108F5F8093DB1027C04423C1F034
:1005E000E3E5FCE184918F010F5F1F4F882321F029
:1005F0000E94553CF801F6CFE2EBFBE184918F01BC
:100600000F5F1F4F882389F00E94553CF801F6CFF9
:100610001092DB1082E0B82E12C1B70189E99BE18C
:100620000E94ABC98AE00E94553C0E949CBB1D827F
:1006300018861C821B8281EC91E09A83898382E276
:100640009FE09093420F8093410FF70180818F329A
:1006500009F05CC087010F5F1F4FCE0101964C016E
:100660000115110509F458C06FE270E0C8010E943D
:10067000FBE25C01009709F450C00817190708F065
:100680004CC03C01601A710AA301B801CE018096EA
:100690000E9424E3E0E2F0E0EC0FFD1FE60DF71D01
:1006A00010826091410F7091420F6115710511F038
:1006B0006C5F7F4F21E0AE01405E5F4FCE0105963B
:1006C0000E948CA981111AC0E5E8FBE184918F0199
:1006D0000F5F1F4F811104C08E01005E1F4F04C0C9
:1006E0000E94553CF801F2CFF80181918F018823D7
:1006F00019F00E94553CF8CF8EE288C09092420FCC
:100700008092410F85010F5F1F4FAACF83E49FE0C6
:100710009093420F8093410F87019091410F8091F8
:10072000420F692F782FDD2009F45AC06115710539
:1007300011F06C5F7F4F21E0A80180EC90E10E94F6
:100740008CA9882309F448C08091D1109091D210CF
:10075000A091D310B091D41080936D1190936E112D
:10076000A0936F11B09370111092711110927211C9
:100770001092731110927411B80187E79BE10E94E7
:10078000ABC940916D1150916E1160916F117091D4
:1007900070118FE69BE10E943BC98AE00E94553CA4
:1007A000E0E6FBE184917F019FEFE91AF90A8823D3
:1007B00021F00E94553CF701F5CFB80180E090E0B0
:1007C0000E94D3818091050F882319F085E09FE076
:1007D00001C0C80160E02AC0B8018CE49BE110C0F0
:1007E0006115710511F06C5F7F4F26E5A80180EC63
:1007F00090E10E948CA981110CC0B80188E39BE1B3
:100800000E94ABC98EE20E94553C8AE00E94553C92
:100810000FC081E08093F30EB70186E29BE10E9456
:10082000ABC98AE00E94553C60E0C8010E94FDC847
:10083000CE0101960E94AF7A2DC0BB24B394E3E5AC
:10084000FCE184918F010F5F1F4F882321F00E94EC
:10085000553CF801F6CFEDEAFBE184918F010F5F83
:100860001F4F882321F00E94553CF801F6CFE1E0AC
:10087000BE1619F0E7EAFBE102C0E1EAFBE1849170
:100880008F010F5F1F4F882309F4C7CE0E94553C8C
:10089000F801F5CFAE960FB6F894DEBF0FBECDBF10
:1008A000DF91CF911F910F91FF90EF90DF90BF905C
:1008B000AF909F908F907F906F900895CF92DF922E
:1008C000EF92FF920F931F93CF93DF93CDB7DEB7D5
:1008D000EDB6FEB6DC010D900020E9F79D01281B66
:1008E000390B2C5F3F4F4DB75EB7421B530B0FB612
:1008F000F8945EBF0FBE4DBF0DB71EB70F5F1F4F01
:100900009F938F938FE19BE19F938F931F930F93FF
:100910000E94D6DB680154E0C50ED11C0F900F90E9
:100920000F900F900F900F90F6018081882349F06F
:10093000082E000C990B0E94BFE2F60181936F0113
:10094000F3CF60E0C8010E949139882319F0C801F3
:100950000E946E7A8BE19BE190934F0D80934E0D38
:100960000E94AE390FB6F894FEBE0FBEEDBEDF9109
:10097000CF911F910F91FF90EF90DF90CF9008954E
:10098000AF92BF92CF92DF92EF92FF920F931F939D
:10099000CF93DF93CDB7DEB7AA970FB6F894DEBF3B
:1009A0000FBECDBF8091210F8F938091200F8F9329
:1009B00082E19BE19F938F937E0181E2E80EF11C1F
:1009C000FF92EF920E94D6DB0F900F900F900F9046
:1009D0000F900F9010E0F70101900020E9F7319798
:1009E000EE19FF091E1784F46701C10ED11C17FD13
:1009F000DA94F6018081082E000C990B0E94BFE268
:100A0000F60180831F5FE7CF40E050E0BA0186E245
:100A10009FE00E941DC200E0CE0101966C01809112
:100A2000290F823028F4011114C08FEF9FEF16C0F8
:100A300080912E0F90912F0FA091300FB091310F18
:100A40008F719927AA27BB27892B8A2B8B2B59F7C4
:100A50001AC08091200F9091210F01969093210F41
:100A60008093200FAA960FB6F894DEBF0FBECDBFBD
:100A7000DF91CF911F910F91FF90EF90DF90CF907A
:100A8000BF90AF90089540E050E0B60186E29FE04D
:100A90000E9478C118163CF6F60101900020E9F793
:100AA00031971E2F1C19115068F05601A10EB11C70
:100AB00017FDBA94F501808190E00E94BFE2F50134
:100AC0008083F1CF8A858E3709F4A9CF45E050E0C5
:100AD000B701C6010E9416E3892B09F0A0CFC70118
:100AE0000E945E8401E09BCF4F925F926F927F9253
:100AF0008F929F92AF92BF92FF920F931F93CF93CB
:100B0000DF93182F89E990E190934D0D80934C0D60
:100B10001092B51082E090E0A0E0B0E080939E10CB
:100B200090939F10A093A010B093A11010924B0D22
:100B30001092470D1092480D1092490D10924A0DD7
:100B40008FEF9FEFDC018093430D9093440DA093B2
:100B5000450DB093460D112379F1153008F0F9C019
:100B600040E060E070E0CB010E94C5BF882309F43B
:100B7000F0C020E1129FC00111248D5C944FFC0154
:100B8000E254FE4F20812F7709F0E3C03C9640816C
:100B9000518162817381443651056105710508F404
:100BA000D8C0349780809180A280B3808114910452
:100BB000A104B10421F4CDC0812C912C540140E05A
:100BC000C501B4010E94C5BFF82E882309F4C1C035
:100BD00080914E0B90914F0B8115924009F0B9C056
:100BE000A091530BAA2309F4B4C06091510B7091EA
:100BF000520B6115710509F4ACC02091500B2223F2
:100C000009F4A7C0A093B0102093A21080E030E0B8
:100C1000E1E0F0E0C82FAF01082E02C0440F551FDD
:100C20000A94E2F72417350741F0982F8F5F983028
:100C300089F789E08093AB108CC08093AB10209132
:100C4000590B30915A0B2115310519F040E050E055
:100C500008C02091670B3091680B4091690B50914F
:100C60006A0B2093A3103093A4104093A5105093C7
:100C7000A61024013501460E571E611C711C4092BE
:100C8000B1105092B2106092B3107092B410E09113
:100C9000540BF091550BF093B710E093B610B0E001
:100CA0000E943FE0460E571E681E791E4092B81003
:100CB0005092B9106092BA107092BB1085E0EE0F9E
:100CC000FF1F8A95E1F7E150FE4FEF2FFF27E695D2
:100CD0004E0E5F1E611C711C4092AC105092AD1004
:100CE0006092AE107092AF102091560B3091570B5E
:100CF0002115310521F0890120E030E008C0009184
:100D0000630B1091640B2091650B3091660BB5015C
:100D1000A4014419550966097709400F511F621F44
:100D2000731F04C07695679557954795CA95D2F776
:100D30004093A7105093A8106093A9107093AA1025
:100D4000453F2FE052076105710528F48CE0809340
:100D5000B510F12C1AC0453F5F4F6105710510F4C5
:100D600080E111C080916F0B9091700BA091710B7D
:100D7000B091720B8093B8109093B910A093BA10F1
:100D8000B093BB1080E28093B5108F2DDF91CF918F
:100D90001F910F91FF90BF90AF909F908F907F9089
:100DA0006F905F904F900895CF92DF92EF92FF92F5
:100DB0001F93CF93DF9310929D1010929A108093FF
:100DC00099100E94F352EB01A89561E0809199106F
:100DD0000E94876089E990E10E94AA782698259A66
:100DE000279A249A2C9A85E080939B1082E58CBDEB
:100DF0001DBC1AE08FEF0E94AF781150D9F720E0A8
:100E000030E0A90160E089E990E10E94BB78182FE9
:100E100080939C10813049F00E94F3526C1B7D0B33
:100E2000613D774060F381E054C02AEA31E040E060
:100E300050E068E089E990E10E94BB7882FF03C03E
:100E400010939D100EC014E00E94B47880939C1003
:100E50001150D1F78A3A11F082E03BC082E08093D2
:100E60009D1080919D10823021F0C12CD12C7601F3
:100E700005C0C12CD12CE12C80E4F82E20E030E01C
:100E8000A90167E389E990E10E94BB78A701960177
:100E900069E289E990E10E94BB7880939C108823E5
:100EA00049F00E94F3526C1B7D0B613D774030F39B
:100EB0008AE00FC080919D10823009F520E030E07B
:100EC000A9016AE389E990E10E94BB78882349F08F
:100ED00088E080939A1089E990E10E94AA7880E0E6
:100EE00016C00E94B478807C803C19F483E0809323
:100EF0009D100E94B4780E94B4780E94B47889E969
:100F000090E10E94AA7883E080939B1081E0DF91BA
:100F1000CF911F91FF90EF90DF90CF9008952F9287
:100F20003F924F925F926F927F928F929F92AF9279
:100F3000BF92CF92DF92EF92FF920F931F93CF93C6
:100F4000DF9310924E088091D00D9091D10DA09119
:100F5000D20DB091D30D81309048A105B10540F07C
:100F60001092D00D1092D10D1092D20D1092D30D7F
:100F7000C091D00D8091870D1816DCF4282F082E13
:100F8000000C330B215031094C2F0C2E000C550B4B
:100F90004217530774F0CFEFC80F8C2F90E0A0E0FA
:100FA000B0E08093D00D9093D10DA093D20DB0936B
:100FB000D30D1092700A80913C08C81714F4C093A6
:100FC0003C0880913C08082E000C990B04962C2FAD
:100FD0000C2E000C330B8217930724F48CEF8C0F2C
:100FE00080933C0810913C08D0E08EE7282E8DE0DD
:100FF000382E9CED892E95E0992EA12CB12C26ED52
:10100000422E26E0522E612C712C35EBE32E38E572
:10101000F32E4EE7C42E4AEAD42E11111DC0809142
:101020005008811106C080913201882309F443C021
:1010300009C0C111F8CF0E94579B8091700A882384
:1010400091F3BEC081E0C11180E024E041ED5DE19B
:101050006D2F0E9425C82FC0113069F5809150086E
:10106000811105C080913201811112C024C0C130AC
:10107000C9F78091820D8C278093820D83E0809345
:1010800032010E947EAA8091700A882359F398C089
:101090008091820D811103C020EC3DE102C024EC5F
:1010A0003DE181E0C13009F080E001E048EC5DE124
:1010B0006D2F0E946CD58091820D882309F478C031
:1010C000123009F073C080915008811106C08091E0
:1010D0003201882309F46AC05AC0C230C1F791E0D6
:1010E00090934E0810924A0810924B0810924C08A8
:1010F00010924D080E94309B23E02093320186EB32
:101100009DE19093DF0D8093DE0D3092DD0D2092F6
:10111000DC0D8092D80D9092D90DA092DA0DB0928C
:10112000DB0D4092D40D5092D50D6092D60D709289
:10113000D70D20E030E04AE754E460917E0D7091D5
:101140007F0D8091800D9091810D0E94A5DC20E0A3
:1011500030E84BEB54E40E9459E00E9456E1609362
:10116000D00D7093D10D8093D20D9093D30DF0924A
:101170003101E0923001D092E20DC092E10D109267
:10118000E00D8091700A882309F4A1CF19C08EE781
:101190009DE00E94CD9E9C0181E0C23009F080E07C
:1011A00000E04CEA5DE16D2F0E946CD583E001C048
:1011B00082E0DF5F1F5FD53009F02FCF8093870D6E
:1011C000DF91CF911F910F91FF90EF90DF90CF9023
:1011D000BF90AF909F908F907F906F905F904F9057
:1011E0003F902F9008951F93CF93DF9310924E0856
:1011F0008091D00D9091D10DA091D20DB091D30DD1
:1012000081309048A105B10540F01092D00D1092A8
:10121000D10D1092D20D1092D30DC091D00D8091AE
:10122000860D1816DCF4282F082E000C330B2150E5
:1012300031094C2F0C2E000C550B4217530774F03C
:10124000CFEFC80F8C2F90E0A0E0B0E08093D00DDE
:101250009093D10DA093D20DB093D30D1092700A3C
:1012600080913C08C81714F4C0933C0880913C0856
:10127000082E000C990B04962C2F0C2E000C330B0F
:101280008217930724F48CEF8C0F80933C08109105
:101290003C08D0E011111AC080915008811106C09D
:1012A00080913201882309F48DC009C0C111F8CFA3
:1012B0000E94579B8091700A882391F38AC081E035
:1012C000C11180E024E044EA5DE179C01130E9F425
:1012D00080915008811106C080913201882309F461
:1012E00071C00BC0C130C1F783E299E60E945C5F18
:1012F0008091700A882381F36CC081E0C13009F0CD
:1013000080E023E04BE95DE15AC01230E9F48091BE
:101310005008811106C080913201882309F452C01F
:101320000BC0C230C1F785EE9CE80E945C5F8091E3
:10133000700A882381F34DC081E0C23009F080E05B
:1013400023E04EE85DE13BC01330E1F480915008AA
:10135000811105C0809132018823A1F10BC0C330F7
:10136000C9F785E39BE80E945C5F8091700A88233F
:1013700089F32FC081E0C33009F080E023E049E821
:101380005DE11DC01430F1F480915008811105C059
:10139000809132018823B1F00BC0C430C9F78DEEC3
:1013A00099E80E945C5F8091700A882389F311C0DC
:1013B00081E0C43009F080E023E040E85DE16D2F7A
:1013C0000E9425C8DF5F1F5FD53009F063CFD0933F
:1013D000860DDF91CF911F910895FF920F931F9378
:1013E000CF93DF9310924E088091D00D9091D10D44
:1013F000A091D20DB091D30D81309048A105B105D7
:1014000040F01092D00D1092D10D1092D20D10928A
:10141000D30DC091D00D8091850D1816DCF4282FC6
:10142000082E000C330B215031094C2F0C2E000CD0
:10143000550B4217530774F0CFEFC80F8C2F90E075
:10144000A0E0B0E08093D00D9093D10DA093D20D89
:10145000B093D30D1092700A80913C08C81714F411
:10146000C0933C0880913C08082E000C990B049610
:101470002C2F0C2E000C330B8217930724F48CEFC7
:101480008C0F80933C0810913C08D0E0FF24F3942B
:1014900011111DC080915008811106C08091320148
:1014A000882309F4D5C009C0C111F8CF0E94579B09
:1014B0008091700A882391F3D2C081E0C11180E04D
:1014C00024E049E75DE16D2F0E9425C8C1C01130BD
:1014D00071F580915008811106C0809132018823F6
:1014E00009F4B6C017C0C130C1F7C0934E081092BE
:1014F0004A0810924B0810924C0810924D0863E174
:101500007EE08FE69DE10E9414D58091700A8823C9
:1015100021F3A5C083E19EE00E94C6C49C0181E046
:10152000C13009F080E000E045E65DE18EC0123098
:1015300071F580915008811106C080913201882395
:1015400009F486C017C0C230C1F7F0924E0810925D
:101550004A0810924B0810924C0810924D0867E10F
:101560007EE08BE59DE10E9414D58091700A88236E
:1015700021F375C087E19EE00E94C6C49C0181E012
:10158000C23009F080E000E041E55DE15EC013306B
:1015900071F580915008811106C080913201882335
:1015A00009F456C017C0C330C1F7F0924E0810922C
:1015B0004A0810924B0810924C0810924D086BE1AB
:1015C0007EE087E49DE10E9414D58091700A882313
:1015D00021F345C08BE19EE00E94C6C49C0181E0DE
:1015E000C33009F080E000E04DE35DE12EC014302F
:1015F00079F580915008811105C0809132018823CE
:1016000039F117C0C430C9F7F0924E0810924A0859
:1016100010924B0810924C0810924D086FE17EE03A
:1016200083E39DE10E9414D58091700A882329F3F9
:1016300016C08FE19EE00E94C6C49C0181E0C430C8
:1016400009F080E000E049E25DE16D2F0E946CD579
:10165000DF5F1F5FD53009F01BCFD093850DDF9181
:10166000CF911F910F91FF9008952F923F924F922B
:101670005F926F927F928F929F92AF92BF92CF9222
:10168000DF92EF92FF920F931F93CF93DF9310920D
:101690004E088091D00D9091D10DA091D20DB091B6
:1016A000D30D81309048A105B10540F01092D00DC6
:1016B0001092D10D1092D20D1092D30DC091D00D79
:1016C0008091840D1816DCF4282F082E000C330BA3
:1016D000215031094C2F0C2E000C550B421753078B
:1016E00074F0CFEFC80F8C2F90E0A0E0B0E08093B3
:1016F000D00D9093D10DA093D20DB093D30D109235
:10170000700A80913C08C81714F4C0933C0880917B
:101710003C08082E000C990B04962C2F0C2E000C64
:10172000330B8217930724F48CEF8C0F80933C08C3
:1017300050903C08D0E043E0442E5EED352E22244C
:10174000239462EFC62E6CE1D62E7AEFA72E7CE1B1
:10175000B72EEAE08E2EEDE19E2EF2E16F2EFDE136
:101760007F2E51101DC080915008811106C08091BC
:101770003201882309F40FC109C0C111F8CF0E94BA
:10178000579B8091700A882391F30CC181E0C111AD
:1017900080E024E042E25DE16D2F0E9425C8FBC09D
:1017A00081E058123DC080915008811106C080919F
:1017B0003201882309F4EFC016C0C130C1F7E12C13
:1017C00010E8F12E07E714E420E030E040E85FE3A2
:1017D0006EE67DE08AE19DE10E944BCE8091700A29
:1017E000882329F3DFC04F923F921F922F928EE6FB
:1017F0009DE09F938F939F928F927F926F92DF9342
:1018000081E0C13009F080E08F930E94DCD5ADB754
:10181000BEB71C960FB6F894BEBF0FBEADBFBBC01F
:10182000B2E05B123DC080915008811106C08091EA
:101830003201882309F4AFC016C0C230C1F7E12CD1
:1018400010E8F12E07E714E420E030E040E85FE321
:1018500062E77DE082E09DE10E944BCE8091700ABC
:10186000882329F39FC04F923F921F922F9282E7C5
:101870009DE09F938F93DF92CF92BF92AF92DF93C1
:1018800081E0C23009F080E08F930E94DCD58DB7F3
:101890009EB70C960FB6F8949EBF0FBE8DBF7BC04F
:1018A00093E0591236C080915008811106C0809192
:1018B0003201882309F46FC01CC0C330C1F7E12C8A
:1018C00010E8F12E07E714E42DEC3CEC4CEC5DE362
:1018D00066E77DE08AEE9CE10E94C8CDAEE2B7E506
:1018E000B0933101A09330018091700A8823F9F2FE
:1018F00059C086E79DE00E947BC59C0181E0C33012
:1019000009F080E000E042EE5CE16D2F0E946CD5B2
:1019100042C0B4E05B123FC080915008811105C005
:10192000809132018823B9F116C0C430C9F7E12C87
:1019300010E8F12E07E714E420E030E040E85FE330
:101940006AE77DE08AED9CE10E944BCE8091700AAF
:10195000882331F327C04F923F921F922F928AE73C
:101960009DE09F938F93AAECBCE1BF93AF93A2ED50
:10197000BCE1BF93AF93DF9381E0C43009F080E016
:101980008F930E94DCD58DB79EB70C960FB6F89456
:101990009EBF0FBE8DBFDF5F5394D53009F0E1CEFF
:1019A000D093840DDF91CF911F910F91FF90EF9015
:1019B000DF90CF90BF90AF909F908F907F906F906F
:1019C0005F904F903F902F900895EF92FF920F936A
:1019D0001F93CF93DF9300D000D0CDB7DEB7109226
:1019E0004E088091D00D9091D10DA091D20DB09163
:1019F000D30D81309048A105B10540F01092D00D73
:101A00001092D10D1092D20D1092D30D1091D00DD5
:101A10008091830D1816DCF4282F082E000C330B50
:101A200021503109412F012E000C550B421753074D
:101A300074F01FEF180F812F90E0A0E0B0E08093CA
:101A4000D00D9093D10DA093D20DB093D30D1092E1
:101A5000700A80913C08181714F410933C08809188
:101A60003C08082E000C990B0496212F012E000C27
:101A7000330B8217930724F48CEF810F80933C087B
:101A8000E0903C08F12CE1101DC0809150088111BC
:101A900006C080913201882309F47AC109C011116E
:101AA000F8CF0E94579B8091700A882391F378C1E8
:101AB00081E0111180E024E043EC5CE16F2D0E9495
:101AC00025C866C181E0E81228C0809150088111C4
:101AD00006C080913201882309F45AC111C0113027
:101AE000C1F720E030E040E251E46AE67DE08DEBB2
:101AF0009CE10E949DD48091700A882351F350C1CB
:101B00008AE69DE00E94FCC59C0181E0113009F04D
:101B100080E000E047EB5CE138C122E0E21228C03F
:101B200080915008811106C080913201882309F408
:101B30002FC111C01230C1F720E030E048EC52E470
:101B400066E67DE08DEA9CE10E949DD48091700A5A
:101B5000882351F325C186E69DE00E94FCC59C01C7
:101B600081E0123009F080E000E043EA5CE10DC161
:101B700083E0E81228C080915008811106C080914E
:101B80003201882309F404C111C01330C1F720E0E9
:101B900030E048EC52E462E67DE08AE99CE10E9494
:101BA0009DD48091700A882351F3FAC082E69DE0AB
:101BB0000E94FCC59C0181E0133009F080E000E048
:101BC00041E95CE1E2C024E0E21236C080915008B5
:101BD000811106C080913201882309F4D9C011C057
:101BE0001430C1F724E630E040E050E062E57DE0EB
:101BF0008AE89CE10E94BAD38091700A882351F34D
:101C0000CFC06091520D7091530D8091540D909101
